:020000040800F2
:10000000C0130020750100087D0100087F01000871
:10001000810100088301000885010008000000003C
:100020000000000000000000000000008701000840
:1000300089010008000000008B0100088D01000804
:100040008F0100088F0100088F0100088F01000850
:100050008F0100088F0100088F0100088F01000840
:100060008F0100088F0100088F0100088F01000830
:100070008F01000845040008152200088F010008C0
:100080008F0100088F0100088F0100088F01000810
:100090008F010008511200088F0100088F0100082D
:1000A0008F0100088F0100088F0100088F010008F0
:1000B0008F0100088F0100088F0100088F010008E0
:1000C0008F0100088F0100088F0100088D210008B2
:1000D0008F0100088F01000800F002F800F03AF8E4
:1000E0000AA090E8000C82448344AAF10107DA4593
:1000F00001D100F02FF8AFF2090EBAE80F0013F0AB
:10010000010F18BFFB1A43F00103184784320000A7
:10011000A4320000103A24BF78C878C1FAD8520738
:1001200024BF30C830C144BF04680C607047000071
:100130000023002400250026103A28BF78C1FBD8F0
:10014000520728BF30C148BF0B6070471FB51FBDA5
:1001500010B510BD00F000F91146FFF7F7FF02F0EF
:10016000D7FB00F01EF903B4FFF7F2FF03BC00F069
:1001700021F900000948804709480047FEE7FEE7EB
:10018000FEE7FEE7FEE7FEE7FEE7FEE7FEE7FEE747
:1001900004480549054A064B70470000191200083B
:1001A000D9000008C00E0020C0130020C00F00209E
:1001B000C00F002040EA010310B59B070FD1042AAD
:1001C0000DD310C808C9121F9C42F8D020BA19BA22
:1001D000884201D9012010BD4FF0FF3010BD1AB187
:1001E000D30703D0521C07E0002010BD10F8013BDC
:1001F00011F8014B1B1B07D110F8013B11F8014B03
:100200001B1B01D1921EF1D1184610BD032A40F2EA
:10021000308010F0030C00F0158011F8013BBCF1A8
:10022000020F624498BF11F801CB00F8013B38BFC0
:1002300011F8013BA2F1040298BF00F801CB38BFCE
:1002400000F8013B11F0030300F04F80083AC0F0C2
:10025000088051F8043B083A51F804CBA0E8081094
:10026000F5E7121D5CBF51F8043B40F8043BAFF3C7
:100270000080D20724BF11F8013B11F801CB48BF21
:1002800011F8012B24BF00F8013B00F801CB48BF57
:1002900000F8012B70474FF0000200B5134694465A
:1002A0009646203922BFA0E80C50A0E80C50B1F1CE
:1002B0002001BFF4F7AF090728BFA0E80C5048BFE2
:1002C0000CC05DF804EB890028BF40F8042B08BF80
:1002D000704748BF20F8022B11F0804F18BF00F87C
:1002E000012B704770477047704710B5203AC0F037
:1002F0000B80B1E81850203AA0E81850B1E8185027
:10030000A0E81850BFF4F5AF5FEA027C24BFB1E863
:100310001850A0E8185044BF18C918C0BDE81040D4
:100320005FEA827C24BF51F8043B40F8043B08BFDD
:100330007047D20728BF31F8023B48BF11F8012BA4
:1003400028BF20F8023B48BF00F8012B704700008F
:10035000004870475C0E00207546FFF7F9FFAE4677
:1003600005006946534620F00700854618B020B5C1
:10037000FFF70EFFBDE820404FF000064FF00007EA
:100380004FF000084FF0000B21F00701AC46ACE83D
:10039000C009ACE8C009ACE8C009ACE8C0098D46AA
:1003A000704710B50446AFF300802046BDE810400A
:1003B000FFF7D9BE01491820ABBEFEE726000200B8
:1003C0007047000000210112CA43014B1A607047B8
:1003D000003C004030B50146A1F12000C0F30B0203
:1003E00085233524101942F2107568431D44B0FB73
:1003F000F5F2B2F5805F01D2104601E040F6FF70E1
:1004000080B230BD30B501460020002300220B121F
:100410000B4C2468CDB204EA0502094C5034246820
:1004200001F0030504EA05442243054C241F246817
:100430001C4014B10AB1012000E0002030BD0000D2
:10044000043C004010B54FF40870FFF7DBFF50B1DB
:100450004FF40870FFF7B6FF0349096888B2FFF749
:10046000B9FF0249088010BD4C3C004080000020CC
:1004700030B10749096841F48001054A116005E07F
:100480000349096821F48001014A116070470000A6
:10049000083C004010B59AB9F723144C6370144B14
:1004A00003EBC0035B5C802444EA13130F4CA3707E
:1004B0000F4B03EBC0035B5C03F00F03E37014E02E
:1004C000012A12D1F723094C6370094B03EBC003D7
:1004D0005B5C002444EA1313044CA370044B03EB4D
:1004E000C0035B5C03F00F03E37010BDBE0100208E
:1004F0002E32000810B5012006490860AE222F21D7
:10050000002000F009F800204FF08441C1F8BC023F
:1005100010BD0000BC02004270B504460D461646F0
:100520004FF480510A4800F04DFB04F00701A0226F
:1005300042EA410000F052FD284600F04FFD3046EF
:1005400000F04CFD4FF48051014800F03EFB70BDBF
:100550000004004010B5012148F2E00000F0DAFC90
:1005600000F074FB40F26711C72000F09BFE10BD45
:1005700010B500F06BFB00F03FF81848007A012836
:1005800012D11648007C01280ED11448407858B981
:100590001248007940B91249086880F3088800BF02
:1005A0004868804700BFFEE70C484078012813D117
:1005B0000A48807A01280FD10848807901280BD198
:1005C0000648007A40B90548007C28B9034880787D
:1005D00010B901200349087010BD0000D8000020A8
:1005E00000E0FF1F7900002030B504460D46294683
:1005F000204600F077FD30BD2DE9FF4100270024A3
:100600000025A04600BF20E000251AE00021324866
:1006100000EB840041553048143000EB8400415514
:100620002D48283000EB840041552B483C3000EB2E
:10063000840041552848503000EB84004155681C27
:10064000C5B2042DE2DB601CC4B2052CDCDB002645
:100650003DE04FF478004FF0804188611F4830F84A
:10066000160088614FF49670039000BF0398411EF6
:1006700003910028FAD11A48006880B22DF81600BC
:1006800006F0FF0800271FE03DF81600154911F895
:10069000172001219140084050B101210E48283017
:1006A00000EB8800C15539464046FFF79DFF09E041
:1006B00000210948283000EB8800C15539464046E2
:1006C000FFF792FF781CC7B2042FDDDB761C052EE6
:1006D000BFD3BDE8FF810000D9000020702F0008C3
:1006E000100400400A3000080448006810B10348B4
:1006F000406808B9012070470020FCE7007000083E
:10070000044800680449884201D101207047002054
:10071000FCE70000006800081234567810B5142277
:1007200004490548FFF772FD142204490448FFF705
:100730006DFD10BD3A300008420D00202630000843
:100740002E0D002001490860704700001418004079
:10075000002123498279002A3AD00A4612680368A8
:100760009A430B461A600A1D126803689A430B1DD0
:100770001A60027911440A6803681A430A60184A29
:100780000832126803689A43154B08331A601A1D21
:10079000126803689A43124B0C331A604279102A8C
:1007A0000ED11A1F126803681A430D4B08331A60E2
:1007B0001A1D126803681A43094B0C331A600DE0C6
:1007C0000749427911440A6803681A430A6005E040
:1007D000027911440A6803689A430A60704700006E
:1007E000001800404FF080400069C0F341003649D6
:1007F00008703648007810B1012862D143E03448CF
:10080000007831490978884205D100202F490870C5
:100810003049087036E02E480078032827D12A484E
:100820000078012802D0022815D109E001202949C9
:10083000087026490870244800782549087014E09B
:100840000220244908700120204908701E480078C1
:100850001F49087009E000201E4908701B490870F4
:10086000194800781A49087000BF00BF09E000204D
:100870001849087015490870134800781449087021
:1008800000BF00BF1DE010480078032818D11148B0
:100890000078012802D0022808D103E001200E4987
:1008A000087003E001200D49087000BF00BF002060
:1008B0000849087005490870034800780449087021
:1008C00000BF00BF704700007A0000207E000020BB
:1008D0007B0000207F0000207C0000207D000020A5
:1008E0003EB50446144A07CA8DE8070001201349A3
:1008F000086004F01F0012490843124908601248BA
:1009000010490C310860114808600E494FF0801002
:100910000DF1010290470020084908604FF4BE0025
:100920000849086007480830006800F0040008B172
:1009300001203EBD0020FCE780330008600C014030
:10094000400D5F7F0078014008DA885190655812A9
:1009500070B5EFF3108000F0010572B60420FFF7C8
:10096000BFFF044605B962B6204670BD70B50446A7
:10097000EFF3108000F0010672B606488047064883
:1009800004600820FFF7ACFF054606B962B62846AA
:1009900070BD00009D3200081078014070B504461B
:1009A000EFF3108000F0010672B606488047064853
:1009B00004600C20FFF794FF054606B962B628468E
:1009C00070BD00009D3200081078014010B5002A6B
:1009D0007CD10D2878D2DFE800F077070B0F1317D2
:1009E0001B1F233F5B6269000A234F4C23706CE09E
:1009F0000A234E4C237068E00A234D4C237064E0B8
:100A00000A234C4C237060E001234B4C23705CE0C4
:100A100001234A4C237058E00123494C237054E0D1
:100A2000484B1B78032B05D10123474C2370474CBF
:100A3000237010E0434B1B78012B04D1444C2370EE
:100A4000444C237007E03F4B1B7823B90123424CF1
:100A50002370424C237038E03A4B1B78032B05D1AE
:100A600001233F4C2370394C237010E0354B1B7829
:100A7000012B04D13B4C2370364C237007E0314BE3
:100A80001B7823B90123384C2370344C23701CE0AD
:100A90002C4B1B7843F001032A4C237015E0294BA3
:100AA0001B7843F00203274C23700EE02F4B1B787A
:100AB000012B05D100232D4C237004E006E003E058
:100AC00001232A4C237000E000BF2BE0012A29D12A
:100AD0000C2825D2DFE800F024060A0E1224242474
:100AE0002424161D0023104C23701AE000230F4C01
:100AF000237016E000230E4C237012E000230D4CEF
:100B000023700EE00F4B1B7823F001030D4C237074
:100B100007E00C4B1B7823F002030A4C237000E023
:100B200000BF00BF10BD00008D0000208C00002021
:100B30008F0000208E0000209200002091000020F5
:100B400090000020960000208500002087000020F3
:100B50008200002084000020880000208A000020FD
:100B600086000020830000208900002098000020DB
:100B700010B5CB43036302F003034FF055346343D6
:100B8000C36210BD30B50B461146DC430463C1F3AC
:100B900001744FF055356C430460C1F30064644246
:100BA0004460C1F301546C438460C1F301446C435D
:100BB000C46001F00F044FF0113504FB05F1016230
:100BC000416230BD0A0482617047816170474161B2
:100BD0007047000070B506460C46154606F0020048
:100BE00008B100F03FFC06F0040020B100201649D7
:100BF000087000F025FC04F0010008B100F058FC7A
:100C000004F0020008B101F049F804F0040008B152
:100C100001F04CF804F0080008B101F066F805F0A6
:100C2000020008B101F040F805F0040008B101F03D
:100C30005BF805F0080008B101F058F806F0010073
:100C400008B100F01DFC70BDC600002010B50121E8
:100C500048F2600000F05EF94FF4003240F6824145
:100C60000748FFF78FFF4FF08052F8219000FFF701
:100C700089FFF8214FF08040FFF7A9FF10BD000069
:100C8000000400400FB5002019E04FF478024FF047
:100C900080439A611F4A32F810209A614FF496728D
:100CA000039200BF039A531E0393002AFAD11A4AF3
:100CB000126840F682431A402DF81020401C052887
:100CC000E3D3002023E0154A32F810203DF810301D
:100CD00082EA0301114A32F810200A400F4B33F820
:100CE00010308B431A430E4B23F810203DF8102090
:100CF0000A4B23F810201A4632F81020094B23F82B
:100D000010201A4632F8102002B100BF401C0528FE
:100D1000D9D30FBD702F000810040040240D00200F
:100D2000100D00201A0D002030B5B2B9052808DCDE
:100D3000144B5B78441E0125A5402B43114C637076
:100D40001FE0062803D101230E4CA37119E00728E8
:100D500017D1FF230B4CA37113E0012A11D10528F1
:100D600008DC084B5B78441E0125A540AB43054CCD
:100D7000637006E0062801D0072802D10023014C49
:100D8000A37130BD2400002070B5002100230F2284
:100D9000C47804B3154C246804F4E064C4F5E0643A
:100DA000210AC1F10403CA40447804FA03F18478AB
:100DB0001440214309010E4C0678A155047804F033
:100DC0001F050124AC4005786D11AD0005F1E0254B
:100DD000C5F8004109E0047804F01F050124AC4087
:100DE000044D0678761145F8264070BD0CED00E004
:100DF00000E400E080E100E002490143024A1160A2
:100E0000704700000000FA050CED00E000200249E8
:100E10008862C86270470000000001400320024958
:100E200088620C20C86270470000014010B512BBF8
:100E3000012806D002280AD003280ED0042818D191
:100E400011E001230D4C23700D4C237012E001239F
:100E50000C4C23700A4C23700CE001230A4C2370C5
:100E60000A4C237006E00123094C2370074C2370C1
:100E700000E000BF00E000BF10BD000082000020C5
:100E800084000020830000208500002087000020CF
:100E900086000020A1B1154A1268C3B21A43134B51
:100EA0001A601A1D1268C0F30F231A430F4B1B1D43
:100EB0001A601A1D126842EA10621B1D1A6013E0C4
:100EC0000A4A1268C3B29A43084B1A601A1D126884
:100ED000C0F30F239A43054B1B1D1A601A1D12689D
:100EE00022EA10621B1D1A60704700003C0C014092
:100EF00010B5020A29B1064B1B681343044C23604A
:100F000004E0034B1B689343014C236010BD0000B9
:100F1000880C014029B1064A12680243044B1A604A
:100F200004E0034A12688243014B1A6070470000D4
:100F3000480C014029B1064A12680243044B1A606A
:100F400004E0034A12688243014B1A6070470000B4
:100F5000900C0140034908600121024A121D1160F2
:100F600070470000080C0140B9B10122114B1A6012
:100F70000822104B583B1A601A46126800F006030C
:100F80001A430C4B583B1A601A46126800F00103D2
:100F90001A43084B583B1A600BE0064A583A12684D
:100FA00002F00802034B583B1A6000221A60014B02
:100FB0001A6070476C0C014018B10121034A11609E
:100FC00002E00021014A1160704700007C0C0140E2
:100FD0000149086070470000340C014001460020C0
:100FE000704710B500F002F810BD00000CB50020ED
:100FF000019000900320354988620C20C86280204F
:10100000334908600846006808604FF401403049E1
:101010002C3108604FF6FC702E4908600F202D49D6
:101020003039086002202C4908600120091F08603F
:1010300000BF29480830006800F0010000900198C6
:10104000401C0190009820B94BF6803101988842ED
:10105000EFD1009888B321482149086000201C493D
:10106000091F086080201A49091D086008460068A9
:10107000086001201649183908602020091F0860FF
:101080000846006808600846006840F001000860F3
:10109000C0201149243108600120091D086000BFEB
:1010A0000D482C3000680328FAD102200849143971
:1010B00008600120091D086002E0FFE700BFFEE7AD
:1010C000002002498862C8620CBD00000000014097
:1010D0001C0C0140300C0040500401401200000381
:1010E00000540140144A02EB8002525C012A11D1E3
:1010F000114A283202EB8002525CE2B900230E4A08
:1011000002EB8002535401230B4A143202EB80029B
:10111000535410E0084A283202EB8002525C012A44
:1011200009D10123044A02EB80025354024A1432CB
:1011300002EB800253547047D900002001464FF063
:10114000E022516100224FF0E0239A6105221A61EA
:1011500000BF4FF0E022106900F001021AB100F464
:101160008032002AF5D04FF0E022126922F001020D
:101170004FF0E0231A61704730B5214C246834B138
:10118000012C06D0022C08D0032C27D103E01D48E7
:1011900026E01D4824E01D4822E0194C083C246844
:1011A00004F01F04641C012505EB5401184C24684D
:1011B000C4F38114C4F103040C2505EB8402104C24
:1011C000241F2468012C04D1104C5443B4FBF1F0CB
:1011D00003E00C4C5443B4FBF1F001E0094800BFBC
:1011E00000BF074C1034246804F07F04641C012500
:1011F00005EB5403B0FBF3F4064D2C6030BD00004A
:10120000080C014000127A00006CDC02001BB700E1
:1012100074040140C000002010B503200949886211
:101220000C20C86240F2BE700749086000200549E2
:101230008862C862FFF7D5FE4FF00060034908607E
:1012400010BD0000000001409404014008ED00E0E2
:1012500010B501210E4800F0A9F8B8B101210C48E1
:1012600000F05AF80B480068401C0A4908600A4818
:101270000068401C0849086008480068401C07498D
:10128000086007480068401C0549086010BD000060
:101290000020004064000020700000206C0000204E
:1012A000680000207FB505460C46012148F2040085
:1012B000FFF730FE174800F03FF80121154800F015
:1012C000AFF80295ADF804400020ADF80C00ADF881
:1012D000060001A90F4800F087F801210D4800F031
:1012E0001BF8012211460B4800F071F815208DF80B
:1012F000000000208DF801008DF8020001208DF81B
:1013000003006846FFF740FD0121024800F008F89D
:101310007FBD000000200040CA4392B202617047C6
:1013200021B1026842F00102026004E002684FF657
:10133000FE731A400260704710B504461748844295
:1013400008D101210220FFF7F5FD00210220FFF75F
:10135000F1FD22E01248844208D101210420FFF768
:10136000E9FD00210420FFF7E5FD16E00D48844269
:1013700008D101210820FFF7DDFD00210820FFF73B
:10138000D9FD0AE00848844207D101211020FFF767
:10139000D1FD00211020FFF7CDFD10BD001C004045
:1013A00000200040002400400028004030B50246E4
:1013B000002000230024156905EA0103D56805EA29
:1013C000010413B10CB1012000E0002030BD10B5C4
:1013D0001AB1C3680B43C36004E0C368CC43A4B232
:1013E0002340C36010BD0000002203689AB24FF68C
:1013F0008F731A404B881A434FF6FF431A400B89EC
:101400001A4302604B68C3620B888362034B9842A5
:1014100001D18B7A0363012343617047001C0040B4
:1014200021B1026842F00402026004E002684FF653
:10143000FB731A400260704710B500F0C3FB10BD8B
:1014400010B501200549C8710020487214210448D4
:10145000FEF721FF00F02EFE10BD0000004001400D
:10146000480E002010B50548807C032805D100F007
:101470004DFE0248C07C0149887410BD480E002012
:1014800010B50648807C032807D00448807C0349B7
:10149000C8740320887400F075FE10BD480E00204B
:1014A00010B500F0A9FB10BD10B500F0DDFB10BDBC
:1014B00070B50020834988730846447C04F004001A
:1014C00018B1002048748049087004F0100028B159
:1014D00080207C49487400207B4908707A48007855
:1014E000002845D104F00100002841D00025082241
:1014F0007649002000F0FCF9002074498860084615
:10150000C08888810020C8810846007800F060000B
:1015100010B900F057F9054615B900F003FC05466F
:10152000002068498873012D04D0022D09D0032DB5
:1015300015D10DE0402063494874012062490870CC
:1015400014E040205F49487402205F4908700DE0B4
:1015500048205C49487400205B49087006E0602020
:101560005849487403205849087000BF00BF00BFA5
:1015700055480078012850D104F0020000284CD1D1
:101580005048447C04F0100018B104F00100002819
:1015900043D102244D4880894D490978884213DAA5
:1015A0004A4882898168802000F0DEF94748C08976
:1015B0004649898908444549C8810020888144F00A
:1015C0000804414908701BE040488168404802789F
:1015D000802000F0C9F93D4880683D4909780844F9
:1015E0003A4988600846808939490978401A37495C
:1015F00088810846C0893649097808443349C8813A
:101600003248C0893149C988884204D144F008046D
:1016100000202D4908702B4844742B48007802287C
:101620004FD12848447C04F00100002849D04024D0
:10163000264880892649097888420FDA234882891A
:101640008168002000F054F92048C0891F49898929
:1016500008441E49C881002088811BE01B4881681E
:101660001B480278002000F043F9184880681849A8
:101670000978084415498860084680891449097822
:10168000401A124988810846C089114909780844DE
:101690000E49C8810D48808988B944F0080400F0DB
:1016A00027FB032805D044F02004032006490870D6
:1016B00002E00020044908700020024988730148B4
:1016C000447470BD00400140C6000020480E002058
:1016D0008C33000810B507484078092806D101204E
:1016E00000F0DEFB08B1032010BD00BF00BF0020EA
:1016F000FAE70000480E002008B53148007800F0F5
:101700006000202839D12E4840780C2834D2DFE8F8
:1017100000F033060C16333333333320272D00F01B
:1017200089FB08B1012008BD26E02548C0880128B2
:1017300004D100F073FB08B10120F4E71CE020485D
:10174000C088012804D100F06BFB08B10120EAE752
:1017500012E0002000F0A4FB08B10220E3E70BE058
:1017600000F092FB08B10320DDE705E000F08EFBFE
:1017700008B10320D7E700BF20E01148007800F04F
:101780006000D8B90E484078062817D10C4AD178A5
:1017900010796A4600F0F8FA0949886008468068BE
:1017A00058B108468089BDF80010884203DDBDF8B5
:1017B0000000034988810120B5E700BF0020B2E79F
:1017C000480E002010B5314840780A285AD2DFE888
:1017D00000F0050F5916591D265930502B48C08866
:1017E000022804D100F014F908B1012010BD4AE02C
:1017F000002000F061F908B10320F7E743E0012081
:1018000000F05AF908B10320F0E73CE01F480078E7
:1018100020B900F037F908B10320E7E733E01B48AF
:101820000078802804D100F0BDF808B10120DDE780
:1018300029E01648007880281AD11448C088012869
:1018400016D11248807C20B1012803D002280FD184
:1018500008E000BF00200E49088008460B49886058
:101860000120C3E709481030084988600120BDE71E
:1018700009E00648007820B900F052F908B10320C9
:10188000B4E700E000BF00BF0020AFE7480E002033
:10189000C400002000F00F0159B1064A917300F016
:1018A00080021AB14022034B5A7402E08022014B9D
:1018B0001A75704700400140014601F00F0292B1D5
:1018C0000A48827301F0800030B10848407C00F083
:1018D000100040B1012070470448007D00F0200056
:1018E00008B10120F7E70020F5E7000000400140C3
:1018F00030B500F00F04064D05EB840304E01C78BE
:1019000001F8014B541EA2B2002AF8D130BD0000EC
:101910002040014000F00F0159B1064A917300F0D8
:1019200080021AB11022034B5A7402E02022014BAC
:101930001A75704700400140F0B504460E46174640
:101940003A463146204600F00FF804F00F053DB14D
:1019500004F0800020B103488573012001494874D8
:10196000F0BD00000040014030B500F00F04064D0E
:1019700005EB840304E011F8014B1C70541EA2B265
:10198000002AF8D130BD00002040014010B51421DC
:101990000248FEF780FC00F055FB10BD480E002009
:1019A0007047000008B51948C078012804D0022803
:1019B00008D0032816D10DE0684600F0DDF9134980
:1019C000886011E011498878694600F0C5F90F492F
:1019D000886009E00D498878694600F00FFA0B49E4
:1019E000886001E0002008BD00BF0848806808B991
:1019F0000020F8E705488089BDF80010884203DD23
:101A0000BDF80000014988810120ECE7480E002064
:101A100038B50020194908801948007800F01F00E7
:101A200020B1012819D0022820D117E01449087CE0
:101A3000694600F091F90446E07900F0400010B1E9
:101A400001200E4908800E48407C28B10B480088D0
:101A500040F00200094908800AE009E008480579D9
:101A60002846FFF729FF0549088001E0002038BD1E
:101A700000BF0248024988600120F8E7C400002046
:101A8000480E00200A48807800F07F010848807CDA
:101A900002280BD00748017019B10120044A907444
:101AA00002E00020024A9074012070470020FCE709
:101AB000480E00200040014070B5054617480078E8
:101AC00000F01F0010B1022824D10DE01348408817
:101AD000012808D115B11149487402E000200F49CE
:101AE0004874012070BD15E00C48408888B90B4847
:101AF000047904F00F0060B11DB1E0B2FFF70AFFF6
:101B000005E0E0B2FFF7C6FEE0B2FFF749FF0120B3
:101B1000E8E700BF00BF0020E4E70000480E002017
:101B200010B51D488478807C012802D002282CD171
:101B30000EE054B1204600F0EBFA40B116480474B0
:101B4000022015498874012010BD0120FCE720E027
:101B50004CB900201049087401208874002000F05E
:101B60001DF80120F0E70C48007CA0420AD0204676
:101B700000F014F8204600F0CBFA28B106480474AF
:101B80000120E1E70120DFE703E0204600F006F84E
:101B900000BF00BF0020D7E7480E00200849C979E0
:101BA00021F00201064AD1711146C97921F00401E0
:101BB000D1711146C97921F00801D1717047000037
:101BC0000040014010B5012148F22000FFF7A2F9C2
:101BD0000322D1024FF08040FEF7CAFF044AD1022F
:101BE0004FF08040FEF7CEFF06200249C87210BDBC
:101BF000030000200040014010B50E20002817DB34
:101C000000F01F0201219140154A430942F82310B8
:101C100000BF00BF00BFBFF34F8F00BF00BF00BFBA
:101C200000BF00BF00BFBFF36F8F00BF00BF00BF8A
:101C300000BF00210846FFF797F9FFF7EFF80948C2
:101C4000006820F01F0007490860FFF7DFF8002058
:101C5000FFF7B2F900214FF40070FFF71BF910BD38
:101C600080E100E09004014010B5012148F220001D
:101C7000FFF750F900224FF4C0514FF08040FEF7BB
:101C800081FF4FF088524FF480518804FEF77AFFAD
:101C90004FF480518804FEF795FF10BD00200149E4
:101CA000086070474000002070470000002007498E
:101CB0000860074908600749086007490860074944
:101CC0000860074908600749086070474400002021
:101CD000480000204C000020500000205800002048
:101CE000540000205C0000207047704770470000DF
:101CF00010B500240A48007800F07F0021280DD19B
:101D00000748007938B106480079012803D0044813
:101D10000079022802D1FFF7DDFC0446204610BD01
:101D2000480E002010B500240A48007800F01F007B
:101D300001280DD10748007938B1064800790128FB
:101D400003D004480079022802D1FFF7D5FC0446ED
:101D5000204610BD480E00200246012A08DA054838
:101D60008078044BDB7840EA032008800148704704
:101D70000020FCE7F72E00080146122008800148E9
:101D800070470000E52E0008034663B9212902D000
:101D9000222928D103E009201080144870474120EF
:101DA00010801348FAE7012B0DD1212902D02229F6
:101DB00019D104E0092010800C481930EEE7DC202E
:101DC00010800C48EAE7022B0DD1212902D02229EC
:101DD00009D104E00920108004483230DEE71820E1
:101DE00010800548DAE70020D8E70000092F000836
:101DF000B02D0008F12D0008CD2E00080246032A60
:101E000008D2054850F8220000780880024850F8AF
:101E1000220070470020FCE70800002000207047E7
:101E200002480349886001207047000060000020DC
:101E3000480E00201148007960B91048C078012888
:101E400008D10E48C088082804D10D480B49886085
:101E5000012070470948007902280DD10748C07851
:101E6000032809D10548C088B0F5807F04D1054812
:101E7000024988600120ECE70020EAE7480E0020D4
:101E80005E0100206F0B002001207047024880781F
:101E90000249087001207047480E002060000020B1
:101EA0002DE9F04106465B48007968B95948C07889
:101EB000022809D15748C088012805D156485549FC
:101EC00088600120BDE8F0815248007902287DD168
:101ED0005048C0780328FAD14E48C08840F608011F
:101EE0008842F4D126B94D484A4988600120E9E783
:101EF0004A4800780728EAD14848407832287DD1FE
:101F00004648807840B94648FEF730FD4548464986
:101F100008604348FEF742FD444F00253F48807863
:101F200007EBC0273D44002445E02846FEF71EFD90
:101F3000FEF70EFD002035E0210201EB80010831A3
:101F4000364A515C3A4A12681144394A11602102FA
:101F500001EB80010931314A515C354A1268114464
:101F6000334A1160210201EB80010A312B4A515C96
:101F70002F4A126811442E4A1160210201EB8001A0
:101F80000B31264A515C2A4A12681144284A1160D2
:101F9000210201EB80010831204A5258224941F8C0
:101FA0002020401C4028C7D32846FEF7F7FC05F543
:101FB0008075601CC4B2082CB7DB01201D49087075
:101FC000164880781549C978884201E01FE015E07D
:101FD00013D1012018490860104840790F49097948
:101FE00000EB01201249098889B2884205D10020FE
:101FF000114908600A48FEF7B9FC00BF074840785D
:10200000302802D10D480E49086001205AE700200F
:1020100058E70000480E002034000020670200202E
:1020200000680008123456780079014000700008FA
:10203000140000203600002018000020A5A5A55A95
:102040003C00002008B501210804FEF723FF012110
:102050004802FEF71FFF01214802FEF749FF002159
:102060004FF40070FEF744FF0120FEF7B1FF01209E
:10207000FEF7A2FF02200D49086001210520FEF7AE
:1020800073FF00200A49C872C87148720E208DF88B
:10209000000001208DF8010000208DF802000120D1
:1020A0008DF803006846FEF76FFE08BD404C014006
:1020B0000040014000200C4908600C4908600C49B0
:1020C00008600C4908600C4908600C4908600C491C
:1020D00008600C49086001200B4948700846C07A26
:1020E00040F00100C872704740000020440000200A
:1020F000480000204C000020500000205400002028
:10210000580000205C0000200040014070470000A3
:102110000146012931D11A4A907300209074082099
:102120001074402050740820507450741046C079C8
:1021300040F00200D07102209073002090740820BB
:102140001074402050740820507450741046C079A8
:1021500040F00400D0710320907300209074082098
:102160001074402050740820507450741046C07988
:1021700040F00800D071012070470020FCE700000B
:102180000040014010B500F0CBF810BD10B54FF481
:102190008020FEF7D7FA1D48006868B91C4800681F
:1021A00000F0040040B10120184908601848006898
:1021B00020F00400164908601448006801280DD179
:1021C0001348006800F0010040B102200F49086088
:1021D0000F48006820F001000D4908600B480068B6
:1021E000022812D10A48006800F0020068B10320FA
:1021F000064908600648006820F0020004490860AB
:1022000000200860232000F013F810BD74000020A7
:10221000444C014070B5054884798578067932468A
:1022200029462046FEF7D6FC70BD00000040014064
:10223000002817DB00F01F02012191400A4A4309E0
:1022400042F8231000BF00BF00BFBFF34F8F00BF95
:1022500000BF00BF00BF00BF00BFBFF36F8F00BF54
:1022600000BF00BF7047000080E100E010B501240E
:1022700072B60948807C02280BD10848006840B932
:10228000092207498220FFF757FB01200349086014
:10229000002462B6204610BD480E00205C000020DD
:1022A000BE01002010B52320FFF7C2FFFEF7B6FDE8
:1022B00002201A4908600120091F086000BF174862
:1022C0000830006800F001000028F8D00120134910
:1022D0002831086000BF11482C3000680328FAD16B
:1022E00001200E4918390860FEF790FD0220FEF724
:1022F00031FE0120FEF760FE01214802FEF7CAFD13
:1023000001210520FEF730FEFEF736FF40F267118F
:1023100040F2E730FEF7C6FF10BD00005004014058
:102320001CB500210846FEF71FFE00214FF4007087
:10233000FEF7B0FD0020FEF73FFE0020FEF70AFE8C
:10234000FEF76CFD002028490860274928390860FD
:10235000091F0860244940390860FEF757FDFEF761
:102360000BFF3B2140F2E730FEF79CFFFEF7C2F87F
:10237000FEF754FD18201C4918310860FEF746FD91
:1023800001210804FEF786FD4FF4706017490860CC
:102390000846006800F47060086001214FF40240B4
:1023A000FEF7B8FD4FF48020009000208DF8040067
:1023B00008208DF8050001208DF806006846FEF71C
:1023C000C7F900200A4908602320002809DB00F033
:1023D0001F02012191404209920002F1E022C2F85D
:1023E000001100BF1CBD000078040140444C0140B6
:1023F00074000020F0B50B460021002432BB284DAC
:102400006D78A3F1E0063543254E757057280FDC33
:10241000244D2D5C2909234D2D5C05F00F06012567
:10242000B540ECB21E4D6D5C25431D4E755435E034
:1024300000F0E005E02D31D1194D6D7800F00F0767
:102440000126BE403543164E757027E0012A25D17E
:10245000134D6D78A3F1E006B543114E7570572802
:102460000FDC104D2D5C29090E4D2D5C05F00F067B
:102470000125B540ECB20A4D6D5CA543084E75547C
:102480000CE000F0E005E02D08D1054D6D7800F07E
:102490000F070126BE40B543014E7570F0BD000028
:1024A000AE010020CE31000810B5012472B60948F3
:1024B000807C02280BD10848006840B910220749E7
:1024C0008220FFF739FA012003490860002462B630
:1024D000204610BD480E002048000020AE0100201C
:1024E00010B552B9084B13F81030084C6370064B06
:1024F00003EB40035B78A37005E0012A03D10023BE
:10250000024C6370A37010BD763200081C000020DE
:1025100010B5012472B60948807C02280BD1084806
:10252000006840B9082207498220FFF705FA012018
:1025300003490860002462B6204610BD480E002002
:10254000440000201C0000202DE9F84104460E46FE
:1025500017464FF000080025B7B906EB8400324952
:10256000085C324911F8008006EB84002E49085CB3
:102570002F490D5C2F4800EB840000F806802E48A0
:1025800000EB8400855508E02A4800EB840010F831
:102590000680294800EB8400855D012D01D0022DC5
:1025A00004D13A462946404600F0BCFB032D05D134
:1025B0003A4629464046FFF793FF32E0052D07D102
:1025C00033463A4629464046009400F031F928E067
:1025D000062D05D13A4629464046FEF7F7F920E098
:1025E000072D05D13A4621463046FDF753FF18E046
:1025F000082D05D13A4629464046FEF717FC10E063
:10260000092D05D13A4629464046FEF78DFB08E0E4
:1026100005F0E000E02804D13A4629464046FFF79D
:10262000E9FEBDE8F881000012300008420D0020EC
:102630002E0D0020560D00206A0D002010B501243B
:1026400072B60948807C02280BD10848006840B95E
:10265000082207498120FFF76FF90120034908602C
:10266000002462B6204610BD480E00204000002025
:102670005E01002070B50024002500260A205D4977
:1026800008705D4908705D4908705D49087008224E
:102690005C495D48FDF78EFD40B1FFF7CFFF28B9DB
:1026A000584859490A6802604968416050225149B6
:1026B0005148FDF77FFD002836D0082429E04E4818
:1026C000005D90B94B48005D5049085C05094948D8
:1026D000005D085C00F00F0101208840C6B2474849
:1026E000405DB0434549485511E04348005D4749C6
:1026F000085C05094048005D085C00F00F010120FE
:102700008840C6B23D48405D30433C494855601C56
:10271000C4B2502CD3DB00F0D3FAC0B950223649F2
:102720003448FDF773FD12E0502235493248FDF779
:1027300041FD60B9102232493048FDF73BFD30B110
:1027400010222F492D48FDF761FD00F0B9FA032052
:102750002F4908702F49087008222D492D48FDF790
:1027600029FD40B1FFF7D4FE28B9294829490A6854
:102770000260496841600A202749087027490870AB
:10278000102225492548FDF715FD38B1FFF78CFECD
:1027900020B9102221492048FDF738FD01202049A9
:1027A00008702049087008221D491E48FDF702FDE7
:1027B00040B100F069FA28B919481A490A6802605C
:1027C00049684160042018490870184908700922B6
:1027D00015491648FDF7EEFC50B1FFF747FD38B933
:1027E000114812490A6802604A684260097A017217
:1027F00070BD0000A70D0020C70100207E0D002045
:10280000F70D0020990000205E010020CE31000865
:10281000A10000201C0000208E0D0020AE01002031
:10282000A9000020240000209E0D0020BE010020F1
:10283000F0B50446059D002A2ED12B48007858B9E2
:102840002A48047005EBC300294E305C294E3070D5
:102850000120294E307046E00020274E3070224E75
:102860003070264E3070012007E0254E365C16B1E0
:102870000126244F3E70461CF0B21028F5DB0120E3
:1028800007E0214E365C16B101261E4F3E70461CF5
:10289000F0B20828F5DB26E0012A24D11B48007895
:1028A000012820D10020194E3070134E30700E4E8A
:1028B0003070124E3070012007E0114E365C16B1B8
:1028C0000126104F3E70461CF0B21028F5DB0120A7
:1028D00007E00D4E365C16B101260A4F3E70461CCD
:1028E000F0B20828F5DBF0BDB4000020B2000020F3
:1028F0001230000897000020B3000020B50000202F
:1029000017020020BA0000202C000020B700002091
:10291000FEF732FC4FF44070FEF76EFAFEF7C4FD8E
:10292000FDF726FEFDF7ECFEBB490870BB48806949
:10293000BB4988420AD0FDF7D7FE38B9B6480078BF
:10294000012803D0B7480078012809D10020B349F5
:102950008861FDF7FFFDFFF719F8FEF76DFD0BE04D
:10296000B148B24908600146086880F3088800BF92
:102970004868804700BFFEE7FDF7D0FE4BE1AC485A
:102980000068002830D00020A9490860FDF72AFF20
:10299000A8480078012805D10020A7494870887010
:1029A000A4490870A548007801280CD10020A3494B
:1029B0000870A3490870E9209F494870002088707A
:1029C00001209C4908709E48007801280CD1002005
:1029D0009A4908709A490870EA209749487000207F
:1029E00088700120934908709648006814283BD3EA
:1029F0000120FDF73DFDFEF745F9002700242EE0FC
:102A0000914830F81400914931F8141080EA010817
:102A100000251BE08E4810F815100120884086B272
:102A200008EA060088B1884830F81400304030B118
:102A3000E9B2E0B20022FFF787FD012705E0E9B225
:102A4000E0B20122FFF780FD00276D1C042DE1DBC1
:102A50007D4830F814007D4921F81400641C052CD1
:102A6000CEDB0020774908607A48807C03282ED18D
:102A700072B67848807C032828D1E7B1FFF712FCB2
:102A80007548407840F00400734948707348006806
:102A90004FF47A71B0FBF1F000EB80004400204667
:102AA000FEF74CFB6C48407820F004006A494870FF
:102AB000FEF7D8FC0AE06A480068032806D1002027
:102AC00067490860FFF7EEFBFEF7CCFC62B665488D
:102AD0000088402802DC4020624908806148008864
:102AE000B0F5656F03DB4FF465605E4908805D48B3
:102AF00000884038242190FBF1F05B4908805B4856
:102B000000880988884212D0042059490870F820AA
:102B10004870322088700020C870534800780871CF
:102B2000002048718871C8710872FFF79FFB4E48FA
:102B300000884E490880FFF79DFD4E480078012827
:102B40001ED100204B490870042049490870F82024
:102B500048703220887048480068012806D100205B
:102B600045490860EE204249C87002E0AA20404969
:102B7000C87000203E498871C8710872FFF776FB63
:102B80003E4800683E49884245D1344800684FF4C9
:102B90007A71B0FBF1F0642100FB01F42046FEF7EE
:102BA000CDFAFEF77DFCFEF77FFC00240CE02B48FD
:102BB00000684FF47A71B0FBF1F0642100FB01F57D
:102BC0002846FEF7BBFA641C142CF0DB00201349E6
:102BD00088612A49086000BF00BF00BF00BF00BF76
:102BE000BFF34F8F00BF00BF00BF1048001D00683B
:102BF00000F4E06023490843001D0C49091D0860EA
:102C000000BF00BF00BFBFF34F8F00BF00BF00BFBA
:102C100000BF00BFFDE7B2E6010000200000014058
:102C2000EB9C374A790000200070000808ED00E0B6
:102C300070000020000000201C0000207C0000200C
:102C40007D00002064000020100D0020C80000203E
:102C5000A82D0008480E002000400140C0000020C0
:102C600074000020800000200200002004000020EA
:102C7000BE01002036000020180000203C0000208B
:102C8000A5A5A55A0000FA0510B5012472B6094899
:102C9000807C02280BD10848006840B90822074907
:102CA0008220FEF749FE012003490860002462B635
:102CB000204610BD480E00204C00002024000020BB
:102CC0001FB501240020009001900290039072B67D
:102CD0001048807C022818D10F480068A8B900204D
:102CE00008E00E49095C0E4A125C11430DF8001011
:102CF000411CC8B21028F4DB102269468220FEF77E
:102D00001BFE012004490860002462B6204604B07E
:102D100010BD0000480E00205000002017020020C7
:102D20007E0D002070B50346F2B9E02B0BDBE72BDC
:102D300009DC1C4C2478A3F1E0050126AE403443A5
:102D4000184D2C702CE002200BE0164C245C9C42A9
:102D500000D108E0134C245C14B9124C235402E057
:102D6000401C0828F1DB1BE0012A19D1E02B0BDB0A
:102D7000E72B09DC0B4C2478A3F1E0050126AE40DB
:102D8000B443084D2C700BE0022007E0054C245C96
:102D90009C4202D10024034D2C54401C0828F5DB32
:102DA00070BD00005E010020070001000A000B005A
:102DB00005010906A101050719E029E7150025010C
:102DC0007501950881027508950181010508750155
:102DD00095051901290591027503950191010507D2
:102DE00019002AFF00150026FF00750895068100CE
:102DF000C00600FF0A00FFA1018504150026FF00A0
:102E0000093075089508810209319102C005010950
:102E100002A10185010901A1000509190129051572
:102E20000025017501950581027501950381010554
:102E3000010930093116018026FF7F751095028146
:102E40000609381581257F750895018106050C0A4C
:102E5000380295018106C0C0050C0901A101850356
:102E600019002AFF02150026FF7F751095038100C7
:102E7000750895018101C00600FF0901A1018506C1
:102E8000150026FF000930950375088102C0050171
:102E90000906A101850A050719E029E715002501A2
:102EA0007501950881021900296715002501750132
:102EB000956881021987298B0990099115002501D0
:102EC000750195078102750195018101C00601FF19
:102ED0000901A1018507150026FF00092075089644
:102EE0000708B102C012010002000000400F320DBD
:102EF000B002100102000109025400030100A032D7
:102F00000904000001030101000921100100012250
:102F1000410007058103400001090401000103018C
:102F2000010009211001000122DC00070582034095
:102F30000001090402000103000200092110010040
:102F4000012218000705830340000104030904104F
:102F5000035500530042002000480049004400107F
:102F60000355005300420020004400460055000075
:102F700008001000200040008000E1141A08151815
:102F80000C12134D2B392D171C302A2F64041607F1
:102F9000090D0E0F335029E2000A0B005134001DB9
:102FA0001B0619103637284FE34B5205114C3238A7
:102FB000E0354EE622232E312DE51E1F202124254B
:102FC00026270101010101010101010101010101A6
:102FD00001010101010101010101010101010101E1
:102FE00003010101010101010101010101010101CF
:102FF00001010101010101010101010101010101C1
:1030000001010101010101010101070001000A00A4
:103010000B00000102030405060708090A0B0C0D4A
:103020000E0F101112130101010101010101010133
:1030300001030101010101010101535455565F6073
:1030400061575C5D5E02595A5B586200006306037B
:10305000030303030303030303030101030000004D
:103060000000010101010101010101010101010152
:1030700001FFFFFFFFFF0101060101010101010145
:103080000101010101FFFFFFFFFF01010601010135
:10309000010101010101010101FFFFFFFFFF020129
:1030A00001060101010101010101020601FFFFFF0B
:1030B000FFFF060606FFFF01FFFF060606FF0606E6
:1030C00006FFFFFFFFFF350F08100006070105028E
:1030D0000403454602FFFFFFFFFF293A3B3C3D3E0C
:1030E0003F4041424344452A4CFFFFFFFFFF2B1462
:1030F000020815171C180C12132F30314BFFFFFF5D
:10310000FFFF39040107090A0B0D0E0F3334322873
:103110004EFFFFFFFFFFE0641D0606190511103684
:103120003738E5084DFFFFFFFFFF0A0C0BFFFF2CB0
:10313000FFFF0B000AFF030904FFFFFFFFFFE1147D
:103140001A0815180C12134D2B392D171C302A2F65
:1031500064041607090D0E0F335029E2000A0B0014
:103160005134001D1B0619103637284FE34B52050A
:10317000114A3238E0354EE63E3F453144013A3B94
:103180003C3D4041424301010101010101010101B6
:10319000010101010101010101010101010101011F
:1031A0000103010301010101030101010101010109
:1031B00001010103010103010101010103010101F9
:1031C0002121210121222121212121212121141527
:1031D000161724252627303132333435363740410F
:1031E00042434445464750515253545556576061E7
:1031F00062636465666770717273747576778081D7
:103200008283848586879091929394959697A0A1C6
:10321000A2A3A4A5A6A7B0B1B2B3B4B5B6B7C0C1B6
:10322000C2C3C4C5C6C7E0E1E2E3E4E5E6E7404E59
:10323000415C005E504C212031104251001122307F
:103240003252431E2E122355335A444D591324250E
:103250003435454615142726373648471617282C87
:103260003800493E1C18291D395D4A3C2D192A2B6E
:103270003A3B3D4B1B1A8301CD00E200E900EA0016
:10328000B700B600B5002302270226022402250259
:103290002A022102940192018A0100002DE9F04FD7
:1032A0003248032181620C21C162DFF8C4C00021D1
:1032B000CCF8001008464FF47A76401CB042FCDB94
:1032C0000122CCF800200020401CB042FCDB294841
:1032D000036843F08003036026482C30036843F4FE
:1032E0002063036091461046224A3C3210608A46B1
:1032F0000846214908602148D0F840031E4F0025A8
:10330000C0F307514FF0FF3B3F1F00225C461046C1
:103310003B685FEAC07806D1A34201D1012400E0F6
:10332000002422441C46401C1428F1DB022A1BD92D
:10333000102901D9103900E000210D48001F026852
:1033400022F07F6242EA01520260CCF800A0002025
:10335000401CB042FCDBCCF800900020401CB04286
:10336000FCDB6D1C052DD0DBBDE8F08F00000140BB
:1033700038040140200C014004B8004000F0FF1F59
:10338000086000BF08680006FCD4704740000000D9
:10339000B033000800000020C8000000140100083D
:1033A00078340008C8000020F8120000300100083E
:1033B00000000000000000004B2F00084F2F000805
:1033C0005F2F000800000000000000000000000067
:1033D00000000000000000000000000000000000ED
:1033E00000000000000000000101000000000000DB
:1033F00000000000000000000000000000000000CD
:1034000000000000000000000000000000000000BC
:1034100001000000000000000000000000000000AB
:10342000000000000000000000000000000000009C
:10343000000000000000000000000000000000008C
:10344000000000000000000000000000000000007C
:10345000000000000000000000000000000000006C
:103460000000000000000000000000000A00000052
:0834700000A24A040000000064
:10700000E8490020ED710008F5710008F7710008EB
:10701000F9710008FB710008FD7100080000000014
:10702000000000000000000000000000FF710008E8
:107030000172000800000000037200089D1501089D
:10704000077200080772000807720008077200083C
:10705000077200080772000807720008077200082C
:10706000077200080772000807720008077200081C
:107070000772000829770008252C0108077200080C
:1070800007720008077200080772000807720008FC
:1070900007720008D116010807720008077200087D
:1070A00007720008077200080772000807720008DC
:1070B0000772000807720008E51A01080772000845
:1070C000077200080772000807720008712B010898
:1070D000077200080772000800F002F800F05CF880
:1070E0000AA090E8000C82448344AAF10107DA4523
:1070F00001D100F051F8AFF2090EBAE80F0013F019
:10710000010F18BFFB1A43F00103184740F20000BB
:1071100060F200000A444FF0000C10F8013B13F03D
:10712000070408BF10F8014B1D1108BF10F8015BE0
:10713000641E05D010F8016B641E01F8016BF9D1D3
:1071400013F0080F1EBF10F8014BAD1C0C1B09D12A
:107150006D1E58BF01F801CBFAD505E014F8016B9C
:1071600001F8016B6D1EF9D59142D6D3704700002E
:107170000023002400250026103A28BF78C1FBD840
:10718000520728BF30C148BF0B6070471FB500F0E1
:1071900062F81FBD10B510BD00F08CF91146FFF765
:1071A000F5FF0CF079FF00F0AAF903B4FFF7F2FF46
:1071B00003BC00F0AFF900000B49D1F800C04A68E9
:1071C0005CF8043B1068184442F8040B8C4528BF57
:1071D000A1F1DC0C8A4228BFA1F1DC02C1F800C099
:1071E0004A6020F0004070478044002009488047F2
:1071F00009480047FEE7FEE7FEE7FEE7FEE7FEE799
:10720000FEE7FEE7FEE7FEE704480549054A064BB0
:107210007047000099160108D9700008E844002062
:10722000E8490020E8450020E84500200B4910B55A
:10723000A1F17C020A4CC2E93712372106E000EBCB
:10724000104342F82130074B00FB03400B1EA1F115
:107250000101F4DC10BD0120E8E70000204400201B
:10726000E119D666CD0D010040EA010310B59B0778
:107270000FD1042A0DD310C808C9121F9C42F8D0A0
:1072800020BA19BA884201D9012010BD4FF0FF3051
:1072900010BD1AB1D30703D0521C07E0002010BD67
:1072A00010F8013B11F8014B1B1B07D110F8013BF3
:1072B00011F8014B1B1B01D1921EF1D1184610BDD4
:1072C00040EA0103024630B59B0710D14FF001346C
:1072D00000E008C208C91D1B9D4315EAC41FF8D071
:1072E00013F0FF0102F8011B0DD01B0AF8E711F89B
:1072F000013B002B02F8013B05D011F8013B002BAC
:1073000002F8013BF3D130BD032A40F2308010F087
:10731000030C00F0158011F8013BBCF1020F624430
:1073200098BF11F801CB00F8013B38BF11F8013BC1
:10733000A2F1040298BF00F801CB38BF00F8013B6E
:1073400011F0030300F07C80083AC0F0088051F887
:10735000043B083A51F804CBA0E80810F5E7121DE9
:107360005CBF51F8043B40F8043BAFF30080D20708
:1073700024BF11F8013B11F801CB48BF11F8012BD4
:1073800024BF00F8013B00F801CB48BF00F8012BF7
:1073900070474FF000020429C0F0128010F0030C77
:1073A00000F01B80CCF1040CBCF1020F18BF00F8F8
:1073B000012BA8BF20F8022BA1EB0C0100F00DB8A7
:1073C0005FEAC17C24BF00F8012B00F8012B48BF05
:1073D00000F8012B70474FF0000200B513469446A9
:1073E0009646203922BFA0E80C50A0E80C50B1F11D
:1073F0002001BFF4F7AF090728BFA0E80C5048BF31
:107400000CC05DF804EB890028BF40F8042B08BFCE
:10741000704748BF20F8022B11F0804F18BF00F8CA
:10742000012B704770477047704710B500F03AF86D
:10743000006810BD10B5044600F034F8046010BDBB
:1074400010B5203AC0F00B80B1E81850203AA0E8FF
:107450001850B1E81850A0E81850BFF4F5AF5FEA33
:10746000027C24BFB1E81850A0E8185044BF18C9E6
:1074700018C0BDE810405FEA827C24BF51F8043B8D
:1074800040F8043B08BF7047D20728BF31F8023BE1
:1074900048BF11F8012B28BF20F8023B48BF00F875
:1074A000012B70470048704788440020004870470F
:1074B000884400207546FFF7F9FFAE46050069468F
:1074C000534620F00700854618B020B5FFF79CFE14
:1074D000BDE820404FF000064FF000074FF00008D5
:1074E0004FF0000B21F00701AC46ACE8C009ACE856
:1074F000C009ACE8C009ACE8C0098D46704710B5BA
:107500000446AFF300802046BDE81040FFF74DBEB3
:107510007047000001491820ABBEFEE726000200BC
:1075200010B5012148F6600005F036FE4FF04052DC
:1075300001211E4803F05CF94FF0405201218807F9
:1075400003F056F905F0D6FA05F09CFB012000F097
:107550006FFA05F08FFB00201549087048704FF452
:10756000602048600020886001200873084600F011
:1075700085F901214FF4087000F054F9012000F062
:1075800071F8012000F05CF800F048FA00BF00F04C
:1075900093F80028FBD100F025FA00BF00F0B8F8FE
:1075A0000028FBD1012000F027FA10BD00040040A4
:1075B0000013002010B5184800681849097888425F
:1075C00028D30020144908601548007810BB1548DE
:1075D0000078F8B9144800880A280BDB002012490B
:1075E000088001201149087001221146002000F096
:1075F00089F907E000200D49087001221146082092
:1076000000F080F908480088401C074908800120E4
:1076100000F0F2F910BD00004C020020AC02002086
:1076200050000020510000202C0000202E000020DF
:1076300000210112CA43014B1A607047003C004010
:1076400030B10749096841F00101054A116005E0C0
:107650000349096821F00101014A116070470000E7
:10766000083C004030B10749096841F48011054ADF
:10767000116005E00349096821F48011014A116095
:1076800070470000083C004030B50146A1F12000E1
:10769000C0F30B0285233524101942F2107568439C
:1076A0001D44B0FBF5F2B2F5805F01D2104601E057
:1076B00040F6FF7080B230BD00200449096801F037
:1076C000040109B1012000E000207047083C00409F
:1076D00030B501460020002300220B120B4C246819
:1076E000CDB204EA0502094C5034246801F00305C8
:1076F00004EA05442243054C241F24681C4014B1AD
:107700000AB1012000E0002030BD0000043C004030
:1077100000200449096801F0080109B1012000E0D6
:1077200000207047083C004070B5002400254FF44D
:107730000870FFF7CDFF00285CD04FF40870FFF70A
:1077400077FF2D49096888B2FFF79EFF2B49088013
:107750002B48007838BB084600882A492A4A127804
:1077600021F8120000BF06E0264830F8150020443A
:1077700084B2681CC5B2082DF6DB2046E11704EB85
:107780005171C1F3CF0420480078401C1E49087095
:1077900008460078082801D1002008701B480480A2
:1077A0001B48048026E0154800881A491A4A1278B6
:1077B00021F81200002506E0164830F81500204494
:1077C00084B2681CC5B2082DF6DB2046E11704EB35
:1077D0005171C1F3CF0410480078401C0E49087065
:1077E00008460078082801D1002008700B48048062
:1077F0000B48048070BD00004C3C0040900200200B
:107800002E000020A01300208E02002086020020FF
:107810008A020020B01300208F020020880200207E
:107820008C02002010B502460020D0B289B1124B64
:107830001B6800F0E00423430F4C23600E4B5033D1
:107840001B6800F0030443EA04430B4C50342360EC
:1078500010E0094B1B6800F0E004A343064C2360D2
:10786000054B50331B6800F0030423EA0443024C29
:107870005034236010BD0000043C00407FB5054635
:1078800000240026684605F0B7FC1A490298B0FBB0
:10789000F1F00121C1EB5000C4B2402040EA0420C5
:1078A0001549086014485038046814480440287882
:1078B00044EA0024104850380460001D0468104851
:1078C0000440D5E901100843697840EA41000443C7
:1078D00009484C38046008482838046824F47004C7
:1078E000287B401EC0B2064344EA065402482838AA
:1078F00004607FBD808D5B00543C0040FFFEF0FFC4
:10790000FDF7F1FF70B503460C4600200021092B5E
:1079100013DD334D2868A3F10A0505EB450607255D
:1079200005FA06F18843A3F10A0505EB450502FABD
:1079300005F108432A4D286010E0294D2D1D2868C7
:1079400003EB4306072505FA06F1884303EB4305DD
:1079500002FA05F10843224D2D1D2860072C13DA89
:107960001F4D28352868651E05EB85061F2505FA7D
:1079700006F18843651E05EB850503FA05F108430A
:10798000174D283528602AE00D2C13DA144D2435C4
:107990002868E51F05EB85061F2505FA06F18843D3
:1079A000E51F05EB850503FA05F108430C4D243569
:1079B000286014E00A4D20352868A4F10D0505EB78
:1079C00085061F2505FA06F18843A4F10D0505EB90
:1079D000850503FA05F10843014D2035286070BD87
:1079E0000C3C00400348006840F008000149086072
:1079F00070470000083C004030B10749096841F475
:107A00008001054A116005E00349096821F48001FD
:107A1000014A116070470000083C004003480068BC
:107A200040F004000149086070470000083C004035
:107A300001490860704700008091204270B50446FB
:107A40000D461646B6B9F72025494870254800EB83
:107A50008500005D802141EA10102149887021488D
:107A600000EB8500005D00F00F00C8701E48007834
:107A7000087117E0012E15D1F720194948701948EF
:107A800000EB8500005D002141EA10101449887068
:107A9000144800EB8500005D00F00F00C87012482C
:107AA000007808711148007840B904200C4908702A
:107AB000042215210A480DF0FBF810E004200849C3
:107AC00008700422152106480DF0F2F850210848EC
:107AD000FFF75FFC0122152105480DF0E9F870BDA4
:107AE000420D0020085E0108200000201F00002039
:107AF000E20C002008B5274800780A2824D18A2003
:107B00002549487025480078887025480078C87055
:107B100088200871002048712248007810B9072099
:107B2000087002E004201C490870042215211A483C
:107B30000DF0BEF850211C48FFF72BFC0122152147
:107B400019480DF0B5F824E0124800780F2814D138
:107B500016490978491E164A1278521E032303FB60
:107B600002110A0213490978323102EB01304FF455
:107B70008072094909F05AFC0BE00F480078009028
:107B800004480378044A094801780948007808F055
:107B900087F908BD11020020FD110020140000200B
:107BA000350000201F000020E20C002013020020FE
:107BB00012020020B90200200D02002000B5C3B05F
:107BC0004FF4807103A8FFF706FC424800780128B3
:107BD0000BD14148007800903E4803783F4A404826
:107BE00001784048007808F083FC3A480078022881
:107BF0000DD1394800783749097803AB374ACDE9C8
:107C00000010374801783748007808F0DDFB31482C
:107C1000007803280BD13048007800902D48037875
:107C20002E4A2F4801782F48007808F02BFC29486D
:107C3000007804280BD12C48007800902548037860
:107C4000264A274801782748007808F067FB214832
:107C5000007805280BD1204800781E4909781F4A72
:107C6000CDE90010D178907803AB08F01FFD1948DA
:107C7000007806280BD11848007816490978174A69
:107C8000CDE90010D178907803AB08F073FC11486F
:107C90000078072801D10BF027FA0E480078082851
:107CA00002D10E4808F0A0FD0A48007809280BD13F
:107CB0000948007807490978084ACDE90010D178C9
:107CC000907803AB08F0B2FD00200249087043B081
:107CD00000BD0000110200200D020020FD10002058
:107CE00013020020120200200E02002008B501201D
:107CF00015490860AE232F220021032000F078F8F8
:107D00000A200CF01FFCB12300221146032000F0D2
:107D10006FF80A200CF016FC4023012200210320FA
:107D200000F066F8FF20D8230022022100900320F3
:107D300000F036F80020D8230246012100900320ED
:107D400000F02EF808BD0000BC0200422DE9F0470B
:107D500081460C4615461E46089F4FF480510F4839
:107D600002F06FFD04F00701A02242EA410008F092
:107D700073F9284608F070F94FF0000805E017F88D
:107D8000010B08F069F908F10108B045F7D34FF489
:107D90008051024802F058FDBDE8F0870004004021
:107DA0002DE9F04781460C4615461E46DDF8208039
:107DB0004FF480510D4802F044FD04F00701A02269
:107DC00042EA410008F048F9284608F045F9002742
:107DD00003E0404608F040F97F1CB742F9D34FF466
:107DE0008051024802F030FDBDE8F08700040040F9
:107DF0002DE9F04107460C4615461E464FF48051CA
:107E00000B4802F01EFD04F00701A02242EA4100E7
:107E100008F022F9284608F01FF9304608F01CF94E
:107E20004FF48051024802F00FFDBDE8F0810000E0
:107E300000040040F02927D1A0F156020E2A20D2DA
:107E4000DFE802F009071F1711150D130B1B0F199F
:107E50001F1D152017E0172015E0022013E0012058
:107E600011E008200FE009200DE007200BE01320AF
:107E700009E0142007E0112005E0122003E04C2067
:107E800001E0002000BF1AE0F1290AD1512803D0F7
:107E9000522803D1122003E0112001E0002000BF8E
:107EA0000DE0F5290AD1512803D0522803D114201E
:107EB00003E0132001E0002000BF00E00020704735
:107EC00010B5012148F2E00005F066F902F002FD6C
:107ED00000F016FF02F06CF8FFF722FB05F0C8F87F
:107EE00040F26711C72009F033FDFFF7FFFE10BD18
:107EF00010B56748007858B966480078664909782F
:107F0000884204DB0020634908700BF0F1FFBEE0FB
:107F100062480088B0F57A7F7EDB00205F490880E8
:107F20005F480078032832D05D48007806282ED0BC
:107F30005B48007802282AD05A4890F8FA010128B4
:107F400018D10220574981F8FA010020C1F8FC013C
:107F50000521544890F8892100F5C5708154514895
:107F600090F88901401C4F4981F88901012081F86E
:107F700024028CE04B48D0F82001B0F57A7FC6D3BC
:107F800000204849C1F820010CF048FF7FE0464836
:107F90000078012818D10020434908705021434837
:107FA000FFF7F7F90122152140480CF081FE404807
:107FB00000210160416002203D4908700222152124
:107FC0003B480CF075FE62E03A480078012824D165
:107FD0003948008808BB002036490870042037491A
:107FE0000870FC2048703648007888700020C870FF
:107FF000087148718871C8710872042215212F48D0
:108000000CF056FE50212948FFF7C3F90122152133
:1080100026480CF04DFE3AE00FE02A48007801288F
:1080200035D0072028490870284800784870072272
:10803000152125480CF03CFE29E01E480078012857
:1080400023D11D48008800BB00201A490870042075
:108050001A490870FC2048701D480078887000207C
:10806000C870087148718871C8710872042215219E
:1080700012480CF01DFE50210C48FFF78AF901222E
:1080800015210A480CF014FE01E000F0B9F910BD0A
:108090001F00002004000020C90200206C02002004
:1080A000B6090020300A0020B4090020E20C0020AC
:1080B000F40100204F0000206E020020420D00203D
:1080C0002A0A00209C090020F40F00201400002040
:1080D0002B0A0020704770477047704770470000B8
:1080E00000B587B0182101A8FFF775F9BA480088D4
:1080F00008B107B000BDB9480078012800D1F8E701
:10810000B74890F8110200280ADD01200CF01AFA95
:10811000B34890F81102401EB14981F81102E8E716
:10812000B0480088B0490988884275D0AD480088B9
:10813000C0EBC00000EB4000AC49085C05286CD0E7
:1081400008DC01280DD0022871D003287BD0042838
:1081500076D1EEE0072874D0132873D01428F7D115
:1081600000E1152101A80CF005FA9DF804008DF836
:10817000050000208DF804009D480188491C9D4899
:10818000FFF707F900209A4908800120944981F8F7
:108190002002002081F8210281F8220281F82302C6
:1081A000012101A800F0DAFA3AE08D4890F82102A6
:1081B000182835DB8A4890F8230238B9012088490D
:1081C00081F82302112008F0E1FB07E00020844938
:1081D00081F82302012101A800F0C0FA00208049A3
:1081E00081F82102084690F82202401C81F8220200
:1081F000084690F82202C82812DB4FF480417E48DE
:1082000002F01FFB4FF47A700CF09CF94FF48041A0
:10821000794802F019FB08E0DCE01DE007E012E01D
:108220006F4890F820020128BFD000BFACE01521B4
:1082300001A80CF09FF9022101A800F08FFAA3E039
:10824000A1E06DE063E0152101A80CF093F9032192
:1082500001A800F083FA97E0152101A80CF08AF933
:1082600063480188491C6348FFF793F80020604980
:10827000088001205A4981F82002002081F821025B
:1082800081F8220281F82302052101A800F066FA94
:1082900036E0534890F82102182831DB504890F816
:1082A000230238B901204E4981F82302192008F031
:1082B0006DFB07E000204A4981F82302052101A84F
:1082C00000F04CFA0020464981F82102084690F857
:1082D0002202401C81F82202084690F82202C82897
:1082E0000EDB4FF48041444802F0ABFA4FF47A7051
:1082F0000CF028F94FF480413F4802F0A5FA04E061
:10830000374890F820020128C3D000BF3CE0152177
:1083100001A80CF02FF9032101A800F01FFA33E0A7
:10832000152101A80CF026F99DF8050000F030F9A0
:108330002AE0152101A80CF01DF904210DF105001A
:1083400000F092FA0C200BF071FA2548D0F82001C9
:10835000B0F57A7F05D300202149C1F820010CF047
:108360005DFD11E0152101A80CF004F91C48D0F8BE
:108370002001B0F57A7F05D300201949C1F820010A
:108380000CF04CFD00E000BF00BF00201449C1F814
:1083900020010C2010490880114890F81E02002886
:1083A00009DD0F4890F81E02401E0D4981F81E029B
:1083B0001E2081F811020A4890F81F02002809DDEA
:1083C000074890F81F02401E054981F81F023C2013
:1083D00081F8110200BF8CE6BC0900204700002094
:1083E000300A0020B2090020B0090020A03000208F
:1083F000000A00204A4100200004004070470000AD
:1084000010B5114800780B281BD2DFE800F0061ADF
:10841000090C1A1A111A1A141700FFF75FFE11E05F
:10842000FFF758FE0EE0FFF75BFEFFF755FE09E091
:10843000FFF753FE06E0FFF7E1FF03E0FFF74BFE17
:1084400000E000BF00BF10BDB609002038B50346EC
:10845000284C247894B9C3EB03146400642594FB7E
:10846000F5F4E3B2C1EB0114640094FBF5F4E1B25E
:10847000C2EB0214640094FBF5F4E2B2002035E094
:108480001D4C245C1D4D2C5D8DF800401A4C245C65
:108490001B4D2C5D8DF80140174C245C194D2C5D53
:1084A0008DF80240144C245C174D2C5D8DF8034070
:1084B0009DF80040012C09D19DF80140134D2B552A
:1084C0009DF8024029559DF803402A559DF800402B
:1084D000022C09D19DF801400D4D2B559DF802400D
:1084E00029559DF803402A55441CE0B20E28C7D3F5
:1084F00038BD0000B902002089620108405E010811
:108500006A5E0108945E0108BE5E010866140020E0
:108510003E15002070B50024002500BF06E010487D
:10852000005D08B1012503E0601CC4B2082CF6DB35
:1085300000BF012D12D1002404E00021084801559C
:10854000601CC4B2082CF8DB0A200BF06FF9012183
:10855000034800F003F90A200BF068F970BD000031
:10856000E80A002010B54121084841714421817179
:10857000C171522101723F2141720D2181720A2184
:10858000C1720A200CF00CFC10BD00000841002054
:1085900010B5044642210C4841714121817154219A
:1085A000C171017245214172522181725921C172FA
:1085B0003D21017344730D2181730A21C1730E2083
:1085C0000CF0EEFB10BD00000841002010B5432167
:1085D000074841714F2181714E21C17101720D21F6
:1085E00041720A21817209200CF0DAFB10BD0000F3
:1085F0000841002010B54321084841714F21817185
:108600004E21C17101723F2141720D2181720A21F7
:10861000C1720A200CF0C4FB10BD0000084100200C
:1086200010B544210A484171492181715321C1711A
:10863000432101724F2141724E218172C1720D217D
:1086400001730A2141730C200CF0AAFB10BD00003D
:108650000841002010B502200D4981F81E01442177
:108660000C484171492181715321C171432101722B
:108670004F214172562181724521C17252210173ED
:108680000D2141730A2181730D200CF089FB10BD6F
:10869000300A00200841002010B50446412120483E
:1086A0004171552181715421C1714F2101725321B2
:1086B00041724C2181724521C17201735021417375
:1086C0003D218173012C13D14521C1734E210174C9
:1086D00041214174422181744C21C17445210175AD
:1086E0000D2141750A21817515200CF059FB15E00B
:1086F00044210B48C1734921017453214174412124
:1087000081744221C1744C210175452141750D21AF
:1087100081750A21C17516200CF042FB10BD0000C6
:108720000841002010B544210B4841714521817159
:10873000C17150210172532141724C218172452136
:10874000C1720173502141730D2181730A21C173DC
:108750000E200CF025FB10BD0841002070B5054629
:108760000E46002441203E49887054213C48C17087
:108770002B21017148214171492181714421C1712D
:108780003D2101724672012E1ED1012411E02A5DA5
:10879000E01D3349891C0A54295D32480155005DAA
:1087A000532804D13C202F49B83981F81102601CAC
:1087B000C4B2082CEBDB0D21294841740A218174D5
:1087C00011200CF0EDFA4AE0022E1DD1012406E042
:1087D0002A5DE01D2249891C0A54601CC4B2032C86
:1087E000F6DB0A2405E000211D48801C0155601CB1
:1087F000C4B20F2CF7DB0D21194841740A21817492
:1088000011200CF0CDFA2AE0052E13D1012406E048
:108810002A5DE01D1249891C0A54601CC4B2102C48
:10882000F6DB0D210E4841760A21817619200CF0E5
:10883000B7FA14E0032E12D1012406E02A5DE01DF0
:108840000749891C0A54601CC4B2082CF6DB0D21B0
:10885000034841740A21817411200CF0A1FA70BD03
:1088600008410020E80A002070B505460E460024A5
:1088700041201349887054211148C1702B21017186
:10888000482141714F2181715321C17154210172DD
:108890003D21417200BF07E02A5D04F1080008494C
:1088A000891C0A54601CC4B2142CF5DB0D21044849
:1088B00041770A2181771D200CF072FA70BD00000B
:1088C0000841002010B504464B210F484171452155
:1088D00081715921C171422101724F21417241219F
:1088E00081725221C172442101733D21417304F10F
:1088F0003000C1B2044881730D21C1730A21017493
:108900000F200CF04DFA10BD0841002010B54B218E
:108910000C484171452181715921C1714221017277
:108920004F214172412181725221C1724421017350
:108930003F2141730D2181730A21C1730E200CF078
:108940002FFA10BD0841002010B54C210B48417191
:10895000452181714421C17150210172412141722F
:10896000472181724521C1723F2101730D2141735D
:108970000A2181730D200CF013FA10BD084100206C
:1089800010B54C2108484171492181715321C171B1
:10899000542101723F2141720D2181720A21C1725D
:1089A0000A200CF0FDF910BD0841002010B54E2141
:1089B00013484171412181714D21C17145210172DD
:1089C0003D214172472181724D21C17201734B21BA
:1089D0004173202181734E21C173752101746D2172
:1089E0004174702181746121C174642101750D216C
:1089F00041750A21817515200CF0D2F910BD0000D7
:108A00000841002010B54E21084841714121817173
:108A10004D21C171452101723F2141720D218172A9
:108A20000A21C1720A200CF0BBF910BD08410020D8
:108A300010B5522108484171452181715321C171FE
:108A400045210172542141720D2181720A21C172A6
:108A50000A200CF0A5F910BD0841002010B55221E4
:108A60000848417153218171C171492101723F212F
:108A700041720D2181720A21C1720A200CF090F915
:108A800010BD00000841002038B5044600200090C9
:108A9000412129484171552181715421C1714F21D2
:108AA0000172532141724C2181724521C1720173BF
:108AB000502141733D218173642094FBF0F03030EC
:108AC000C0B28DF802009DF80200002809DD9DF873
:108AD0000200303800EBC00101EB0010A4EB800075
:108AE00084B20A2094FBF0F03030C0B28DF801005F
:108AF0009DF80100002807DD9DF80100303800EBEB
:108B00008000A4EB400084B204F13000C0B28DF8C4
:108B100000009DF802100848C1739DF8011001740F
:108B20009DF8001041740D2181740A21C174122036
:108B30000CF036F938BD00000841002010B5532173
:108B40000D4841714C2181714521C1710172502143
:108B500041724D2181724F21C1724421017345211F
:108B600041733F2181730D21C1730A2101740F20CC
:108B70000CF016F910BD00000841002010B5552179
:108B800008484171412181715221C1715421017202
:108B90003F2141720D2181720A21C1720A200CF01D
:108BA000FFF810BD0841002010B556210B48417157
:108BB000452181715221C1715321017249214172B4
:108BC0004F2181724E21C1723F2101730D214173EA
:108BD0000A2181730D200CF0E3F810BD084100203C
:108BE00010B52B4890F8F0012A49097888420FD037
:108BF00028480078264981F8F001012026490870AC
:108C0000234890F8F00118B90120214981F8100299
:108C100021480078012839D100201F49087002F04E
:108C20003FFF07F037FA04201C490870F220487013
:108C30001B48007888701B480078C8701A48007874
:108C400008711A48007848711948007888711948E5
:108C50000078C8711848007808720E48007838B952
:108C600004200870042215210C480CF021F80DE0B6
:108C70000422152109480CF01BF850210F48FEF77B
:108C800088FB012215210D480CF012F810BD0000E0
:108C9000300A00201F000020D60200204B0D0020CB
:108CA0001202002013020020B9020020B3020020AB
:108CB000B00200203000002014000020E20C002050
:108CC00008B50D48006880B20090BDF80000C0F300
:108CD000002040B10121094880F83410032102200E
:108CE00000F0B8FA07E00021044880F834100321AE
:108CF000022000F0AFFA08BD100400405C0C002018
:108D000010B5012148F2C00004F046FA4FF4803259
:108D1000D110164801F06CFD4FF080524FF4C04165
:108D2000134801F065FD4FF4C041114801F08EFD7C
:108D30004FF400510E4801F087FD4FF480410C487C
:108D400001F082FD00224FF48041084801F050FDFF
:108D500000224FF40071064801F04AFD00224FF452
:108D60008071034801F044FD10BD00000008004080
:108D70000004004078B50346002096E0524C245C85
:108D8000524D2C5D8DF800404F4C245C504D2C5DB5
:108D90008DF801404C4C245C4E4D2C5D8DF802400A
:108DA000494C245C4C4D2C5D8DF803404B4C247891
:108DB000012C1AD14A4C2478FE2C0CD1494C247831
:108DC000042C04D1464C2478641E454D2C7000249C
:108DD000424D2C7023E0434C2478042C1FD1404C8E
:108DE0002478641C3E4D2C7019E03D4C2478012CF5
:108DF0000CD13C4C2478042C04D1394C2478641CCC
:108E0000374D2C700124354D2C7008E0354C2478FA
:108E1000042C04D1324C2478641E314D2C70304C1B
:108E20002478314D2C709DF80040012C1BD12C462C
:108E300024785C43FF2594FBF5F49DF801502B4EFC
:108E40007455294C24784C43FF2594FBF5F49DF888
:108E500002507455244C24785443FF2594FBF5F4B8
:108E60009DF8035074559DF80040022C1BD11E4CF8
:108E700024785C43FF2594FBF5F49DF801501C4ECB
:108E80007455194C24784C43FF2594FBF5F49DF858
:108E900002507455144C24785443FF2594FBF5F488
:108EA0009DF803507455441CE0B20E28FFF466AFE1
:108EB0000C4C2478641C0B4D2C702C462478042C0C
:108EC00001DD00242C7078BD89620108405E010834
:108ED0006A5E0108945E0108BE5E0108D9020020A6
:108EE0005209002055090020DB02002066140020F2
:108EF0003E15002010B50C4890F8F101012812D160
:108F00000948D0F8F40142F2107188420BD30020D6
:108F10000549C1F8F40181F8F101044800780128FD
:108F200001D0FFF743FD10BD300A00201F000020D4
:108F30002148007A01283DD11F480069B0F57A6FB9
:108F400018D300201C4908611C480078022811D061
:108F50001A48007803280DD00521174890F8892178
:108F600000F5C5708154144890F88901401C1249DD
:108F700081F889011048C06843F2B061884219D372
:108F80000E480078032811D00C48007806280DD030
:108F90000621094890F8892100F5C57081540648DA
:108FA00090F88901401C044981F889010020024998
:108FB0000872C86070470000300A0020B60900201F
:108FC000074890F81D0107490978884207D00548ED
:108FD0000078034981F81D0101200349087070479A
:108FE000300A00201F000020D602002010B52348C0
:108FF000807C022840D12248007901283CD181039D
:10900000204801F015FC00BB4FF400511D4801F051
:109010000FFC012819D11A4890F81402401C184975
:1090200081F81402084690F81402642811DB00202D
:1090300081F81402084690F8130250B9012081F813
:1090400013020020C1F8180203E000200C4981F847
:1090500014020B4890F8130201280DD10848D0F8EB
:10906000180241F28831884206D300200449C1F831
:109070001802022081F8130210BD00008C3000207D
:10908000300A00200008004000B50A4890F80102AC
:10909000142801DD07F000FE064890F802021428AB
:1090A00001DD07F0F9FD04480078132801DD07F021
:1090B000F3FD00BD300A0020B902002070B501F0B8
:1090C00009FC00F03BFB3748007A012812D13548F3
:1090D000007C01280ED13348407858B931480079D6
:1090E00040B93149086880F3088800BF4868804764
:1090F00000BFFEE72B484078012851D12948807AEB
:1091000001284DD127488079012849D12548007A86
:10911000002845D12348007CF0BB22488078D8BB8A
:10912000224800684FF47A71B0FBF1F0642100FB33
:1091300001F4204608F014FA00240CE01B480068F3
:109140004FF47A71B0FBF1F0642100FB01F5284681
:1091500008F006FA641C0A2CF0DB154815498861F2
:1091600000BF00BF00BF00BF00BFBFF34F8F00BFF5
:1091700000BF00BF1048006800F4E0600F490843DA
:10918000001D0D49086000BF00BF00BFBFF34F8F37
:1091900000BF00BF00BF00E002E000BF00BFFDE76E
:1091A00070BD00005C0C002000E0FF1FA80900203B
:1091B000EB9C374A000001400CED00E00000FA058E
:1091C00070B5002400252148007800283CD02048B4
:1091D0000079012838D11E484069142834D30A2068
:1091E0001B4981F8680000BF0BE019481830005D8A
:1091F00028B10021164818300155012503E0601CF4
:10920000C4B2082CF1DB00BF012D05D102221049A8
:10921000183181200AF02EFE002501240AE00C48B6
:109220006830005D20B100210948683001550125F2
:10923000601CC4B2102CF2DB012D05D102220449BE
:10924000683182200BF02EF970BD00001F00002055
:10925000300A002030B504460D461E48807C0228A6
:1092600032D11D4800EB8400415D1B48143000EBF7
:109270008400405D81420FD0174800EB8400415DBF
:109280001548143000EB8400415500211248283065
:1092900000EB840041551BE00F48283000EB8400B0
:1092A000405D401CC1B20C48283000EB84004155A1
:1092B0000948283000EB8400405D022808DB29467D
:1092C000204607F001FE03E02946204607F0FCFD9A
:1092D00030BD00008C300020850C00202DE9F047C7
:1092E0008046894614461E462546E11704EB117157
:1092F00009115A310A032746E11704EB11710911CC
:10930000A4EB011102EB01204FF48072124908F026
:109310008DF8A9F1010101EB8102A8F1010102EB35
:109320000111C91C08034FF480720C4908F07EF843
:10933000700009300949095C70000830074A105C68
:1093400001EB0020064908800846008810B901207A
:1093500004490870BDE8F0878C2E00208C2F002077
:10936000A00900209F0900201448007801280FD18F
:1093700000201249087012480078032803D1012008
:109380000F49087004E00E480078401C0C49087032
:109390000C48007801280FD100200A4908700848BD
:1093A0000078012803D103200549087004E004482F
:1093B0000078401E024908707047000097020020A4
:1093C00013020020980200201448007801280FD1D1
:1093D00000201249087012480078032803D10120A8
:1093E0000F49087004E00E480078401C0C490870D2
:1093F0000C48007801280FD100200A49087008485D
:109400000078012803D103200549087004E00448CE
:109410000078401E02490870704700009402002046
:1094200012020020950200204C48007806281CD12A
:109430004B48008847F23051884216DB00204849EB
:109440000880072045490870002046490880082107
:10945000454890F8892100F5C5708154424890F83C
:109460008901401C404981F889013F4890F8FA0180
:1094700002284AD13C48D0F8FC0143F2B06188424E
:1094800024D300203849C1F8FC01FF2081F8FA01FB
:109490000721354890F8892100F5C570815432487C
:1094A00090F88901401C304981F8890107202B4937
:1094B000087000202B4908802C4908702A48007940
:1094C000012849D100202A49087045E02648D0F8F3
:1094D000FC014FF47A61B0FBF1F201FB1200D8BB42
:1094E0000521214890F8892100F5C57081541E4856
:1094F00090F88901401C1C4981F889010846D0F880
:10950000FC01401CC1F8FC0126E0174890F8240239
:10951000022821D11148007803281DD01248D0F824
:10952000FC014FF47A61B0FBF1F201FB120098B933
:1095300005210D4890F8892100F5C57081540A482D
:1095400090F88901401C084981F889010846D0F843
:10955000FC01401CC1F8FC0170470000B609002066
:109560007002002076020020300A00201402002041
:109570001F00002010B5684800680A287DD300202D
:10958000654908604FF40071644801F051F962497F
:10959000087108464079097988426FD05E48C079E1
:1095A000401C5D49C8710846C079322865DB084611
:1095B000007948710846007978BB032058498874BF
:1095C00008F06EFC64200AF031F9FEF78FFB64208E
:1095D0000AF02CF901205349087053480078B8B1BB
:1095E00052480078032813D014200AF0ABFFFEF78E
:1095F000EDFF052007F06EFA14200AF0A3FF00200B
:10960000454981F88901012008720020C86008617D
:109610000020414981F8130252E0FFE73E480079FB
:1096200001284DD108F082FC64200AF0FFF83C4884
:10963000807C022840D1FEF759FB08F031FC642001
:109640000AF0F4F839480078032804D1FEF762FFE5
:109650000A200AF0EBF804202F4981F8FA011420BF
:109660000AF070FFFEF7DCFF072007F033FA142042
:109670000AF068FF0020284901E047E047E081F850
:109680008901042081F8FA01002026490870284841
:109690000078012802D1002025490870224800786E
:1096A00010B90120234908700020234908601A4995
:1096B000087281F8130203E000201749487108710D
:1096C000154890F81C0208BB0120134981F81C02C0
:1096D00008460079012803D100201249087019E0DA
:1096E00001201049087005210B4890F8892100F5E8
:1096F000C5708154084890F88901401C064981F8DA
:109700008901012008720020C860086102E0002081
:109710000149C87110BD0000300A0020000400405B
:109720008C3000201F00002030000020B6090020EF
:10973000340000203B000020080000202DE9FF41FC
:10974000002700240025A04600BF20E000251AE0E5
:109750000021324800EB840041553048143000EBC2
:10976000840041552D48283000EB840041552B489A
:109770003C3000EB840041552848503000EB840019
:109780004155681CC5B2042DE2DB601CC4B2052C37
:10979000DCDB00263DE04FF478004FF0804188612B
:1097A0001F4830F8160088614FF49670039000BF90
:1097B0000398411E03910028FAD11A48006880B22C
:1097C0002DF8160006F0FF0800271FE03DF81600F0
:1097D000154911F8172001219140084050B101218D
:1097E0000E48283000EB8800C1553946404607F046
:1097F0006BFB09E000210948283000EB8800C155C7
:109800003946404607F060FB781CC7B2042FDDDB09
:10981000761C052EBFD3BDE8FF8100005D0C002043
:109820008A5C0108100400402C5D010808B5002086
:109830007EE04149095C414A515C8DF800103E4987
:10984000095C3F4A515C8DF801103B49095C3D4A77
:10985000515C8DF802103849095C3B4A515C8DF827
:1098600003103A490988B1F57A7F4ADD9DF8001066
:10987000012920D135490988C82291FBF2F101F074
:10988000010159B100219DF80120314B99549DF8F7
:10989000022099549DF8032099540CE000219DF872
:1098A00001202B4B995480219DF8022099540021CE
:1098B0009DF8032099549DF80010022936D12349C0
:1098C0000988C82291FBF2F101F0010159B1002190
:1098D0009DF801201F4B99549DF8022099549DF842
:1098E0000320995422E000219DF80120194B99543E
:1098F00080219DF80220995400219DF8032099545D
:1099000014E000219DF80120114B99549DF802208C
:1099100099549DF8032099549DF801200D4B9954BA
:109920009DF8022099549DF803209954411CC8B217
:109930000E28FFF47EAF08BD89620108405E010871
:109940006A5E0108945E0108BE5E01087402002090
:10995000661400203E15002030B5C1B04FF4807170
:1099600001A8FDF738FD01240120C049087002025A
:1099700001A9002007F05AFDBD480078032805D151
:10998000FF208DF804000020B94908709DF80400FC
:10999000012807D09DF80400022803D09DF8040098
:1099A00003287DD19DF80500012807D09DF805000A
:1099B000022803D09DF805000328F2D100249DF869
:1099C0000400AC4908709DF80500AB49087002F02E
:1099D00001FB4FF4807201A94FF4A04007F026FD6F
:1099E000A5480078401EA3490978491E032202FBBE
:1099F0000100022101EB001001A9085C9F490870D9
:109A00009D480078401E9B490978491E02FB0100D1
:109A100002EB001001A9085C99490870964800788B
:109A2000401E94490978491E02FB0100042101EB04
:109A3000001001A9085C934908708F480078401E07
:109A40008C490978491E02FB0100052101EB001039
:109A500001A9085C8C49087087480078401E854938
:109A60000978491E02FB0100062101EB001001A943
:109A7000085C8649087080480078401E7D49097856
:109A8000491E02FB0100072101EB001001A9085C3F
:109A90007F4981F8010278480078401E754900E04E
:109AA000B4E00978491E02FB01000D2101EB001012
:109AB00001A9085C764981F802026F480078401ECF
:109AC0006C490978491E02FB0100082101EB0010D6
:109AD00001A9085C6F49087067480078401E654915
:109AE0000978491E02FB0100092101EB001001A9C0
:109AF000085C6949087060480078401E5D49097833
:109B0000491E02FB01000A2101EB001001A9085CBB
:109B10006249087058480078401E56490978491E25
:109B200002FB01000B2101EB001001A9085C5C495C
:109B3000087051480078401E4E490978491E02FBC2
:109B400001000C2101EB001001A9085C55490870C7
:109B500049480078401E47490978491E02FB010028
:109B60000E2101EB001001A9085C08B1012000E002
:109B700000204D49087002F0B9F902F05BFA0C229E
:109B800001A94FF4204007F051FC9DF8040009F0B2
:109B900038FE46490870002012E000210CE000EB7E
:109BA00040020A44D21C01AB9A5C00EB4003404DDA
:109BB0002B445A544A1CD1B20329F0DB411CC8B2D1
:109BC0000328EADB2C490978491E2A4A1278521EDA
:109BD000032303FB02110A0228490978323102EB00
:109BE00001304FF4807201A907F020FC2349097865
:109BF00001EBC1012F4A02EB4100102203A9FDF73E
:109C000083FB0120194908702B490870012C25D1CC
:109C10000120184908701849087000201849087078
:109C2000142226492648FDF76FFB142225492648B1
:109C3000FDF76AFB02F072FA07F02EF8234800786D
:109C4000012801D0FEF7B2FE0120114981F81C0164
:109C50001949087002200E4981F8100200201C49A1
:109C600008801C49086041B030BD0000B3020020EC
:109C7000A00200201202002013020020B9020020DE
:109C8000A8020020A9020020A6020020B1020020A4
:109C9000300A002098090020AB020020D3020020E7
:109CA000A7020020B202002021000020C9020020EB
:109CB000CA020020C6170020C20200205C5D010815
:109CC000F2130020485D0108DE1300201F00002071
:109CD0002A0000200800002010B500243848007831
:109CE00001282ED100203649087036490870D82145
:109CF0003548FDF74EFBD8213448FDF74AFB01F00B
:109D0000C3FE33480079012801D108F04FF93148EA
:109D10000078B0B130480078032801D1FEF7FAFB93
:109D200007212B4890F8892100F5C57081542848F7
:109D300090F88901401C264981F8890100200872A9
:109D4000C86026480078401E00EB400024490144CA
:109D500024480078401E0C5C04B9FF24FF2C16D068
:109D600040F25370604320490968B1EB401F0ED3A5
:109D700004F0ACFC01F088FE1C480078012803D0F8
:109D800000201349C1F80C02012018490870174837
:109D90000078012812D10E48D0F80C0214498842EC
:109DA0000CD3144800881E2808DA064800780128D9
:109DB00004D10349087000200B49086010BD000061
:109DC0003C00002030000020661400203E150020DA
:109DD000300A00201F000020B609002012020020D7
:109DE000CA020020130200200800002034000020D6
:109DF00020BF0200140000200CB5002100910BE0F0
:109E00000021019102E00199491C01910199102959
:109E1000F9D30099491C009100998142F0D30CBDFF
:109E200008B5002061E03249095C324A515C8DF886
:109E300000102F49095C304A515C8DF801102C4903
:109E4000095C2E4A515C8DF802102949095C2C4AA4
:109E5000515C8DF803109DF8001001291FD129498C
:109E60000988C82291FBF2F101F0010159B10021EA
:109E70009DF80120244B99549DF8022099549DF897
:109E8000032099540BE080219DF801201E4B99542A
:109E900000219DF8022099549DF8032099549DF8C3
:109EA000001002291FD117490988C82291FBF2F13D
:109EB00001F0010159B100219DF80120134B995483
:109EC0009DF8022099549DF8032099540BE08021BD
:109ED0009DF801200D4B995400219DF802209954C2
:109EE0009DF803209954411CC8B20E289BD308BD8D
:109EF00089620108405E01086A5E0108945E0108FB
:109F0000BE5E010876020020661400203E15002087
:109F100001490860704700001418004000212349DF
:109F20008279002A3AD00A46126803689A430B469F
:109F30001A600A1D126803689A430B1D1A600279A1
:109F400011440A6803681A430A60184A0832126802
:109F500003689A43154B08331A601A1D1268036888
:109F60009A43124B0C331A604279102A0ED11A1FF1
:109F7000126803681A430D4B08331A601A1D1268E1
:109F800003681A43094B0C331A600DE00749427904
:109F900011440A6803681A430A6005E00279114413
:109FA0000A6803689A430A6070470000001800407E
:109FB00010B5012148F2200003F0EEF84FF4803292
:109FC0000621900300F014FC10BD00004FF080400B
:109FD0000069C0F34100364908703648007810B176
:109FE000012862D143E03448007831490978884239
:109FF00005D100202F4908703049087036E02E48FE
:10A000000078032827D12A480078012802D00228A6
:10A0100015D109E001202949087026490870244813
:10A0200000782549087014E00220244908700120B6
:10A03000204908701E4800781F49087009E0002078
:10A040001E4908701B490870194800781A490870A1
:10A0500000BF00BF09E000201849087015490870CA
:10A06000134800781449087000BF00BF1DE0104875
:10A070000078032818D111480078012802D002285E
:10A0800008D103E001200E49087003E001200D49CA
:10A09000087000BF00BF002008490870054908701B
:10A0A000034800780449087000BF00BF70470000F3
:10A0B000800200208402002081020020850200200E
:10A0C000820200208302002010B543480068002867
:10A0D00076D04248007800287CD000203E490860B5
:10A0E0003F48007820B93F48007808B9FFF76EFF75
:10A0F0003D48007801280CD100203B4908703B48BE
:10A100000078012802D10020384908700020384921
:10A1100008603848007801282BD1002035490870A4
:10A12000354908700120304908703448008809F02A
:10A1300077FD38B1314800883149097808442F4902
:10A14000088003E02E4800782C4908802D4890F8BC
:10A15000FA01022804D100202A4981F8240208E0EB
:10A16000284890F82402012803D10220254981F8CB
:10A1700024022148007801282CD100201D490870B4
:10A180001D4908700120184908701C48008809F012
:10A1900047FD38B91948008819490978401A174904
:10A1A000088004E0164800784042144908801548A9
:10A1B00090F8FA01022804D10020124981F8240203
:10A1C00008E0104890F82402012803D102200D492C
:10A1D00081F8240210BD000064020020300000203D
:10A1E000500000205100002000000020340000201A
:10A1F0000800002082020020830200202A000020A4
:10A20000D3020020300A002070B504460E461546E1
:10A21000002D7CD1332C7BD2DFE804F07A201A2683
:10A220002A7A2E32363A7A7A3E7A7A7A7A4A5056B0
:10A230005C6294D0FDFCFBFAF9F8F7F6F5F4F3F262
:10A24000F1F0EFEEEDECEBEA7A7A7AB6E9E8E700C6
:10A250000120F9490870F949087083E20120F849A2
:10A260000870F64908707DE21420F649087079E21A
:10A270001420F549087075E20120F449087071E274
:10A280000120F34908706DE20A20F249087069E282
:10A290000A20F149087065E2F0480078012803D1EE
:10A2A0000020EE49087002E00120EC49087059E2F4
:10A2B0000120EB490870EB49087053E20120EA499C
:10A2C0000870E84908704DE20120E8490870E84943
:10A2D000087047E20120E7490870E549087041E24B
:10A2E0004FF4C871E448FDF754F80020E3490880B2
:10A2F000E3480078032801D1FEF70CF90721E14873
:10A3000090F8892100F5C5708154DE4801E02AE209
:10A3100027E290F88901401CDA4981F88901062179
:10A32000D84890F8892100F5C5708154D54890F837
:10A330008901401CD34981F889010020087281F805
:10A3400024020FE24FF4C871CB48FDF722F8002039
:10A35000CA490880CC48007828B90120CA49087049
:10A360000AF018FE04E00020C74908700AF013FE46
:10A3700001F096FB0020C5490870C5490870C54921
:10A380000880C2490870EDE10120BF4908704FF410
:10A39000C871B948FCF7FDFF0020B84908800521C5
:10A3A000B84890F8892100F5C5708154B54890F8F7
:10A3B0008901401CB34981F88901D3E10020B249E9
:10A3C00008704FF4C871AC48FCF7E3FF0020AB49BC
:10A3D0000880AB48007803282BD1FEF79BF80A20B1
:10A3E00009F024FA0721A74816E094E1ADE177E1EE
:10A3F00012E102E1E6E0C9E0D6E0B9E0AAE09BE0C4
:10A4000080E071E062E053E036E043E09AE195E1FC
:10A4100090E18BE12AE01BE090F8892100F5C570FE
:10A420008154984890F88901401C964981F8890127
:10A4300009E093480078062805D147F23050964944
:10A440000880FEF7F1FF00208E4981F8240289E19F
:10A450000120924908704FF4C8718748FCF799FFB2
:10A46000002086490880FEF7F9FA7BE101208C493B
:10A470000870FEF74BFA75E101208A4908704FF425
:10A48000C8717D48FCF785FF00207C490880FEF7F5
:10A4900077FA67E10120844908704FF4C871764863
:10A4A000FCF777FF002075490880FEF77DFB59E136
:10A4B00001207E4908704FF4C8716F48FCF769FFAE
:10A4C00000206E490880FEF795F84BE1012078499D
:10A4D00008704FF4C8716848FCF75BFF00206749BB
:10A4E0000880FEF78FFA3DE10120724908704FF4B1
:10A4F000C8716148FCF74DFF002060490880FEF7F5
:10A5000055FA2FE101206C4908704FF4C8715A4880
:10A51000FCF73FFF0020594908800821594890F86E
:10A52000892100F5C5708154564890F88901401C76
:10A53000544981F8890115E10120604908704FF400
:10A54000C8714D48FCF725FF00204C490880FEF7F4
:10A55000FBF907E101205A4908704FF4C8714648D9
:10A56000FCF717FF002045490880FDF7FBFFF9E0E5
:10A570000120544908704FF4C8713F48FCF709FFA7
:10A5800000203E490880FEF7F9FAEBE001204E4931
:10A5900008704FF4C8713848FCF7FBFE00203749BB
:10A5A0000880FEF7CBFADDE00120484908704FF43F
:10A5B000C8713148FCF7EDFE002030490880FEF7F5
:10A5C000B1F8CFE00120424908704FF4C8712A4821
:10A5D000FCF7DFFE0020294908803E48007801286A
:10A5E00005D100203B490870FEF756F804E0012031
:10A5F00038490870FEF750F8B4E001203649087079
:10A600004FF4C8711C48FCF7C4FE00201B490880A9
:10A610000120FEF739FAA5E00120304908704FF417
:10A62000C8711548FCF7B5FE0020144908800320C6
:10A63000FDF7AEFF96E00000C0020020C20200203D
:10A64000C10200209C0200209D0200209F020020E9
:10A650009E0200209A0200209B020020A8020020F7
:10A66000940200209602002095020020970200200C
:10A6700099020020980200204A410020000A002090
:10A68000B6090020300A00201F000020140200201C
:10A69000150200202A000020700200203E00002049
:10A6A0003D0000204100002040000020420000202A
:10A6B0004300002044000020450000204700002007
:10A6C00048000020490000204A00002046000020E9
:10A6D0004B000020310000204C0000204D000020E5
:10A6E0004FF4C8712F48FCF754FE00202E49088013
:10A6F0004FF480712D48FCF74CFE2DA12B48FCF740
:10A70000DFFD04212948FEF7AFF80C2009F08EF890
:10A710000AF084FB26E04FF4C8712248FCF739FEAA
:10A7200000202149088007F0BBFB1BE00120FEF759
:10A73000C9F817E00220FEF7C5F813E00320FEF782
:10A74000C1F80FE00AF0CAFC0CE01F4800780128AD
:10A7500003D100201C49087002E001201A4908704A
:10A7600000E000BF1CE0012D1AD1032C06D0042C00
:10A7700008D0082C0ED0092C10D107E00020134976
:10A7800008700CE000201249087008E00020114910
:10A79000087004E000201049087000E000BF00BF0E
:10A7A00070BD00004A410020000A0020540D002026
:10A7B000303132333435363738393031323334355D
:10A7C0003637383900000000390000209C02002094
:10A7D0009D0200209B0200209A02002010B5CB436E
:10A7E000036302F003034FF055346343C36210BDAB
:10A7F00030B50B461146DC430463C1F301744FF0DE
:10A8000055356C430460C1F3006464424460C1F395
:10A8100001546C438460C1F301446C43C46001F093
:10A820000F044FF0113504FB05F10162416230BDA8
:10A830000246002013690B400BB1012000E000200C
:10A8400070470A04826170478161704741617047B7
:10A8500070B504460D46164604F0080008B107F02E
:10A8600099FB04F0020008B107F076FB04F0040045
:10A8700020B100201649087007F05CFB05F00100CC
:10A8800008B107F097FB05F0020008B107F088FF58
:10A8900005F0040008B107F08BFF05F0080008B1CF
:10A8A00007F0A9FF06F0020008B107F07FFF06F0ED
:10A8B000040008B107F09EFF06F0080008B107F099
:10A8C0009BFF04F0010008B107F054FB70BD0000CD
:10A8D000AE09002010B5012148F2600002F05CFCD6
:10A8E0004FF4003240F682410748FFF781FF4FF0F6
:10A8F0008052F8219000FFF77BFFF8214FF0804055
:10A90000FFF7A4FF10BD0000000400407FB5002445
:10A910000026002540E04FF478004FF08041886128
:10A920001F4830F8150088614FF49670039000BFFF
:10A930000398411E03910028FAD11A48006880B29A
:10A940002DF81500EEB2002423E0022E02D1032CD4
:10A9500000D11CE03DF81500134911F81420012125
:10A960009140084048B10121104800EB8600015594
:10A9700021463046FEF76EFC08E000210B4800EB54
:10A980008600015521463046FEF764FC00BF601C7E
:10A99000C4B2042CD9DB6D1C052DBCD37FBD0000D7
:10A9A0008A5C0108100400402C5D0108850C002021
:10A9B00070B500240025002600BFD8E00025D2E0B5
:10A9C000864800EB8400405D01287DD1002183484A
:10A9D00000EB8400415500208149086081480078DF
:10A9E000012803D100207F490870BBE07B48143860
:10A9F00000EB8400405D012867D17B480078401C53
:10AA0000794908700121794800EB8400415505EB34
:10AA100084007749085C05EB8401764A5054142081
:10AA200005EB8401744A5054022C0FD1032D0DD133
:10AA30007248007810B90120704908706F4800789A
:10AA4000022816D103206D49087012E054B94DB99F
:10AA50006B48007868B9012069490870002069498D
:10AA6000088006E0E9B2E0B2002209F0E1F86649A8
:10AA7000087066480078012873D1634800780A2876
:10AA80006FD06148007807286BD0042060490870B7
:10AA9000F82048705F4800EB8400405D802141EA67
:10AAA00010105B4988705B4800EB8400405D00F04B
:10AAB0000F00C870584890F80802087100204871CB
:10AAC0008871C871087201E039E019E053480078D4
:10AAD00038B904200870042215214D480AF0E8F81E
:10AAE0003FE0042215214A480AF0E2F850214C4880
:10AAF000FCF74FFC0122152149480AF0D9F830E053
:10AB000039480078401E384908700021374800EB6A
:10AB100084004155022C13D1032D11D13748007800
:10AB2000012805D102203549087000203D490880E0
:10AB300032480078032814D104203049087010E00E
:10AB400044B93DB92E48007801280AD102202C4989
:10AB5000087006E0E9B2E0B2012209F069F82A497A
:10AB6000087000BF6D1C042DFFF62AAF641C052C75
:10AB7000FFF624AF00240CE0002507E01B4800EBA3
:10AB80008400405D012800D1761C6D1C042DF5DB8E
:10AB9000641C052CF0DB204890F80801012814D132
:10ABA0001D4890F8090101280FD1022E0DD11A4835
:10ABB00090F81C0188B91C48007870B903201A4924
:10ABC000087000201949086007E000201649087045
:10ABD00016490860104981F81C0170BD710C0020F5
:10ABE000080000203400002001000020380B002065
:10ABF000AC5A0108C41900201C1A002016000020BD
:10AC00001A0000201C0000202F0000201502002048
:10AC10004B0D0020085E0108300A00201F000020B4
:10AC2000E20C002018000020A00200206802002092
:10AC30000E48007812280DD10D480078032803DB58
:10AC400000200B49087010E009480078401C0849B2
:10AC500008700AE006480078012803DB0020044958
:10AC6000087002E00120024908707047B902002014
:10AC7000BD02002010B504461E480078012804D10A
:10AC80001D480078012800D110BD1C48007801281B
:10AC90002ED11B48007801282AD1052C04DA002285
:10ACA00011464C2001F032FC052C06DB192C04DC8B
:10ACB00000221146FF20FDF7C9FB192C06DD3C2CB4
:10ACC00004DC2A22AC21FF20FDF7C0FB3C2C06DD72
:10ACD0005A2C04DC0022FF210846FDF7B7FB5A2C52
:10ACE00006DD642C04DC0022FF211046FDF7AEFBDC
:10ACF00000BFC9E7A602002014020020A70200201E
:10AD00003000002000B5094890F8130201280BD14B
:10AD10000648D0F8180241F28831884204D2002255
:10AD2000FF211046FEF726F800BD0000300A002083
:10AD300000B506480078032807D10548008840F68A
:10AD4000B831884201DAFEF771FD00BDB609002076
:10AD50007402002000B506480078072806D105488F
:10AD60000088B0F5FA6F01DAFFF75AF800BD00006D
:10AD7000B60900207602002000202D49097831B95B
:10AD80002C4991F801122C4A1170142005E0294930
:10AD900091F80212284A11701420284909781429C0
:10ADA00011DB2549097819B90021234A117004E003
:10ADB00021490978491E204A11700121204A117049
:10ADC0001E4A117007E01D49097821B11B49097815
:10ADD000491C1A4A11701B490978142911DB1649BC
:10ADE0000978814202DB1449087004E012490978AD
:10ADF000491C114A11700121114A1170114A117038
:10AE000007E01049097821B10E490978491C0D4A1B
:10AE100011700749097829B907490978054A82F864
:10AE2000011204E004490978024A82F802127047CC
:10AE30001F000020300A0020B00200209B020020EA
:10AE4000D60200209A0200201F480078142812DB46
:10AE50001E480078012803DC01201C49087004E02A
:10AE60001A480078401E19490870012018490870D6
:10AE70001549087007E01448007820B1124800789E
:10AE8000401C1149087013480078142812DB0F4841
:10AE90000078142803DB14200C49087004E00B48E8
:10AEA0000078401C094908700120094908700949C7
:10AEB000087007E00748007820B106480078401C79
:10AEC00004490870704700009D020020B302002072
:10AED000B40200209C0200201348007801280FD102
:10AEE00000201149087011480078122803D1002071
:10AEF0000E49087004E00D480078401C0B490870AA
:10AF00000B48007801280ED1002009490870074835
:10AF1000007818B912200549087004E00348007849
:10AF2000401E024908707047C0020020B90200208C
:10AF3000C102002010480078012807D100200E49E6
:10AF400008704FF47A700D49088013E001200A4917
:10AF500008704FF4FA7009490880094800780628FB
:10AF600003DB00200649087004E005480078401C17
:10AF70000349087070470000D4020020C602002078
:10AF8000DE02002000B50848007806280AD10748EC
:10AF9000008847F23051884204DA7F2200210846B7
:10AFA00001F078FE00BD0000B6090020700200200C
:10AFB00018B57B480078012801D101F02BFF7948B2
:10AFC000007801281AD178480078012816D17748EE
:10AFD0000078012812D17648007818B175480078B9
:10AFE000012803D10D2003F027FB02E0002003F02D
:10AFF00023FB0120704981F81D02CFE069480078E9
:10B00000012865D168480078002861D16748007838
:10B0100001285DD167480078002859D1664890F82A
:10B020001D020128E9D1002000210022624B83F893
:10B030001D22624A1278012A01D1012107E05F4AEC
:10B040001278C2EB0222142392FBF3F2D1B2002059
:10B050003BE05B4A125C5B4B9A5C8DF80020584ADF
:10B06000125C594B9A5C8DF80120554A125C574B83
:10B070009A5C8DF80220524A125C554B9A5C8DF80E
:10B0800003209DF80120534B9A5C4A43FF2392FB17
:10B09000F3F29DF801304F4CE2549DF80220234614
:10B0A0009A5C4A43FF2392FBF3F29DF80230E2548C
:10B0B0009DF8032023469A5C4A43FF2392FBF3F258
:10B0C0009DF80330E254421CD0B20E28C1D365E093
:10B0D00034480078002861D13448007801285DD1D7
:10B0E00034480078002859D1334890F81D020128CF
:10B0F00054D10020002100222F4B83F81D222F4A1B
:10B100001278012A01D1012107E02C4A1278C2EB02
:10B110000222142392FBF3F2D1B200203BE0284A32
:10B12000125C284B9A5C8DF80020254A125C264B55
:10B130009A5C8DF80120224A125C244B9A5C8DF8AF
:10B1400002201F4A125C224B9A5C8DF803209DF866
:10B150000120204B9A5C4A43FF2392FBF3F29DF8B7
:10B1600001301C4CE2549DF8022023469A5C4A436D
:10B17000FF2392FBF3F29DF80230E2549DF8032086
:10B1800023469A5C4A43FF2392FBF3F29DF8033077
:10B19000E254421CD0B20E28C1D300BF18BD00003B
:10B1A000A902002014020020D4020020A6020020E0
:10B1B000B9020020A7020020300A0020B0020020BF
:10B1C00089620108405E01086A5E0108945E010818
:10B1D000BE5E01086614002000B50448007818B16E
:10B1E0000248007802F0B4F800BD00009809002081
:10B1F00000B503480078FF2801D005F08DFF00BDA1
:10B200002000002010B517480078022803D1002044
:10B210001449087004E013480078401C1149087074
:10B220004FF4807210494FF4A04006F0FFF80D482B
:10B2300002780E480078401E0D490978491E032304
:10B2400003FB0100082101EB001007490A54052007
:10B2500006F02AF94FF4807203494FF4A04006F03B
:10B260004CF910BD980900208C2D002013020020FD
:10B270001202002038B500200090002441480078D8
:10B28000012862D14048007801285ED13F4800780B
:10B2900040BB00BF23E03E48005D3E49085C8DF89E
:10B2A00001003B48005D3C49085C8DF802003848CD
:10B2B000005D3A49085C8DF80300394800789DF834
:10B2C0000110384A5054384800789DF80210505404
:10B2D000364800789DF803105054601CC4B20E2C00
:10B2E000D9D332E000242EE02948005D2949085CCA
:10B2F0008DF801002648005D2749085C8DF80200A2
:10B300002348005D2549085C8DF80300A01C00EB74
:10B3100040002749085C9DF80110224A5054A01CA7
:10B3200000EB40002249084440789DF80210505438
:10B33000A01C00EB40001E49084480789DF80310D3
:10B340005054601CC4B20E2CCED3002511E0194815
:10B35000405D60B1174A1849284604F0A1F8154825
:10B36000405D401E13494855012014490870681C6F
:10B37000C5B2582DEBDB11480078012801D104F04B
:10B3800069F838BDA602002014020020BD0200208A
:10B39000896201086A5E0108945E0108BE5E0108C8
:10B3A000B602002066140020B7020020B802002078
:10B3B000A16001081C1A0020C4190020D502002039
:10B3C00038B5002000900024002544E05048405D3E
:10B3D00000283ED04F48007801282DD14C48405DD0
:10B3E000142829D100204C4908704C4908704C4958
:10B3F0000870FBF7E1FE072190FBF1F201FB120060
:10B40000484908700846007800EB40004649085C4F
:10B41000414908704348007800EB40004249084425
:10B4200040783E4908703F48007800EB40003E49B4
:10B43000084480783A490870354A3C49284603F068
:10B440006BFF3348405D401E314948550120384963
:10B450000870681CC5B2582DB8DB35480078012843
:10B4600001D103F0F7FF3348007801282CD132488E
:10B470000078012828D1002423E03048005D3049BD
:10B48000085C8DF801002D48005D2E49085C8DF8A0
:10B4900002002A48005D2C49085C8DF803001E4814
:10B4A00000789DF80110294A50541C4800789DF8F6
:10B4B000021050541A4800789DF803105054601C34
:10B4C000C4B20E2CD9D322E000241EE01B48005D3C
:10B4D0001B49085C8DF801001848005D1949085C9B
:10B4E0008DF802001548005D1749085C8DF80300CF
:10B4F00000209DF80110154A50549DF80210505438
:10B500009DF803105054601CC4B20E2CDED338BD1D
:10B510001C1A0020BD020020B6020020B702002045
:10B52000B8020020B50200208C600108C419002078
:10B53000D5020020A6020020140200208962010822
:10B540006A5E0108945E0108BE5E01086614002070
:10B5500038B500200090002441480078012862D1CD
:10B560004048007801285ED13F48007840BB00BFCA
:10B5700023E03E48005D3E49085C8DF801003B48F1
:10B58000005D3C49085C8DF802003848005D3A498E
:10B59000085C8DF80300394800789DF80110384A9E
:10B5A0005054384800789DF80210505436480078BE
:10B5B0009DF803105054601CC4B20E2CD9D332E055
:10B5C00000242EE02948005D2949085C8DF801001F
:10B5D0002648005D2749085C8DF802002348005D7D
:10B5E0002549085C8DF80300A01C00EB40002749AA
:10B5F000085C9DF80110224A5054A01C00EB40004A
:10B600002249084440789DF802105054A01C00EBD9
:10B6100040001E49084480789DF803105054601C77
:10B62000C4B20E2CCED3002511E01948405D60B1A4
:10B63000174A1849284603F04FFA1548405D401E46
:10B6400013494855012014490870681CC5B2582D8B
:10B65000EBDB11480078012801D103F0FBFE38BD77
:10B66000A602002014020020BD0200208962010809
:10B670006A5E0108945E0108BE5E0108B602002001
:10B6800066140020B7020020B8020020A160010863
:10B690001C1A0020C4190020D502002010B538481B
:10B6A0000078132869D2DFE800F00A0D12171C1F7A
:10B6B000222B34373A3D4556595C5F62650003F0F2
:10B6C00005F85BE02F48007800F0B6F956E02D4809
:10B6D000007800F0B1F951E02A48007800F0ACF9A8
:10B6E0004CE000F07FF949E000F056F846E02648CB
:10B6F0000278264801782648007800F063F83DE09B
:10B7000021480278214801782148007804F048FB5C
:10B7100034E0FFF71DFF31E0FFF752FE2EE0FFF7A8
:10B72000A9FD2BE01B48007802F084FA012019499A
:10B73000087023E013480078012804D115480078E8
:10B7400002F03EFB03E01348007802F073FA012098
:10B750001049087012E000F01FF90FE000F006F940
:10B760000CE000F05FF809E000F084F806E000F07B
:10B77000B7F803E000F0D8F800E000BF00BF10BD4C
:10B78000B9020020BD020020B8020020B70200204C
:10B79000B6020020BA02002000B50948007801F086
:10B7A0006BFE07480078FF2803DB0020044908707F
:10B7B00004E003480078401C0149087000BD000007
:10B7C000BA02002070B504460D46164612480178AC
:10B7D0001248007801F042FF1148007801280DD18D
:10B7E0000E480078401C0D49087008460078FF2874
:10B7F00011D1087000200A4908700CE00748007851
:10B80000401E064908700846007820B900200870DC
:10B8100001200349087070BDBC020020BA0200205C
:10B82000BE02002010B51148007818B91048007801
:10B8300001F09CFF03F00EFE0C480078052808DBA1
:10B8400000200A4908700A480078401C084908701E
:10B8500004E006480078401C044908700448007859
:10B86000072802DB00200249087010BDBA02002040
:10B87000BC02002010B51848007802F0EFF8164816
:10B880000078401C1449087008460078012802D14D
:10B890001E201249088010480078052802D1322065
:10B8A0000E4908800C480078132802D11E200B494D
:10B8B0000880094800781D2802D11E200749088009
:10B8C000054800784C2806DB0020034908704FF437
:10B8D000FA700249088010BDBA020020C40200209C
:10B8E00010B50F4801780F48007802F0FFFE0C48B1
:10B8F000007805280DDB0020094908700948007808
:10B9000018B901200749087008E0002005490870AF
:10B9100004E003480078401C0149087010BD000095
:10B92000BA020020DF02002010B50C4803780C4852
:10B9300002780C4801780C48007803F039FC0A487A
:10B940000078142803DB14200749087004E0064837
:10B950000078401C0449087010BD0000B8020020A7
:10B96000B7020020B6020020BA02002010B5094834
:10B97000007801F09DFF074800780F2803DB0020C6
:10B980000449087004E003480078401C014908702D
:10B9900010BD0000BA02002010B510480178104810
:10B9A000007802F091FF0E480078122808DB002092
:10B9B0000B49087009480078401C0849087004E0E9
:10B9C00007480078401C064908700448007807289A
:10B9D00002DB00200149087010BD0000BC020020FD
:10B9E000BA02002000B511480278114801781148C8
:10B9F000007803F05DF90E480078082808DB002085
:10BA00000B49087009480078401C0849087004E098
:10BA100007480078401C06490870044800780C2844
:10BA200002DB00200149087000BD0000BC020020BC
:10BA3000BA020020BD02002010B50446104802786A
:10BA400010480178204603F0F3FD0E4800780828DE
:10BA500008DB00200B49087009480078401C0849A1
:10BA6000087004E007480078401C06490870044844
:10BA70000078242802DB00200149087010BD000076
:10BA8000BC020020BA02002008B50448D8230022D6
:10BA9000012100900846FCF759F908BD6614002002
:10BAA00030B5B9B07148007828B9714890F80102F2
:10BAB0007049087004E06E4890F802026D49087001
:10BAC0006C480078012801D1012507E06948007819
:10BAD000C0EB0020142190FBF1F085B2002403E0BC
:10BAE00003A90D55601CC4B2D82CF9DB624800785C
:10BAF00001283FD100243BE004EB84005F49084467
:10BB0000407898B304EB8400085C5D49085C012828
:10BB10002CD15C480078C0EB0020142190FBF1F0A0
:10BB200004EB8401554A515C574A515C03AA5054B6
:10BB300054480078C0EB0020142190FBF1F004EB96
:10BB400084014E4A515C514A515C03AA50544D48FD
:10BB50000078C0EB0020142190FBF1F004EB84018D
:10BB6000464A515C4A4A515C03AA5054601CC4B214
:10BB70002A2CC1DB4748047804EB8400464908447A
:10BB8000407898B304EB8400085C3D49085C0128C8
:10BB90002CD142480078C0EB0020142190FBF1F03A
:10BBA00004EB84013C4A515C374A515C03AA50546F
:10BBB0003A480078C0EB0020142190FBF1F004EB30
:10BBC0008401354A515C314A515C03AA50543348D0
:10BBD0000078C0EB0020142190FBF1F004EB84010D
:10BBE0002D4A515C2A4A515C03AA50542C480078D3
:10BBF000012803D02B48007801282CD1002428E00C
:10BC00002948005D1E49085C8DF808002648005D43
:10BC10001D49085C8DF809002348005D1B49085C3C
:10BC20008DF80A002048005D1949085C8DF80B006A
:10BC30009DF8080001280AD1FF209DF8091003AAE9
:10BC400050549DF80A1050549DF80B105054601C2D
:10BC5000C4B20E2CD4D303A8D82300220221009012
:10BC60000120FCF773F839B030BD00001F00002040
:10BC7000300A0020B0020020A9020020741A00201F
:10BC8000405E0108B10200206A5E0108945E01086E
:10BC9000BE5E010820000020461B0020B2020020EA
:10BCA000A6020020A70200208962010800B5C1B0E9
:10BCB0004FF4807101A8FBF78EFB7E490978491E7D
:10BCC0007D4A1278521E032303FB02110A027B49AC
:10BCD0000978323102EB01304FF4807201A905F08E
:10BCE000A5FB7649097801EBC101754A02EB4100D9
:10BCF000102203A9FBF708FB7048007800EBC00096
:10BD00006F4911F810006F4908706C48007800EB1B
:10BD1000C0006B4901EB400080786B4908706748B0
:10BD2000007800EBC000664901EB4000C07967492C
:10BD300008706248007800EBC000614901EB4000E8
:10BD4000007A634908705D48007800EBC0005C49E8
:10BD500001EB4000407A5F4908705848007813288A
:10BD600075D2DFE800F00A152029323B444D5158C6
:10BD70005F666D757E858E959C0000205249087027
:10BD800055490870554908700520554908808EE0CE
:10BD900000204D490870504908705049087028200B
:10BDA0004F49088083E000204B4908704B490870D8
:10BDB00014204B4908807AE0002047490870474921
:10BDC000087014204649088071E00020424908703C
:10BDD000424908700A204249088068E000203E4934
:10BDE0000870404908700A203D4908805FE0002043
:10BDF000394908703B4908700A203949088056E0E3
:10BE000064203749088052E0002037490870142028
:10BE1000334908804BE00020334908701420304932
:10BE2000088044E000203049087014202C49088024
:10BE30003DE028202A49088000202749087036E084
:10BE40001420274908800020234908702FE02DE0A6
:10BE500000202149087021490870282020490880C5
:10BE600025E000201C49087032201D4908801EE092
:10BE700000201949087019490870282018490880BD
:10BE800015E00020144908703220154908800EE0A2
:10BE900000201149087096201149088007E0002011
:10BEA0000D49087014200E49088000E000BF00BF53
:10BEB00041B000BD1302002012020020B902002090
:10BEC000C6170020B3020020BD020020B6020020E9
:10BED000B7020020B8020020BA020020BC020020F5
:10BEE000C4020020BE020020D502002010B50024AC
:10BEF00065E034490978491E01EB8102324909782D
:10BF0000491E02EB0111891C090301EB04204FF4C7
:10BF100080722E4905F08AFA00204CE000EB800187
:10BF200008312A4A515CC4EBC40202EB420200EB26
:10BF3000420202EB8202264B1A44517000EB800150
:10BF40000931224A515CC4EBC40202EB420200EB0D
:10BF5000420202EB8202995400EB80010A311B4A33
:10BF6000515CC4EBC40202EB420200EB420202EB62
:10BF700082021A44917000EB80010B31134A515C2C
:10BF8000C4EBC40202EB420200EB420202EB82026B
:10BF90001A44D17000EB80010C310C4A515CC4EBA7
:10BFA000C40202EB420200EB420202EB82021A449C
:10BFB0001171411CC8B22A28B0DB601CC4B2012C2C
:10BFC00097DB10BD13020020120200208C2D0020F0
:10BFD000741A002010B512490978491E01EB81023C
:10BFE00010490978491E02EB0111491C08034FF45E
:10BFF00080720D4905F01AFA00240DE00A4904F197
:10C000000800085C09490855074904F11C00085C50
:10C0100007490855601CC4B2142CEFDB10BD0000AA
:10C020001302002012020020FD110020DE13002068
:10C03000F213002010B5002465E034490978491E48
:10C0400001EB810232490978491E02EB0111091DF9
:10C05000090301EB04204FF480722E4905F0E6F944
:10C0600000204CE000EB800108312A4A515CC4EB0F
:10C07000C40202EB420200EB420202EB8202264BB8
:10C080001A44517000EB80010931224A515CC4EB23
:10C09000C40202EB420200EB420202EB820299541C
:10C0A00000EB80010A311B4A515CC4EBC40202EB75
:10C0B000420200EB420202EB82021A44917000EB52
:10C0C00080010B31134A515CC4EBC40202EB420203
:10C0D00000EB420202EB82021A44D17000EB8001B5
:10C0E0000C310C4A515CC4EBC40202EB420200EB7F
:10C0F000420202EB82021A441171411CC8B22A2882
:10C10000B0DB601CC4B2012C97DB10BD1302002011
:10C11000120200208C2D0020461B002070B5002448
:10C1200004E00020F0490855601C84B2FF2CF8DDC3
:10C13000002005F0B9F90120EB4908704870022091
:10C1400088700020C870087148714FF4807205F043
:10C15000D4F9002404E00020E3490855601C84B2AF
:10C16000FF2CF8DD052005F09FF901249CE0012556
:10C1700095E0681E611E032303FB0100DA4901EB11
:10C1800000100470681E611E03FB0100012101EB19
:10C190000010D5490D54601E032101FB0050C2B2AE
:10C1A000681E611E03FB0100022101EB0010CE4955
:10C1B0000A540022681E611E03FB010003EB0010FD
:10C1C000C9490A54681E611E03FB0100042101EBEA
:10C1D0000010C5490A54681E611E03FB01000521B9
:10C1E00001EB0010C0490A540122681E611E03FBC6
:10C1F0000100062101EB0010BB490A541422681EFD
:10C20000611E03FB0100072101EB0010B6490A542F
:10C210000022681E611E03FB0100082101EB0010D3
:10C22000B1490A540822681E611E03FB010009215E
:10C2300001EB0010AC490A540122681E611E03FB89
:10C2400001000A2101EB0010A7490A54681E611E73
:10C2500003FB01000B2101EB0010A3490A54142237
:10C26000681E611E03FB01000C2101EB00109E49BA
:10C270000A541222681E611E03FB01000D2101EB0E
:10C28000001099490A540022681E611E03FB010038
:10C290000E2101EB001094490A54681C85B2032D4D
:10C2A0007FF767AF601C84B2032C7FF760AF4FF459
:10C2B00080728D494FF4A04005F01FF901208B4991
:10C2C000087000240CE08A48015D874A04F10800E8
:10C2D00011548848015D04F11C001154601C84B2A3
:10C2E000142CF0DB01241EE0012518E0691E01EB8F
:10C2F0008102611E02EB0111491CC8B205F0D4F89D
:10C30000691E01EB8102611E02EB0111491C080349
:10C310004FF48072744905F0F0F8681C85B2032D63
:10C32000E4DD601C84B2032CDEDD002404E0002088
:10C330006D490855601C84B2FF2CF8DD002494E0A0
:10C34000012004EBC4016C4A02F81100664908722E
:10C35000002004EBC40102EB4101487062494872BD
:10C3600004EBC40102EB410188705F49887204EB61
:10C37000C40102EB4101C8705B49C87204EBC401FF
:10C3800002EB410108715849087304EBC40102EB48
:10C39000410148715449487304EBC40102EB410167
:10C3A00088715149887304EBC40102EB4101C871E3
:10C3B0004D49C87304EBC40102EB410108724A49BC
:10C3C0000874FF2004EBC40102EB410148724649A6
:10C3D0004874022C19D0032C17D0042C15D0062C2D
:10C3E00013D0072C11D0082C0FD00B2C0DD00C2CF7
:10C3F0000BD00E2C09D0102C07D0112C05D0092CF5
:10C4000003D00A2C01D00F2C0ED1012004EBC40163
:10C41000394A02EB4101887004EBC400114601EB7C
:10C42000400080783049887204F13201C8B205F0CA
:10C430003BF8002515E004F13201090301EB05206A
:10C440004FF48072284905F058F804F132010903CD
:10C4500001EB05204FF48072234904F0E7FF681CCC
:10C4600085B2092DE7DB601C84B2132CFFF668AFA0
:10C4700000201D490870002505E0FF21E81C1A4A2C
:10C480001154681C85B2092DF7DB0A2005F00CF861
:10C490004FF4807214494FF4204005F02EF81249F1
:10C4A000087807F0AEF915490870002412E000255D
:10C4B0000CE004EB4400C01C28440B49085C04EB6E
:10C4C00044010F4A11444855681C85B2032DF0DB26
:10C4D000601C84B2032CEADB00200A4908600120BA
:10C4E0000949087070BD00008C2D0020B9020020A1
:10C4F000DE130020F2130020C6170020C90200201E
:10C50000CA02002008000020D302002078B50346AC
:10C51000002096E0524C245C524D2C5D8DF800407A
:10C520004F4C245C504D2C5D8DF801404C4C245CEC
:10C530004E4D2C5D8DF80240494C245C4C4D2C5DD9
:10C540008DF803404B4C2478012C1AD14A4C2478A6
:10C55000FE2C0CD1494C2478082C04D1464C24786C
:10C56000641E454D2C700024424D2C7023E0434C3A
:10C570002478082C1FD1404C2478641C3E4D2C702C
:10C5800019E03D4C2478012C0CD13C4C2478082C2B
:10C5900004D1394C2478641C374D2C700124354D5E
:10C5A0002C7008E0354C2478082C04D1324C2478C7
:10C5B000641E314D2C70304C2478314D2C709DF818
:10C5C0000040012C1BD12C4624785C43FF2594FBB2
:10C5D000F5F49DF801502B4E7455294C24784C43AA
:10C5E000FF2594FBF5F49DF802507455244C2478F3
:10C5F0005443FF2594FBF5F49DF8035074559DF8C2
:10C600000040022C1BD11E4C24785C43FF2594FB78
:10C61000F5F49DF801501C4E7455194C24784C4388
:10C62000FF2594FBF5F49DF802507455144C2478C2
:10C630005443FF2594FBF5F49DF803507455441CB6
:10C64000E0B20E28FFF466AF0C4C2478641C0B4D4E
:10C650002C702C462478082C01DD01242C7078BD28
:10C6600089620108405E01086A5E0108945E010863
:10C67000BE5E0108D80200205109002054090020A4
:10C68000DB020020661400203E15002010B50120BA
:10C6900004E000211D4A1154411CC8B21028F8DBE7
:10C6A0001B48007818B90A201849087002E00520D4
:10C6B0001649087005221521144808F0F9FA0120DE
:10C6C00004E00021134A1154411CC8B20828F8DBC9
:10C6D0000F48007818B901200E49087002E00320C5
:10C6E0000C490870132215210A4808F0E1FA08489D
:10C6F000007848B10A20084981F81102012081F828
:10C700001E0200200549088010BD0000A40F002073
:10C710001F00002004020020300A00206C020020CC
:10C7200070B50024002500269C48007800EB4000EE
:10C7300009309B49095C9948007800EB40000830BB
:10C74000974A105C00F07F0001EB002095490880BB
:10C7500008460088142801DA142008809248002135
:10C76000016041608D48007800EB400008308C4942
:10C77000085C00F08000802856D18848007800EBE3
:10C7800040000A30085C00F0E000E02811D10124EC
:10C790008248007800EB40000A30085C00F00F018E
:10C7A00001208840C5B28148005D28437F49085573
:10C7B00091E07A48007800EB40000A307849085C44
:10C7C00000F0B000B02811D177484078734909785B
:10C7D00001EB41010A31724A515C01F00F02012163
:10C7E0009140084370494870012674E06B48007816
:10C7F00000EB40000A306A49085C6D49085C040996
:10C800006648007800EB40000A306549085C6849DA
:10C81000085C00F00F0101208840C5B26348005D4C
:10C8200028436249085556E05C48007800EB400018
:10C830000A305B49085C00F0E000E02811D10124D7
:10C840005648007800EB40000A30085C00F00F0109
:10C8500001208840C5B25548005DA843534908559A
:10C8600039E04E48007800EB40000A304C49085C43
:10C8700000F0B000B02811D14B4840784749097802
:10C8800001EB41010A31464A515C01F00F020121DE
:10C89000914088434449487001261CE03F48007895
:10C8A00000EB40000A303E49085C4149085C04093D
:10C8B0003A48007800EB40000A303949085C3C49AE
:10C8C000085C00F00F0101208840C5B23748005DC8
:10C8D000A843364908553148007800EB40000D3038
:10C8E0002F49085CB8BB33480088012818DC32485F
:10C8F000007848B901202F49088000202F4908708E
:10C9000014202849088023E000202A4908800120BB
:10C910002B4908702949087014202249088017E023
:10C92000244800884FF6FF7188420BD021480088C8
:10C93000401E20490880012021490870142019490F
:10C94000088005E001201E49087014201549088060
:10C95000002012490870012E0FD11A48007818B92A
:10C9600001201149087002E003200F4908701322CA
:10C9700015210D4808F09CF90EE01248007818B90E
:10C980000A200A49087002E00520084908700522BB
:10C990001521064808F08CF970BD00009D090020A3
:10C9A0008C2E0020A409002004020020A40F0020E7
:10C9B000D0620108A00900209F0900209C090020E6
:10C9C0009E0900201F00002010B51C480078012897
:10C9D00016D100201949087001201949087000205B
:10C9E0001849087014201849088018480378184816
:10C9F00002781848017818480078FCF76FFC08E0C6
:10CA000016480078012804D1002014490870FFF767
:10CA10003DFE0B48007801280FD1FFF781FE094841
:10CA20000078401C074908700D480078012804D19F
:10CA300000200B4908700349087010BD9B090020B5
:10CA40009C0900209D090020A4090020A5020020C7
:10CA50009A0900201302002012020020A2090020DF
:10CA60009E09002070B504460E4615461F48002159
:10CA700001604160ADB9052C07DC4078611E0122E0
:10CA80008A401043194948701FE0062C03D1012049
:10CA90001649887119E0072C17D1FF2013498871B6
:10CAA00013E0012D11D1052C08DC10484078611EDF
:10CAB00001228A4090430D49487006E0062C01D0BF
:10CAC000072C02D10020094988710948007818B95B
:10CAD00001200649087002E003200449087003227F
:10CAE0001521024808F0E4F870BD0000FC010020A8
:10CAF0001F00002008B54FF4A06000F047F80D209B
:10CB00008DF8000000208DF801008DF80200012052
:10CB10008DF80300684600F001F808BD70B50021EB
:10CB200000230F22C47804B3154C246804F4E06495
:10CB3000C4F5E064210AC1F10403CA40447804FA50
:10CB400003F184781440214309010E4C0678A15565
:10CB5000047804F01F050124AC4005786D11AD0088
:10CB600005F1E025C5F8004109E0047804F01F054F
:10CB70000124AC40044D0678761145F8264070BD7E
:10CB80000CED00E000E400E080E100E00249014338
:10CB9000024A1160704700000000FA050CED00E049
:10CBA00010B500244FF400712E48FDF741FE2E49C8
:10CBB0000871FF2048710020087200BF09E00021C1
:10CBC0002948183001555030015550300155601C2E
:10CBD000C4B2502CF3DB002023494861FF2081F8C8
:10CBE0001D0181F81E01002081F8240181F88901CE
:10CBF000002404E000211D480155601CC4B2642CCF
:10CC0000F8DB0020184981F8F001012081F8F101DA
:10CC10000020C1F8F40181F8F80181F8F901FF2042
:10CC200081F8FA01002081F80002012081F8100249
:10CC3000002081F8110281F8130281F81C020C49CE
:10CC40008874094981F8140281F81D0281F81E02D6
:10CC500081F824025020A1F8260240F64260A1F893
:10CC6000280210BD00040040300A0020BA0B00204A
:10CC70008C300020002002498862C86270470000A2
:10CC8000000001400320024988620C20C8627047FE
:10CC90000000014078B50346002096E0524C245C29
:10CCA000524D2C5D8DF800404F4C245C504D2C5D56
:10CCB0008DF801404C4C245C4E4D2C5D8DF80240AB
:10CCC000494C245C4C4D2C5D8DF803404B4C247832
:10CCD000012C1AD14A4C2478FE2C0CD1494C2478D2
:10CCE000082C04D1464C2478641E454D2C70002439
:10CCF000424D2C7023E0434C2478082C1FD1404C2B
:10CD00002478641C3E4D2C7019E03D4C2478012C95
:10CD10000CD13C4C2478082C04D1394C2478641C68
:10CD2000374D2C700124354D2C7008E0354C24789B
:10CD3000082C04D1324C2478641E314D2C70304CB8
:10CD40002478314D2C709DF80040012C1BD12C46CD
:10CD500024785C43FF2594FBF5F49DF801502B4E9D
:10CD60007455294C24784C43FF2594FBF5F49DF829
:10CD700002507455244C24785443FF2594FBF5F459
:10CD80009DF8035074559DF80040022C1BD11E4C99
:10CD900024785C43FF2594FBF5F49DF801501C4E6C
:10CDA0007455194C24784C43FF2594FBF5F49DF8F9
:10CDB00002507455144C24785443FF2594FBF5F429
:10CDC0009DF803507455441CE0B20E28FFF466AF82
:10CDD0000C4C2478641C0B4D2C702C462478082CA9
:10CDE00001DD00242C7078BD89620108405E0108D5
:10CDF0006A5E0108945E0108BE5E0108D702002049
:10CE00005009002053090020DB0200206614002096
:10CE10003E15002008B50020DDE000EB8001704ADF
:10CE20001144497800297DD000EB8001515C6D4AA6
:10CE3000515C8DF8001000EB8001694A515C6A4A30
:10CE4000515C8DF8011000EB8001654A515C674A26
:10CE5000515C8DF8021000EB8001614A515C644A1C
:10CE6000515C8DF8031000EB80015D4A1144497854
:10CE7000FF2902D15F4A11704BE05F49097801290F
:10CE800020D100EB8001564A11444978FE290DD18A
:10CE900000EB800111444978491E00EB8002504BA1
:10CEA0001A4451700021544A11702BE000EB8001AC
:10CEB0004B4A11444978491C00EB8002484B1A4404
:10CEC00051701FE000EB8001454A11444978012967
:10CED0000DD100EB800111444978491C00EB800220
:10CEE0003F4B1A4451700121434A11700AE000EB94
:10CEF00080013B4A11444978491E00EB8002384BBF
:10CF00001A44517000EB8001354A11444978394A7E
:10CF100011709DF8001001292CD100EB8001304ADE
:10CF2000114400E055E08978324A12785143FF22DB
:10CF300091FBF2F19DF80120304B995400EB8001F8
:10CF4000274A1144C9782B4A12785143FF2291FB9A
:10CF5000F2F19DF80220995400EB8001204A11441F
:10CF60000979244A12785143FF2291FBF2F19DF88E
:10CF7000032099549DF8001002292AD100EB80016A
:10CF8000174A114489781B4A12785143FF2291FBBA
:10CF9000F2F19DF801201A4B995400EB8001104AE0
:10CFA0001144C978134A12785143FF2291FBF2F1E0
:10CFB0009DF80220995400EB8001094A1144097937
:10CFC0000C4A12785143FF2291FBF2F19DF80320A5
:10CFD0009954411CC8B22A28FFF61FAF08BD0000B3
:10CFE000741A0020405E01086A5E0108945E010820
:10CFF000BE5E0108DB020020D9020020661400207A
:10D000003E15002010B512BB012806D002280AD018
:10D0100003280ED0042818D111E001230D4C2370F1
:10D020000D4C237012E001230C4C23700A4C23702A
:10D030000CE001230A4C23700A4C237006E0012304
:10D04000094C2370074C237000E000BF00E000BFD4
:10D0500010BD0000940200209602002095020020DE
:10D0600097020020990200209802002070470000DB
:10D070000EB5012149F2E00000F08EF84FF0805229
:10D080005113C803FDF7B4FB00201F4908604FF09F
:10D09000805211141D48FDF7ABFB4FF480511B4823
:10D0A000FDF7D2FB4FF0805240211848FDF7A0FB5E
:10D0B00040211648FDF7C8FB154A38211348FDF7F3
:10D0C00097FB144802F06AFF0020ADF8000007202B
:10D0D000ADF802000020ADF80400ADF8060008200D
:10D0E000ADF808000020ADF80A006946094802F0D2
:10D0F00098FF01221146074802F0A0FF01210548D0
:10D1000002F044FF0EBD0000BC02004200040040DB
:10D110000500002000300040A1B1154A1268C3B2DA
:10D120001A43134B1A601A1D1268C0F30F231A43D7
:10D130000F4B1B1D1A601A1D126842EA10621B1D5C
:10D140001A6013E00A4A1268C3B29A43084B1A6085
:10D150001A1D1268C0F30F239A43054B1B1D1A605A
:10D160001A1D126822EA10621B1D1A607047000027
:10D170003C0C014010B5020A29B1064B1B68134351
:10D18000044C236004E0034B1B689343014C236071
:10D1900010BD0000880C014029B1064A1268024304
:10D1A000044B1A6004E0034A12688243014B1A6080
:10D1B00070470000480C014029B1064A126802433A
:10D1C000044B1A6004E0034A12688243014B1A6060
:10D1D00070470000900C014029B1064A12680243D2
:10D1E000044B1A6004E0034A12688243014B1A6040
:10D1F00070470000940C0140F0B501462D4F3F6888
:10D2000037B1012F06D0022F08D0032F29D103E018
:10D21000294828E0294826E0294824E0254F083FEE
:10D220003F6807F01F077F1C4FF0010C0CEB570203
:10D23000244F3F68C7F38117C7F103074FF00C0C69
:10D240000CEB87031B4F3F1F3F68012F04D11C4F7E
:10D250005F43B7FBF2F003E0174F5F43B7FBF2F019
:10D2600001E0154800BF00BF124F10373F6807F0BC
:10D270007F077F1C4FF0010C0CEB57040D4F143748
:10D280003F6807F07F077F1C0CEB5705094F1837E5
:10D290003F6807F07F077F1C0CEB57060860B0FB68
:10D2A000F4F74F60B0FBF5F78F60B0FBF6F7CF6097
:10D2B000F0BD0000080C014000127A00006CDC0296
:10D2C000001BB70074040140034908600121024AB1
:10D2D000121D116070470000080C0140B9B1012215
:10D2E000114B1A600822104B583B1A601A461268FC
:10D2F00000F006031A430C4B583B1A601A4612689A
:10D3000000F001031A43084B583B1A600BE0064A31
:10D31000583A126802F00802034B583B1A60002288
:10D320001A60014B1A6070476C0C014018B1012162
:10D33000034A116002E00021014A116070470000B9
:10D340007C0C01400149086070470000340C01402A
:10D3500038B50146002301293CD1002037E03F4A7F
:10D36000125C3F4CA25C8DF800203C4A125C3D4CA4
:10D37000A25C8DF80120394A125C3B4CA25C8DF80E
:10D380000220364A125C394CA25C8DF803209DF8CD
:10D390000020012A0AD100229DF80140344D2A556F
:10D3A0009DF802402A559DF803402A559DF800201B
:10D3B000022A0AD100229DF801402E4D2A559DF8DF
:10D3C00002402A559DF803402A55421CD0B20E282F
:10D3D000C5D342E0022940D100203CE0204A125C43
:10D3E0008DF800201F4A125C8DF801201E4A125C45
:10D3F0008DF802201D4A125C8DF8032000230022C4
:10D4000006E0164CA45C844200D10123541CE2B215
:10D410000E2AF6D3EBB99DF80020012A0AD100228A
:10D420009DF80140124D2A559DF802402A559DF85D
:10D4300003402A559DF80020022A0AD100229DF8B7
:10D4400001400C4D2A559DF802402A559DF8034095
:10D450002A55421CD0B22A28C0DB38BD8962010897
:10D46000405E01086A5E0108945E0108BE5E010824
:10D47000661400203E1500202DE9F84340BBDFF87C
:10D48000BCC19CF800C0BCF1000F06D14FF0010CEC
:10D49000DFF8A88188F800C01AE0DFF8A0C19CF886
:10D4A00000C0BCF1010F06D14FF0020CDFF88C81F7
:10D4B00088F800C00CE0DFF884C19CF800C0BCF123
:10D4C000020F05D14FF0000CDFF8708188F800C022
:10D4D000DFF868C19CF800C0BCF1000F06D1FF2244
:10D4E000002300240025FF2600271AE0DFF84CC1A6
:10D4F0009CF800C0BCF1010F06D10022FF230024DC
:10D5000000250026FF270CE0DFF830C19CF800C0A2
:10D51000BCF1020F05D100220023FF24FF250026C5
:10D520000027002185E0DFF818C11CF801C0BCF11C
:10D53000FF0F7AD0DFF80CC11CF801C08DF800C0D5
:10D54000DFF804C11CF801C08DF801C0DFF8FCC091
:10D550001CF801C08DF802C0DFF8F4C01CF801C04F
:10D560008DF803C09DF800C0BCF1010F2CD1C0F1B3
:10D57000FF0C0CFB02FC05FB00CC4FF0FF089CFBF2
:10D58000F8FC9DF80180DFF8CC9009F808C0C0F1E4
:10D59000FF0C0CFB03FC06FB00CC4FF0FF089CFBD0
:10D5A000F8FC9DF8028009F808C0C0F1FF0C0CFBE4
:10D5B00004FC07FB00CC4FF0FF089CFBF8FC9DF837
:10D5C000038009F808C030E09DF800C0BCF1020FEC
:10D5D0002BD1C0F1FF0C0CFB02FC05FB00CC4FF083
:10D5E000FF089CFBF8FC9DF80180DFF86C9009F8BF
:10D5F00008C0C0F1FF0C0CFB03FC06FB00CC4FF095
:10D60000FF089CFBF8FC9DF8028009F808C0C0F1F7
:10D61000FF0C0CFB04FC07FB00CC4FF0FF089CFB4D
:10D62000F8FC9DF8038009F808C001F1010C0CF02A
:10D63000FF012A29FFF677AFBDE8F883DC0200205E
:10D64000E85E0108405E01086A5E0108945E010818
:10D65000BE5E0108661400203E1500207FB504461A
:10D660000E4600256AE03748405D8DF80C003648CC
:10D67000405D8DF80D003548405D8DF80E00344852
:10D68000405D8DF80F003348007810B1012811D1AA
:10D6900009E0314800780290304800780190304825
:10D6A0000078009007E06B4601AA02A9284607F01F
:10D6B00095FC00E000BF00BF9DF80C0001281BD1C5
:10D6C0009DF808006043FF2190FBF1F09DF80D10DC
:10D6D000244A50549DF804006043FF2190FBF1F070
:10D6E0009DF80E1050549DF800006043FF2190FB00
:10D6F000F1F09DF80F1050549DF80C0002281BD13A
:10D700009DF808006043FF2190FBF1F09DF80D109B
:10D71000154A50549DF804006043FF2190FBF1F03E
:10D720009DF80E1050549DF800006043FF2190FBBF
:10D73000F1F09DF80F105054681CC5B22A2D92DBF1
:10D740007FBD0000405E01086A5E0108945E01082A
:10D75000BE5E0108BD020020B6020020B702002014
:10D76000B8020020661400203E1500202DE9F14F7C
:10D7700082B0029F00247AE03F48005DFF2874D009
:10D780003E48005D8DF804003D48005D8DF80500C1
:10D790003C48005D8DF806003B48005D8DF80700B1
:10D7A0003548055D394810F80480BD4203DAE81DAC
:10D7B000C01BC5B201E0E81BC5B205EB450034490A
:10D7C00001EB400010F80800012828D1314800780A
:10D7D00048B9314890F80090304890F800A030489F
:10D7E00090F800B01FE04FF00009CA46CB46F9F7A9
:10D7F000E3FC072190FBF1F201FB1200C6B206EB3D
:10D800004600284911F8009006EB4600084490F8BD
:10D8100001A006EB4600084490F802B003E04FF088
:10D820000009CA46CB469DF8040001280CD19DF89A
:10D8300005101D4A02F801909DF8061002F801A09B
:10D840009DF8071002F801B09DF8040002280CD1E1
:10D850009DF80510154A02F801909DF8061002F88F
:10D8600001A09DF8071002F801B0601CC4B22A2C78
:10D8700082DBBDE8FE8F0000E85E0108405E010823
:10D880006A5E0108945E0108BE5E01083860010806
:10D8900062600108BD020020B6020020B70200202D
:10D8A000B80200208C600108661400203E1500209C
:10D8B0002DE9F04F89B0064600240020069006208E
:10D8C000059000200490002500BFA5E05548005DAC
:10D8D000FF287CD05448005D06905248005D0490BB
:10D8E000DDE90512881A07F0F2FC00221346CDE9A3
:10D8F000000106F04DF8CDE9020107F0BBFCC5B20E
:10D90000284607F0FBFCCDE9000105F07FFBCDE9DF
:10D91000020107F0AFFCC5B20F2D02DBA5F10F002D
:10D92000C5B2AE4205DA06F10F00401B00F0FF0859
:10D9300002E0701B00F0FF08B8F1100F03DBA8F144
:10D94000100000F0FF08394810F8081004988142D0
:10D9500028D13748007848B9364890F800903648C2
:10D9600090F800A0354890F800B01FE04FF0000993
:10D97000CA46CB46F9F720FC072190FBF1F201FBE8
:10D980001200C7B207EB47002D4911F8009007EBD2
:10D990004700084490F801A007EB4700084490F8BE
:10D9A00002B003E04FF00009CA46CB462548005DAF
:10D9B0008DF81C002448005D8DF81D002348005D93
:10D9C0008DF81E002248005D8DF81F0000E021E068
:10D9D0009DF81C0001280CD19DF81D001D4901F87F
:10D9E00000909DF81E0001F800A09DF81F0001F8AE
:10D9F00000B09DF81C0002280CD19DF81D001649AE
:10DA000001F800909DF81E0001F800A09DF81F008D
:10DA100001F800B0601CC4B22A2CFFF657AF09B061
:10DA2000BDE8F08FE85E01083C5F0108186201085C
:10DA3000BD020020B6020020B7020020B80200207C
:10DA40008C600108405E01086A5E0108945E01086E
:10DA5000BE5E0108661400203E1500202DE9F84F37
:10DA600004460025C9E06748405DFF287ED0042CAD
:10DA700006DC22463146284603F05EF9064640E0C1
:10DA8000122C06DC22463146284603F0D1F9064620
:10DA900037E01C2C1ADC142D16D1A4F1130000EB76
:10DAA000C00101EB0010FF21B1EB400F01DC0026AB
:10DAB00027E0A4F1130000EBC00101EB0010FF21EF
:10DAC000A1EB4000C6B21CE000261AE0322C06DCB6
:10DAD00022463146284603F0B9F9064611E0A4F182
:10DAE0003300C0EB0010FF21B1EB400F01DC00263A
:10DAF00007E0A4F13300C0EB0010FF21A1EB4000D0
:10DB0000C6B24148405D8DF800004048405D8DF848
:10DB100001003F48405D8DF802003E48405D8DF8B1
:10DB2000030056B33C48007848B93C4890F8008060
:10DB30003B4890F800903B4890F800A021E04FF05F
:10DB40000008C146C246F9F737FB072190FBF1F206
:10DB500001FB1200C7B207EB4700334911F8008000
:10DB600007EB4700084490F8019000E043E007EB22
:10DB70004700084490F802A003E04FF00008C146B7
:10DB8000C2469DF80000012818D108FB06F0FF21CD
:10DB900090FBF1F09DF80110244A505409FB06F067
:10DBA000FF2190FBF1F09DF8021050540AFB06F0A3
:10DBB000FF2190FBF1F09DF8031050549DF80000F8
:10DBC000022818D108FB06F0FF2190FBF1F09DF828
:10DBD0000110174A505409FB06F0FF2190FBF1F0A9
:10DBE0009DF8021050540AFB06F0FF2190FBF1F063
:10DBF0009DF803105054681CC5B22A2DFFF633AFB0
:10DC0000BDE8F88FE85E0108405E01086A5E010821
:10DC1000945E0108BE5E0108BD020020B60200202D
:10DC2000B7020020B80200208C60010866140020B2
:10DC30003E1500202DE9F04387B006460024A0E001
:10DC40005348005DFF287DD05248005D8DF81800D4
:10DC50005148005D8DF819005048005D8DF81A009C
:10DC60004F48005D8DF81B00002E72D14D480078A2
:10DC70000C2817D1F9F7A0FA1E2190FBF1F201FB55
:10DC80001200401C48490855012048490855F9F739
:10DC900093FA072190FBF1F201FB1200401C44496A
:10DCA000085517E0F9F788FA1E2190FBF1F201FB05
:10DCB0001200401C3C49085501203C490855F9F721
:10DCC0007BFA0546C01705EB5070C010A5EBC000ED
:10DCD000374908550027B846B9463548005DB0B108
:10DCE0003348005D401E00EB400032490F5C304875
:10DCF000005D401E00EB4000084490F801802C4875
:10DD0000005D401E00EB4000084490F802909DF832
:10DD1000180001280AD100209DF81910264A5054F5
:10DD20009DF81A1050549DF81B1050549DF818007F
:10DD3000022824D100209DF81910204A50549DF843
:10DD40001A1001E01BE004E050549DF81B105054E1
:10DD500015E01648005D30B904AB05AA06A92046B7
:10DD600000F0E6F90BE004A805A906AA4B46CDE9A8
:10DD70000021029042463946204600F0EDFA601C30
:10DD8000C4B22A2CFFF65CAF07B0BDE8F0830000F8
:10DD9000E85E0108405E01086A5E0108945E0108C1
:10DDA000BE5E0108B902002046190020701900204B
:10DDB0009A1900208C600108661400203E1500208E
:10DDC0002DE9F14F86B0002495E1CE48005DFF2893
:10DDD0007DD0CD48005D8DF81400CC48005D8DF8F5
:10DDE0001500CB48005D8DF81600CA48005D8DF81F
:10DDF00017000698002833D10220C7490855C749A3
:10DE00000855F9F7D9F9072190FBF1F201FB12004F
:10DE1000401CC34908550025002600270846005D20
:10DE200088B10846005D00EB4000BE490D5CBC486F
:10DE3000005D00EB400008444678B948005D00EB07
:10DE40004000084487788DF810508DF811608DF8E7
:10DE500012708DF80C508DF80D608DF80E7020E169
:10DE6000AE48005D00283ED1F9F7A6F9C82190FB25
:10DE7000F1F201FB12003230A74908550846005D57
:10DE8000A6490855A648005D072803D10120A449EA
:10DE9000085504E0A248005D401CA1490855A0486F
:10DEA000005D88B19E48005D00EB40009D490D5C1F
:10DEB0009B48005D00EB4000084446789848005DB0
:10DEC00000EB4000084487788DF8105000E010E126
:10DED0008DF811608DF812708DF80C508DF80D6072
:10DEE0008DF80E70DDE08D48005D401E8B490855B1
:10DEF0008B48005D00EB40008A4911F8008088489B
:10DF0000005D072803D1084690F800B007E0844878
:10DF1000005D401C00EB4000824911F800B08048D1
:10DF2000005D00EB40007F49084490F801907C4878
:10DF3000005D072803D108464078029008E0784841
:10DF4000005D401C00EB4000764908444078029098
:10DF50007348005D00EB40007249084490F802A04D
:10DF60006F48005D072803D108468078019008E0DB
:10DF70006B48005D401C00EB40006A490844807813
:10DF800001906748005D00287ED06448005D00FB7A
:10DF900008F06149095D90FBF1F15F48005D5F4A5F
:10DFA000125D801A00FB0BF05B4A125D90FBF2F0F1
:10DFB0000844C0B28DF810005848005D00FB09F01D
:10DFC0005549095D90FBF1F25348005D5349095DE5
:10DFD000401A029948435049095D90FBF1F0104402
:10DFE000C0B28DF811004D48005D00FB0AF04A49AF
:10DFF000095D90FBF1F24848005D4849095D401A0F
:10E00000019948434449095D90FBF1F01044C0B2C6
:10E010008DF812004148005D00FB08F03E49095DA3
:10E0200090FBF1F13C48005D3C4A125D801A00FB18
:10E030000BF0394A125D90FBF2F00844C0B28DF843
:10E040000C003648005D00FB09F03349095D90FB88
:10E05000F1F23148005D3149095D401A02994843A7
:10E060002D49095D90FBF1F01044C0B28DF80D0010
:10E070002A48005D00FB0AF02749095D90FBF1F298
:10E080002548005D254900E00BE0095D401A019933
:10E0900048432149095D90FBF1F01044C0B28DF86E
:10E0A0000E009DF8140001280FD19DF810009DF876
:10E0B00015101D4A50549DF811009DF8161050542B
:10E0C0009DF812009DF8171050549DF81400022876
:10E0D0000FD19DF80C009DF81510144A50549DF86E
:10E0E0000D009DF8161050549DF80E009DF8171065
:10E0F0005054601CC4B22A2CFFF667AE07B0BDE8CE
:10E10000F08F0000E85E0108405E01086A5E0108C9
:10E11000945E0108BE5E01081C190020461900200B
:10E120009A1900208C600108661400203E1500201A
:10E130002DE9F04104460D4616461F467B48005D1A
:10E14000002831D179490855012079490855794885
:10E1500000780C2811D07848005D18B1002076496D
:10E1600008550AE0F9F728F88046C01708EB507008
:10E17000C010A8EBC000704908552878012807D1C5
:10E18000002069786D4A5054A9785054E978505469
:10E19000287802280DD100206978694A5054A9785E
:10E1A0005054E978505404E06048005D401E5F49D7
:10E1B00008555F48005D00287ED15F48005D00285B
:10E1C0007BD060480078B0BB5848005D5E49097854
:10E1D00048431E2190FBF1F030705448005D5B49CC
:10E1E000097848431E2190FBF1F070704F48005DA4
:10E1F0005749097848431E2190FBF1F0B0704B4815
:10E20000005D5149097848431E2190FBF1F03870B8
:10E210004648005D4D49097848431E2190FBF1F0C6
:10E2200078704248005D4A49097848431E2190FBB6
:10E23000F1F0B8705DE0FFE73F48005D00EB4000A3
:10E240004449085C3949095D48431E2190FBF1F0BF
:10E2500030703948005D00EB40003E49084440788A
:10E260003249095D48431E2190FBF1F0707032483D
:10E27000005D00EB40003749084480782B49095D78
:10E2800048431E2190FBF1F0B0702B48005D00EB7D
:10E2900040003049085C2549095D48431E2190FB38
:10E2A000F1F038702448005D00EB40002949084433
:10E2B00040781E49095D01E035E013E048431E2126
:10E2C00090FBF1F078701C48005D00EB40002149A4
:10E2D000084480781549095D48431E2190FBF1F000
:10E2E000B87006E0002030707070B07038707870D0
:10E2F000B8702878012809D1307869780F4A5054CD
:10E300007078A9785054B078E97850542878022869
:10E3100009D1387869780A4A50547878A9785054E5
:10E32000B878E9785054BDE8F08100004619002023
:10E3300070190020B90200209A19002066140020EC
:10E340003E150020BD020020B6020020B7020020CA
:10E35000B80200208C6001082DE9F04106AC70CCB9
:10E36000AB4F3F5C1E2F49D1DFF8A4C20CF8007000
:10E370000027DFF8A0C20CF8007000210022002363
:10E38000A54F3F5CEFB1A54F3F7837B9A44F39781F
:10E39000A44F3A78A44F3B7813E09F4F3F5C07EBC4
:10E3A0004707DFF888C21CF807109B4F3F5C07EB5C
:10E3B000470767447A78984F3F5C07EB4707674405
:10E3C000BB782778012F0AD16778DFF864C20CF890
:10E3D0000710A7780CF80720E7780CF807302778A3
:10E3E000022F12D16778DFF84CC20CF80710A7781B
:10E3F0000CF80720E7780CF8073006E0844F3F5C04
:10E400007F1CDFF80CC20CF80070824F3F5C012FBC
:10E410007ED1814F3F5C002F7BD0804F3F78E7BBA0
:10E420007B4F3F5CDFF8F8C19CF800C007FB0CF79E
:10E430004FF01E0C97FBFCF72F70754F3F5CDFF819
:10E44000E4C19CF800C007FB0CF74FF01E0C97FBD3
:10E45000FCF76F706E4F3F5CDFF8CCC19CF800C0DA
:10E4600007FB0CF74FF01E0C97FBFCF7AF70684FE3
:10E470003F5CDFF8ACC19CF800C007FB0CF74FF025
:10E480001E0C97FBFCF73770614F3F5CDFF894C1BF
:10E490009CF800C007FB0CF700E012E04FF01E0CE8
:10E4A00097FBFCF777705A4F3F5CDFF87CC19CF814
:10E4B00000C007FB0CF74FF01E0C97FBFCF7B77082
:10E4C0007CE0554F3F5C07EB4707DFF860C11CF865
:10E4D0000770DFF83CC11CF800C007FB0CF74FF0D9
:10E4E0001E0C97FBFCF72F704B4F3F5C07EB470769
:10E4F000DFF838C167447F78DFF814C11CF800C02A
:10E5000007FB0CF74FF01E0C97FBFCF76F7001E058
:10E510007CE04CE0404F3F5C07EB4707DFF80CC165
:10E520006744BF78DFF8E8C01CF800C007FB0CF7B1
:10E530004FF01E0C97FBFCF7AF70374F3F5C07EBBB
:10E540004707DFF8E8C01CF80770DFF8C4C01CF804
:10E5500000C007FB0CF74FF01E0C97FBFCF7377061
:10E560002D4F3F5C07EB4707DFF8C0C067447F785B
:10E57000DFF89CC01CF800C007FB0CF74FF01E0C26
:10E5800097FBFCF77770244F3F5C07EB4707DFF8FA
:10E590009CC06744BF78DFF878C01CF800C007FB58
:10E5A0000CF74FF01E0C97FBFCF7B77006E0002746
:10E5B0002F706F70AF7037707770B7702778012F3A
:10E5C00010D12F7894F801C0DFF8648008F80C703F
:10E5D0006F7894F802C008F80C70AF7894F803C014
:10E5E00008F80C702778022F10D1377894F801C002
:10E5F000DFF8408008F80C70777894F802C008F8CB
:10E600000C70B77894F803C008F80C70BDE8F0817E
:10E6100046190020701900209A190020BD02002020
:10E62000B6020020B7020020B80200208C6001086A
:10E63000661400203E15002008B5002135E01C4A74
:10E64000525C1C4B9A5C8DF80020194A525C1A4BA4
:10E650009A5C8DF80120164A525C184B9A5C8DF832
:10E660000220134A525C164B9A5C8DF803209DF8E9
:10E670000020012A09D19DF80120124B98549DF8E1
:10E68000022098549DF8032098549DF80020022AF7
:10E6900009D19DF801200C4B98549DF80220985404
:10E6A0009DF8032098544A1CD1B20E29C7D308BD47
:10E6B00089620108405E01086A5E0108945E0108F3
:10E6C000BE5E0108661400203E150020002006E012
:10E6D0000021044A1154044A1154411CC8B2D828DC
:10E6E000F6DB7047661400203E1500202DE9F34F3D
:10E6F00085B0644903C9CDE90301069D0024BBE050
:10E700006148005DFF287DD06048007858B96048B6
:10E71000075DAF4204DA07F10800401BC6B20DE006
:10E72000781BC6B20AE05B48075DAF4204DA07F126
:10E730000800401BC6B201E0781BC6B25648005D17
:10E740008DF808005548005D8DF809005448005DBB
:10E750008DF80A005348005D8DF80B005248007890
:10E7600010B101283CD109E0504890F80090504881
:10E7700090F800A04F480078019032E04FF0000977
:10E78000CA4600200190F8F717FD072190FBF1F22F
:10E7900001FB120B4848005D0BFB00FBF8F70CFD7A
:10E7A000072190FBF1F201FB12003749095D01FBE3
:10E7B00000B0072190FBF1F201FB120000F0FF080E
:10E7C00008EB48003D4911F8009008EB4800084468
:10E7D00090F801A008EB480008448078019000E020
:10E7E00000BF00BF9DF80800012820D103A8805D6C
:10E7F00000FB09F0FF2190FBF1F09DF80910304A71
:10E80000505400E036E003A8805D00FB0AF0FF21D1
:10E8100090FBF1F09DF80A10505403A8805D019917
:10E820004843FF2190FBF1F09DF80B1050549DF8E8
:10E83000080002281ED103A8805D00FB09F0FF211B
:10E8400090FBF1F09DF809101E4A505403A8805D1A
:10E8500000FB0AF0FF2190FBF1F09DF80A105054E4
:10E8600003A8805D01994843FF2190FBF1F09DF8DA
:10E870000B105054601CC4B22A2CFFF641AF07B0F5
:10E88000BDE8F08FC86201083C5F0108DF0200208C
:10E89000125F0108665F0108405E01086A5E0108B8
:10E8A000945E0108BE5E0108BD020020B602002091
:10E8B000B7020020B8020020E85E01088C60010861
:10E8C000661400203E1500202DE9F04F89B0044663
:10E8D0000F4600260020079008908046069005907D
:10E8E000814682464FF0FF0B0025049000BFD9E01F
:10E8F0006F48805D8DF81C006E48805D8DF81D00AE
:10E900006D48805D8DF81E006C48805D8DF81F009D
:10E910008DF820606A48805D0690DDE90521881A3F
:10E9200006F0D5FC02460B46CDE900010020014669
:10E9300005F02EF8CDE9020106F09CFC00F0FF087E
:10E94000404606F0DBFCCDE9000104F05FFBCDE9B9
:10E95000020106F08FFC00F0FF0808EB0700C5B2CB
:10E96000072D01DBE81FC5B2062D32D105EB4500AE
:10E970005449085CC4F1120148435249097801FB2B
:10E980000400122190FBF1F000F0FF0905EB4500B7
:10E990004C4908444078C4F1120148434949497838
:10E9A00001FB0400122190FBF1F000F0FF0A05EBDF
:10E9B0004500444908448078C4F112014843414964
:10E9C000897801FB0400122190FBF1F000F0FF0BAD
:10E9D0003AE005EB45003B49085CC4F112014843AD
:10E9E000691C01EB4101374A515C01FB0400122113
:10E9F00090FBF1F000F0FF0905EB450011460844DB
:10EA00004078C4F112014843691C01EB41011144F3
:10EA1000497801FB0400122190FBF1F000F0FF0A9D
:10EA200005EB4500114608448078C4F112014843C3
:10EA3000691C01EB41011144897801FB040012219A
:10EA400090FBF1F000F0FF0B9DF81C00012811D1A4
:10EA50009DF820101C4A049850549DF81D001B4935
:10EA600001F800909DF81E0001F800A09DF81F001D
:10EA700001F800B09DF81C00022811D19DF820106B
:10EA8000134A049850549DF81D00124901F8009053
:10EA90009DF81E0001F800A09DF81F0001F800B0CD
:10EAA000701CC6B22A2EFFF623AF09B0BDE8F08F66
:10EAB000405E01086A5E0108945E0108BE5E0108BE
:10EAC000E85E01088C60010816160020661400201C
:10EAD000EE1600203E1500202DE9F04FA9B00646A5
:10EAE0000F46914600202690259024902390804642
:10EAF00019F80600C0F1140000F0FF0A0025B6E086
:10EB00005E48405DFF287DD05D48405D26905B48B3
:10EB1000405D2490B85D5A49085C2590B85D57491E
:10EB2000085C2390DDE92312881A06F0D0FBCDE9BA
:10EB30000201DDE92512881A06F0C9FBCDE90001C2
:10EB4000DDE9022304F024FFCDE9040106F092FB85
:10EB500000F0FF08404606F0D1FBCDE9020104F0C9
:10EB600055FACDE9040106F085FB00F0FF08C24527
:10EB70007BD10AEB0800C4B2242C02DBA4F12400F0
:10EB8000C4B24048405D8DF89C003F48405D8DF820
:10EB90009D003E48405D8DF89E003D48405D8DF8EB
:10EBA0009F003C48007810B1012838D109E03A486C
:10EBB00090F800B0394800780790394800780690FE
:10EBC0002EE004EB44003749085C04EB440108AA3A
:10EBD000505404EB440008A911F800B004EB4400C1
:10EBE00030490844407804EB44011144487004EB78
:10EBF000440008A908444078079004EB44002949E0
:10EC0000084400E031E0807804EB4401114488704E
:10EC100004EB440008A908448078069000E000BF97
:10EC200000BF9DF89C0001280DD19DF89D001E4954
:10EC300001F800B09DF89E101B4A079850549DF8AB
:10EC40009F10069850549DF89C0002280DD19DF805
:10EC50009D00164901F800B09DF89E10134A0798D0
:10EC600050549DF89F1006985054681CC5B22A2D28
:10EC7000FFF646AF29B0BDE8F08F0000E85E01085E
:10EC80003C5F0108405E01086A5E0108945E01086D
:10EC9000BE5E0108BD020020B6020020B7020020BF
:10ECA000B80200208C600108661400203E15002088
:10ECB0002DE9F74F8BB00B46164600255AE2002788
:10ECC00051E2DFF8BC9409EB850919F80740FF2CE5
:10ECD0007ED0B54206DA05F10C09A9EB060909F068
:10ECE000FF0203E0A5EB060909F0FF02114622B17D
:10ECF000A2F1010909F0FF0000E00B20DFF8849485
:10ED000019F804908DF80490DFF87C9419F80490B9
:10ED10008DF80590DFF8749419F804908DF806903A
:10ED2000DFF86C9419F804908DF80790DDF82C90BA
:10ED3000B9F1000F75D1DFF85C9419F80290DFF893
:10ED400058A49AF800A009FB0AF94FF0FF0A99FBB2
:10ED5000FAF902EB420A0DF1080B0BF80A90DFF802
:10ED6000349419F80290DFF834A49AF800A009FB53
:10ED70000AF94FF0FF0A99FBFAF902EB420ADA446A
:10ED80008AF80190DFF80C9419F80290DFF810A4CB
:10ED90009AF800A009FB0AF94FF0FF0A99FBFAF96B
:10EDA00002EB420ADA448AF80290DFF8E89319F895
:10EDB0000090DFF8E4A39AF800A009FB0AF94FF0ED
:10EDC000FF0A99FBFAF900EB400A0BF80A9000E001
:10EDD000C5E1DFF8C09319F80090DFF8C0A39AF8F6
:10EDE00000A009FB0AF94FF0FF0A99FBFAF900EBC2
:10EDF000400ADA448AF80190DFF8989319F80090F5
:10EE0000DFF89CA39AF800A009FB0AF94FF0FF0A6B
:10EE100099FBFAF900EB400ADA448AF8029046E0DE
:10EE2000FFE702EB4209DFF87CA31AF8099002EB36
:10EE3000420A0DF1080B0BF80A9002EB4209DFF8C9
:10EE400064A3D14499F8019002EB420ADA448AF8AB
:10EE5000019002EB4209DFF84CA3D14499F80290EB
:10EE600002EB420ADA448AF8029000EB4009DFF82C
:10EE700034A31AF8099000EB400A0BF80A9000EB53
:10EE80004009DFF820A3D14499F8019000EB400A33
:10EE9000DA448AF8019000EB4009DFF808A3D14476
:10EEA00099F8029000EB400ADA448AF8029001EBEC
:10EEB00041090DF1080A1AF8099000EB400A0DF11A
:10EEC000080B1BF80AA0D1451BDD01EB4109DA460E
:10EED0001AF8099000EB400A1BF80AA0A9EB0A09EE
:10EEE00003F1010A09FB0AF94FF0090A99FBFAF943
:10EEF00001EB410A1BF80AA0AAEB090909F0FF0C73
:10EF00002EE001EB41090DF1080A1AF8099000EB17
:10EF1000400A0DF1080B1BF80AA0D1451ADA00EBE4
:10EF20004009DA461AF8099001EB410A1BF80AA0D9
:10EF3000A9EB0A0903F1010A09FB0AF94FF0090AD2
:10EF400099FBFAF901EB410A1BF80AA0D14409F038
:10EF5000FF0C05E001EB41090DF1080A1AF809C0A0
:10EF600001EB41090DF1080AD14499F8019000EB39
:10EF7000400A0DF1080BDA449AF801A0D1451EDDD4
:10EF800001EB4109DA46D14499F8019000EB400ABF
:10EF9000DA449AF801A0A9EB0A0903F1010A09FB76
:10EFA0000AF94FF0090A99FBFAF901EB410ADA4430
:10EFB0009AF801A0AAEB090909F0FF0834E001EB77
:10EFC00041090DF1080AD14499F8019000EB400A7B
:10EFD0000DF1080BDA449AF801A0D1451DDA00EBD7
:10EFE0004009DA46D14499F8019001EB410ADA442C
:10EFF0009AF801A0A9EB0A0903F1010A09FB0AF931
:10F000004FF0090A99FBFAF901EB410ADA449AF840
:10F0100001A0D14409F0FF0806E001EB41090DF120
:10F02000080AD14499F8018001EB41090DF1080A61
:10F03000D14499F8029000EB400A0DF1080BDA4434
:10F040009AF802A0D14521DD01EB410ADA449AF891
:10F0500002A000EB400B0DF1080EF3449BF802B048
:10F06000AAEB0B0A03F1010B0AFB0BF94FEAE97A51
:10F0700009EBDA6A01EB410BF3449BF802B0ABEB0E
:10F080006A1A0AF0FF0ACDF800A03AE001EB410944
:10F090000DF1080AD14499F8029000EB400A0DF1F5
:10F0A000080BDA449AF802A0D14521DA00EB400AB5
:10F0B000DA449AF802A001EB410B0DF1080EF3447B
:10F0C0009BF802B0AAEB0B0A03F1010B0AFB0BF948
:10F0D0004FEAE97A09EBDA6A01EB410BF3449BF85A
:10F0E00002B00BEB6A1A0AF0FF0ACDF800A008E0A4
:10F0F00001EB41090DF1080AD14499F80290CDF8CD
:10F1000000909DF80490B9F1010F11D19DF8059080
:10F11000DFF894A00AF809C09DF806900AF8098063
:10F120009DF807A0DFF880B0DDF800900BF80A909A
:10F130009DF80490B9F1020F11D19DF80590DFF808
:10F140006CA00AF809C09DF806900AF809809DF89D
:10F1500007A0DFF858B0DDF800900BF80A9007F12F
:10F16000010909F0FF07042FFFF6ABAD05F1010916
:10F1700009F0FF050C2DFFF6A2AD0EB0BDE8F08F33
:10F1800097620108405E01086A5E0108945E01080A
:10F19000BE5E010841620108B6020020B7020020ED
:10F1A000B80200208C600108661400203E15002083
:10F1B0002DE9F04F89B006460F46904699464FF02C
:10F1C000000AD34600200790069005900490002482
:10F1D0008CE04948005D8DF820004848005D8DF8BE
:10F1E00021004748005D8DF822004648005D8DF8FB
:10F1F00023004548005D0690DDE90521881A06F0E8
:10F2000066F800221346CDE9000104F0C1FBCDE908
:10F21000020106F02FF8C0B20490049806F06EF8D0
:10F22000CDE9000103F0F2FECDE9020106F022F87B
:10F23000C0B204900498864201DBFF2500E000255F
:10F240003248007830B1012809D002280AD00328BA
:10F250000ED10AE0BA46C346CDF81C9009E04FF043
:10F26000FF0A06E04FF0FF0B03E0FF20079000E0ED
:10F2700000BF00BF9DF82000012818D10AFB05F04F
:10F28000FF2190FBF1F09DF82110214A50540BFB17
:10F2900005F0FF2190FBF1F09DF8221050540798E3
:10F2A0006843FF2190FBF1F09DF8231050549DF826
:10F2B0002000022818D10AFB05F0FF2190FBF1F095
:10F2C0009DF82110134A50540BFB05F0FF2190FBD1
:10F2D000F1F09DF82210505407986843FF2190FBED
:10F2E000F1F09DF823105054601CC4B22A2CFFF694
:10F2F00070AF09B0BDE8F08F405E01086A5E01089A
:10F30000945E0108BE5E0108E45F0108BD020020B2
:10F31000661400203E1500202DE9F04F8BB0054605
:10F320000E464FF0000B0020089007900690824692
:10F33000002473E03C48005DFF286DD03B4810F886
:10F3400004B03948005D0790705D3849085C08904A
:10F35000705D3549085C0690DDE90612881A05F0F3
:10F36000B6FFCDE902010899A1EB0B0005F0AFFF54
:10F37000CDE90001DDE9022304F00AFBCDE9040137
:10F3800005F078FF00F0FF0A504605F0B7FFCDE921
:10F39000020103F03BFECDE9040105F06BFF00F034
:10F3A000FF0ABAF1000F37D12148005D8DF8240023
:10F3B0002048005D8DF825001F48005D8DF826006F
:10F3C0001E48005D8DF827001D4807781D4890F8FD
:10F3D00000801D4890F800909DF8240001280BD172
:10F3E0009DF8250019490F549DF8260001F800806A
:10F3F0009DF8270001F800909DF8240002280BD109
:10F400009DF8250012490F549DF8260001F8008050
:10F410009DF8270001F80090601CC4B22A2C89DBFB
:10F420000BB0BDE8F08F0000E85E01080E60010837
:10F43000405E01086A5E0108945E0108BE5E010834
:10F44000B6020020B7020020B80200206614002097
:10F450003E1500200A2100201BE00F4A125C142AEE
:10F4600003DC00220C4B1A5404E00B4A125C521AC3
:10F47000094B1A54094A125C142A03DC0022074B78
:10F480001A5404E0054A125C521A044B1A54421CE6
:10F49000D0B2D828E1DB7047661400203E1500206A
:10F4A0002DE9F04F89B005460E461746002006901C
:10F4B00005908046785DC0F11400C0B2049000242D
:10F4C00093E04D48005D0690705D4B49085C0590E7
:10F4D000DDE90512881A05F0FAFE00221346CDE98F
:10F4E000000104F055FACDE9020105F0C3FE00F079
:10F4F000FF08404605F002FFCDE9000103F086FD5C
:10F50000CDE9020105F0B6FE00F0FF083B48005DC2
:10F51000715D3A4A515C884265D10498804562D158
:10F520003748005D8DF81C003648005D8DF81D00E1
:10F530003548005D8DF81E003448005D8DF81F00D1
:10F540003348007810B1012829D109E0314890F8FA
:10F550000090314890F800A0304890F800B01FE0CB
:10F56000F7F72AFE072190FBF1F201FB12002C496C
:10F5700008700846007800EB40002A4911F8009016
:10F580002748007800EB4000084490F801A0244888
:10F59000007800EB4000084490F802B000E000BFA3
:10F5A00000BF9DF81C0001280CD19DF81D001E49CC
:10F5B00001F800909DF81E0001F800A09DF81F00C2
:10F5C00001F800B09DF81C0002280CD19DF81D0028
:10F5D000164901F800909DF81E0001F800A09DF862
:10F5E0001F0001F800B0601CC4B22A2CFFF669AFFE
:10F5F00009B0BDE8F08F00003C5F0108E85E01083B
:10F60000405E01086A5E0108945E0108BE5E010862
:10F61000BD020020B6020020B7020020B802002080
:10F62000B50200208C600108661400203E15002001
:10F630002DE9F04F8BB081460C461746002600207E
:10F640000890099080468246079006900590FF201A
:10F65000049000254FF0000B00BF86E3FE48805D5C
:10F660008DF82000FD48805D8DF82100FC48805D0C
:10F670008DF82200FB48805D8DF823008DF8246012
:10F68000F948007801281FD1F84810F806A0504624
:10F6900005F034FE00221346CDE9000104F078F9AC
:10F6A000CDE9020105F0E6FD00F0FF08404605F057
:10F6B00025FECDE9000103F0A9FCCDE9020105F02A
:10F6C000D9FD00F0FF0820E0E94810F806A00799EE
:10F6D000AAEB010005F0FBFD00221346CDE9000175
:10F6E00004F056F9CDE9020105F0C4FD00F0FF0871
:10F6F000404605F003FECDE9000103F087FCCDE9AB
:10F70000020105F0B7FD00F0FF08B84504DA08F182
:10F710002400C01BC5B202E0A8EB0700C5B2D24866
:10F720000078012878D1C5BB05EB4501D14A515C71
:10F73000C4F108025143CF4A92F8692002FB041039
:10F74000C11700EB5171C1F3C701069105EB4501EB
:10F75000C84A11444978C4F108025143C54A92F895
:10F760006A2002FB0410C11700EB5171C1F3C701FD
:10F77000059105EB4501BF4A11448978C4F108029F
:10F780005143BC4A92F86B2002FB0410C11700EBF6
:10F790005171C1F3C70104913EE0FFE705EB45015C
:10F7A000B54A515CC4F1080251436A1E02EB4202A1
:10F7B000B14B9A5C02FB0410C11700EB5171C1F30D
:10F7C000C701069105EB45011A4611444978C4F179
:10F7D000080251436A1E02EB42021A44527802FBAD
:10F7E0000410C11700EB5171C1F3C701059105EB7E
:10F7F00045011A4611448978C4F1080251436A1E32
:10F8000002EB42021A44927802FB0410C11700EB8B
:10F810005171C1F3C701049193480078022859D16E
:10F82000B9F1000F7ED1EDBB9449495D944A12783D
:10F830005143FF2291FBF2F1C4F1080251438F4A78
:10F8400092F823208E4B1B785A43FF2392FBF3F24E
:10F8500002FB0410C11700EB5171C1F3C7010691FF
:10F860008649495D874A12785143FF2291FBF2F1A4
:10F87000C4F108025143814A92F82320814B1B783E
:10F880005A43FF2392FBF3F202FB0410C11700EB73
:10F890005171C1F3C70105917849495D7A4A1278DF
:10F8A000514300E017E0FF2291FBF2F1C4F108029E
:10F8B0005143724A92F82320734B1B785A43FF231B
:10F8C00092FBF3F202FB0410C11700EB5171C1F37C
:10F8D000C7010491ECE06949495D694A12785143D6
:10F8E000FF2291FBF2F1C4F1080251436A1E634BFF
:10F8F0009A5C634B1B785A43FF2392FBF3F202FBA3
:10F900000410C11700EB5171C1F3C70106915B49A7
:10F91000495D5C4A12785143FF2291FBF2F1C4F138
:10F92000080200E02EE051436A1E544B9A5C554B8E
:10F930001B785A43FF2392FBF3F202FB0410C1171A
:10F9400000EB5171C1F3C70105914C49495D4E4A25
:10F9500012785143FF2291FBF2F1C4F108025143A6
:10F960006A1E464B9A5C484B1B785A43FF2392FB16
:10F97000F3F202FB0410C11700EB5171C1F3C70190
:10F98000049195E0C5BB05EB4501404A515CC4F1CB
:10F99000080251433D4A92F8692002FB0410C11746
:10F9A00000EB5171C1F3C701069105EB4501374AE0
:10F9B00011444978C4F108025143344A92F86A204C
:10F9C00002FB0410C11700EB5171C1F3C70105918F
:10F9D00005EB45012D4A11448978C4F108025143D1
:10F9E0002A4A92F86B2002FB0410C11700EB5171F8
:10F9F000C1F3C70104915BE0FFE705EB4501234A32
:10FA0000515CC4F1080251436A1E02EB42021F4BD3
:10FA10009A5C02FB0410C11700EB5171C1F3C701DE
:10FA2000069105EB45011A4611444978C4F10802D4
:10FA300051436A1E02EB42021A44527802FB041040
:10FA4000C11700EB5171C1F3C701059105EB4501E9
:10FA50001A46114489781BE0405E01086A5E01087D
:10FA6000945E0108BE5E0108B9020020E45F01084F
:10FA7000125F0108A1600108796101084162010873
:10FA8000B6020020B7020020B80200200D61010874
:10FA9000C4F1080251436A1E02EB42021A449278F2
:10FAA00002FB0410C11700EB5171C1F3C7010491AF
:10FAB000B1480078032859D1B9F1000F7ED1EDBBD0
:10FAC000AE49495DAE4A12785143FF2291FBF2F1F3
:10FAD000C4F108025143A94A92F82320A84B1B788D
:10FAE0005A43FF2392FBF3F202FB0410C11700EB11
:10FAF0005171C1F3C7010691A049495DA14A12782D
:10FB00005143FF2291FBF2F1C4F1080251439B4A99
:10FB100092F823209B4B1B785A43FF2392FBF3F26E
:10FB200002FB0410C11700EB5171C1F3C70105912D
:10FB30009249495D944A1278514300E017E0FF2250
:10FB400091FBF2F1C4F1080251438C4A92F8232050
:10FB50008D4B1B785A43FF2392FBF3F202FB0410F8
:10FB6000C11700EB5171C1F3C7010491CFE0834984
:10FB7000495D834A12785143FF2291FBF2F1C4F1AF
:10FB8000080251436A1E7D4B9A5C7D4B1B785A4399
:10FB9000FF2392FBF3F202FB0410C11700EB51713B
:10FBA000C1F3C70106917549495D764A1278514300
:10FBB000FF2291FBF2F1C4F1080200E02EE0514374
:10FBC0006A1E6E4B9A5C6F4B1B785A43FF2392FB65
:10FBD000F3F202FB0410C11700EB5171C1F3C7012E
:10FBE00005916649495D684A12785143FF2291FBAD
:10FBF000F2F1C4F1080251436A1E604B9A5C624BF9
:10FC00001B785A43FF2392FBF3F202FB0410C11747
:10FC100000EB5171C1F3C701049178E0C5BB05EB5E
:10FC200045015A4A515CC4F108025143574A92F8BF
:10FC3000692002FB0410C11700EB5171C1F3C70129
:10FC4000069105EB4501514A11444978C4F1080277
:10FC500051434E4A92F86A2002FB0410C11700EB90
:10FC60005171C1F3C701059105EB4501474A1144A4
:10FC70008978C4F108025143444A92F86B2002FB90
:10FC80000410C11700EB5171C1F3C70104913EE0AC
:10FC9000FFE705EB45013D4A515CC4F108025143C1
:10FCA0006A1E02EB4202394B9A5C02FB0410C11738
:10FCB00000EB5171C1F3C701069105EB45011A46EE
:10FCC00011444978C4F1080251436A1E02EB420212
:10FCD0001A44527802FB0410C11700EB5171C1F3B2
:10FCE000C701059105EB45011A4611448978C4F115
:10FCF000080251436A1E02EB42021A44927802FB48
:10FD00000410C11700EB5171C1F3C70104919DF8B4
:10FD10002000012811D19DF824001D4901F800B0F0
:10FD20009DF821101B4A069850549DF82210059802
:10FD300050549DF82310049850549DF82000022838
:10FD400011D19DF82400144901F800B09DF821104C
:10FD5000124A069850549DF82210059850549DF868
:10FD6000231004985054701CC6B22A2EFFF676ACAD
:10FD70000BB0BDE8F08F0000B902002065620108F9
:10FD8000B6020020B7020020B80200207961010805
:10FD90001616002066140020EE1600203E150020E6
:10FDA0002DE9FF4106460F469046002466E035489F
:10FDB000005D8DF80C003448005D8DF80D0033486F
:10FDC000005D8DF80E003248005D8DF80F00FF25B4
:10FDD0003048007810B101280CD104E00296019758
:10FDE000CDF8008007E06B4601AA02A9204605F085
:10FDF000F5F800E000BF00BF9DF80C0001281BD102
:10FE00009DF808006843FF2190FBF1F09DF80D106C
:10FE1000214A50549DF804006843FF2190FBF1F003
:10FE20009DF80E1050549DF800006843FF2190FB90
:10FE3000F1F09DF80F1050549DF80C0002281BD1D2
:10FE40009DF808006843FF2190FBF1F09DF80D102C
:10FE5000124A50549DF804006843FF2190FBF1F0D2
:10FE60009DF80E1050549DF800006843FF2190FB50
:10FE7000F1F09DF80F105054601CC4B22A2C96DB90
:10FE8000BDE8FF81405E01086A5E0108945E0108DA
:10FE9000BE5E0108BD020020661400203E15002051
:10FEA0002DE9F04104460D4616461F46DDF8188040
:10FEB000691E01EB8102611E02EB01113944080346
:10FEC0004FF48072314601F0B1FABDE8F0810000D4
:10FED00000B5C1B01B480078022802D11A49087049
:10FEE0000CE018480078082802D11749087005E08E
:10FEF00014480078102801D1134908704FF480721B
:10FF000001A94FF4A04001F091FA0F4802780F4880
:10FF10000078401E0E490978491E032303FB0100A7
:10FF2000092101EB001001A90A54052001F0BCFAD7
:10FF30004FF4807201A94FF4A04001F0DEFA41B005
:10FF400000BD0000AD020020AB0200201302002023
:10FF50001202002010B5044600BF04210A4800F038
:10FF600057F80028F9D02146074800F091F800BF63
:10FF70000821054800F04CF80028F9D0024800F0AC
:10FF800066F8C0B210BD00000030004011B101227F
:10FF9000826001E0002282607047000010B50446D4
:10FFA0001748844208D101218014FDF705F900218A
:10FFB000A014FDF701F922E01248844208D1012182
:10FFC0004014FDF7F9F800216014FDF7F5F816E08C
:10FFD0000D48844208D101211020FDF7FDF80021D1
:10FFE0001020FDF7F9F80AE00848844207D1012102
:10FFF0002020FDF7F1F800212020FDF7EDF810BDDD
:020000040801F1
:100000000030004000340040009000400094004068
:1000100002460020936A0B400BB1012000E0002053
:1000200070474A884B891A43CB881A438B881A43F6
:100030000B881A4302600A89426170471AB103694A
:100040000B43036102E003698B4303617047014680
:10005000086E80B27047000010B5044600BF04214E
:100060000A48FFF7D5FF0028F9D02146074800F0DD
:100070000FF800BF08210548FFF7CAFF0028F9D094
:100080000248FFF7E4FFC0B210BD0000003000409E
:100090000166704730B5C1B04FF4807101A8F7F721
:1000A0009AF900240EE08D4A12783232120302EBE4
:1000B00004208B4A02EB04214FF4807201F0B6F960
:1000C000601CC4B2092CEEDB844909783231C8B215
:1000D00001F0EAF9834A1278521E834B1B785B1EAB
:1000E000032505FB03227E4B03EB022202F10800ED
:1000F0007A4A127802EBC2027C4B03EB42011022D7
:10010000F7F702F900240EE0744A12783232120333
:1001100002EB0420724A02EB04214FF4807201F0DA
:10012000ECF9601CC4B2092CEEDB4FF4807201A91B
:100130004FF4A04001F07AF96848027869480078E5
:10014000401E69490978491E032303FB010002216F
:1001500001EB001001A90A54654802786148007853
:10016000401E61490978491E03FB010003EB0010A2
:1001700001A90A545F4802785A480078401E5A493B
:100180000978491E03FB0100042101EB001001A9BD
:100190000A545948027853480078401E5249097859
:1001A000491E03FB0100052101EB001001A90A54BF
:1001B000524802784B480078401E4B490978491E46
:1001C00003FB0100062101EB001001A90A544C4871
:1001D00090F8012243480078401E43490978491E9F
:1001E00003FB0100072101EB001001A90A54454857
:1001F00002783C480078401E3B490978491E03FBC1
:100200000100082101EB001001A90A543E480278C0
:1002100034480078401E34490978491E03FB010028
:10022000092101EB001001A90A54384802782D4831
:100230000078401E2C490978491E03FB01000A2161
:1002400001EB001001A90A543148027825480078D2
:10025000401E25490978491E03FB01000B2101EBD3
:10026000001001A90A542B4802781E480078401E4D
:100270001D490978491E03FB01000C2101EB001008
:1002800001A90A541E4890F8022216480078401E20
:1002900015490978491E03FB01000D2101EB0010EF
:1002A00001A90A541C4802780E480078401E0E49E5
:1002B0000978491E03FB01000E2101EB001001A982
:1002C0000A54052001F0F0F84FF4807201A94FF4B0
:1002D000A04001F012F941B030BD0000B902002089
:1002E0008C1D00201302002012020020C6170020DF
:1002F000A8020020A9020020A6020020B1020020CE
:10030000300A002098090020AB020020D302002010
:10031000A7020020B2020020210000202DE9F047B2
:100320000746884616469946089D00240DE005F1CB
:100330003202120302EB0420204A02EB04214FF4A4
:10034000807201F073F8601C84B2092CEFDB05F1B8
:100350003201C8B201F0A8F800240CE0325DA8F127
:100360000100791E032303FB0100144901EB002067
:100370000255601C84B2FF2CF0DD00240DE005F175
:100380003202120302EB04200C4A02EB04214FF468
:10039000807201F0B2F8601C84B2092CEFDB05EB2F
:1003A000C501074A02EB4100102206F10801F6F7E9
:1003B000ABFF002003490870BDE8F0878C1D0020CA
:1003C000C6170020B90200202DE9F05F81468A4659
:1003D0001646DDE90A78002414E0284A92F800B0B5
:1003E0004FEAEB720BEB127212115A32120302EB4C
:1003F0000420234A02EB04214FF4807201F016F826
:10040000601CC4B2102CE8DB1C4991F800B04FEA24
:10041000EB710BEB1171091101F15A0001F044F875
:1004200000250EE0715D154A1078C21700EB1272BC
:100430001211A0EB0212124B03EB02225155681C61
:1004400085B2FF2DEEDD002414E00C4A92F800B0D6
:100450004FEAEB720BEB127212115A32120302EBDB
:100460000420074A02EB04214FF4807201F045F8A2
:10047000601CC4B2102CE8DBBDE8F09F160200201F
:100480008C1D00202DE9F04104460D461646984685
:10049000069F691E01EB8102611E02EB0111C91C5E
:1004A000C8B201F001F8691E01EB8102611E02EB86
:1004B0000111C91C08034FF48072314601F01DF888
:1004C000691E01EB8102611E02EB0111C91C0803C8
:1004D0004FF48072314600F0A9FF4FF4807231462C
:1004E0000248F6F711FFBDE8F08100008C2F0020D4
:1004F0002DE9F04705460E4617469846DDF8209050
:10050000711E01EB8102691E02EB01114144C8B268
:1005100000F0CAFF711E01EB8102691E02EB01119E
:10052000414408034FF48072394600F0E6FF711E23
:1005300001EB8102691E02EB0111414408034FF4F3
:100540008072394600F072FF00240BE004F10800CD
:10055000385C0649085504F11C00385C044908550C
:10056000601CC4B2142CF1DBBDE8F087DE13002060
:10057000F21300202DE9F04705460E4614461F46AB
:10058000DDE90889607948B9711E01EB8102691EB5
:1005900002EB0111891CC8B200F086FF711E01EB4D
:1005A0008102691E02EB0111891C0A03617902EBC9
:1005B00001204FF48072214600F09FFF00204CE0A4
:1005C00000EB80010831615C6279C2EBC20202EB90
:1005D000420200EB420202EB8202324B1A4451709B
:1005E00000EB80010931615C6279C2EBC20202EB6F
:1005F000420200EB420202EB8202995400EB8001BE
:100600000A31615C6279C2EBC20202EB420200EB8A
:10061000420202EB82021A44917000EB80010B311E
:10062000615C6279C2EBC20202EB420200EB420261
:1006300002EB82021A44D17000EB80010C31615C44
:100640006279C2EBC20202EB420200EB420202EB11
:1006500082021A441171411CC8B22A28B0DB6079A9
:10066000F0B9A079104908704FF4807239464FF400
:10067000A04000F0DBFE0C480278701E691E0323C8
:1006800003FB0100062101EB00103A54052000F0A5
:100690000BFF4FF4807239464FF4A04000F02DFF5D
:1006A000BDE8F087741A0020B10200202DE9F04760
:1006B00006460F4614461D46DDE908894FF4807250
:1006C00029464FF4A04000F0B1FEA278781E711EBA
:1006D000032303FB010005EB00100270E278781E93
:1006E00003FB0100012101EB00102A542279781E3E
:1006F000711E03FB0100022101EB00102A546279F4
:10070000781E711E03FB010003EB00102A54A2792E
:10071000781E03FB0100042101EB00102A54E2794A
:10072000781E711E03FB0100052101EB00102A5405
:10073000227A781E711E03FB0100072101EB0010D5
:100740002A54627A781E711E03FB0100082101EB16
:1007500000102A54A27A781E711E03FB01000921A1
:1007600001EB00102A54E27A781E711E03FB01008F
:100770000A2101EB00102A54227B781E711E03FB14
:1007800001000B2101EB00102A54627B781E711EC0
:1007900003FB01000D2101EB00102A54E0790D4903
:1007A0000870607A0C490870A07A0C490870E07AE9
:1007B0000B490870207B0B490870052000F074FE7F
:1007C0004FF4807229464FF4A04000F096FEBDE839
:1007D000F0870000A602002098090020AB0200204C
:1007E000D3020020A702002010B5C0B004464FF489
:1007F00080716846F6F7EFFD207A8DF80000002042
:1008000006E004F10B010A5C411C0DF80120C8B29E
:100810000928F6DB0A2000F047FE4FF48072694693
:100820004FF4204000F069FE40B010BD2DE9F047C4
:1008300005460E4614461F46DDE90889607948B929
:10084000711E01EB8102691E02EB0111091DC8B284
:1008500000F02AFE711E01EB8102691E02EB0111FC
:10086000091D0A03617902EB01204FF480722146D1
:1008700000F043FE00204CE000EB80010831615C99
:100880006279C2EBC20202EB420200EB420202EBCF
:1008900082023B4B1A44517000EB80010931615CCC
:1008A0006279C2EBC20202EB420200EB420202EBAF
:1008B0008202995400EB80010A31615C6279C2EBDB
:1008C000C20202EB420200EB420202EB82021A4435
:1008D000917000EB80010B31615C6279C2EBC20266
:1008E00002EB420200EB420202EB82021A44D17098
:1008F00000EB80010C31615C6279C2EBC20202EB59
:10090000420200EB420202EB82021A441171411CC6
:10091000C8B22A28B0DB607978BBA0791949087081
:10092000E07908B1012000E00020174908704FF479
:10093000807239464FF4A04000F078FD11480278EB
:10094000701E691E032303FB01000C2101EB001044
:100950003A540D480278701E691E03FB01000E21F7
:1009600001EB00103A54052000F09EFD4FF4807218
:1009700039464FF4A04000F0C0FDBDE8F08700000C
:10098000461B0020B20200202100002030B589B0B3
:1009900004460025202101A8F6F71DFD0D21A01E0B
:1009A00001AA11540A21601E11544FF48071880568
:1009B000F9F74AFF1420F9F71FFA002011490880BF
:1009C00000BF0EE000BF104801F025FA00F0200043
:1009D0000028F8D001A8415D0B4801F05FFA681CBF
:1009E000C5B2A542EEDB00BF074801F014FA00F0E3
:1009F00040000028F8D04FF480718805F9F721FFF6
:100A000009B030BD000A00200038004010B50024B5
:100A10002E48B0F8EE01642857DB00202B49A1F8DE
:100A2000EE01084690F8890100284EDD084690F84E
:100A30008A01052806D006280DD0072814D00828DA
:100A400028D11EE0F7F7C2FD052000F043F80A2088
:100A500003F078FD1EE0F7F7FDFD062000F03AF800
:100A60000A2003F06FFD15E00420184981F8FA010F
:100A7000F7F7D6FD072000F02DF80A2003F062FDFD
:100A800008E0F7F7D5FF082000F024F80A2003F06B
:100A900059FD00BF00BF0D4890F88901401E0B4969
:100AA00081F88901084690F8890100280DDD0024AD
:100AB00005E00748611C415C0155601CC4B2034855
:100AC00090F88901401CA042F3DC10BD300A0020E0
:100AD000BA0B002010B5044601202D4981F82002F0
:100AE000002081F8210281F8220281F8230248E0E7
:100AF000274890F821021E2843DB254890F823025E
:100B000038B90120224981F823021120FFF73EFF66
:100B100019E000201E4981F82302052C06D0062C7E
:100B200007D0072C08D0082C0CD108E0F7F74EFDB1
:100B300008E0F7F78FFD05E0F7F772FD02E0F7F741
:100B400077FF00BF00BF0020114981F8210208464D
:100B500090F82202401C81F82202084690F82202F6
:100B6000C8280EDB4FF480410A48F9F76AFE4FF4BB
:100B70007A7003F0E7FC4FF480410648F9F764FE11
:100B800004E0034890F820020128B1D000BF10BD56
:100B9000300A00200004004010B500F001F810BD3C
:100BA0000CB50020019000900320354988620C208C
:100BB000C8628020334908600846006808604FF426
:100BC000014030492C3108604FF6FC702E49086016
:100BD0000F202D493039086002202C49086001207F
:100BE000091F086000BF29480830006800F00100B4
:100BF00000900198401C0190009820B94BF680317C
:100C000001988842EFD1009888B3214821490860B3
:100C100000201C49091F086080201A49091D08602E
:100C2000084600680860012016491839086020202D
:100C3000091F08600846006808600846006840F020
:100C400001000860C0201149243108600120091DFD
:100C5000086000BF0D482C3000680328FAD102203C
:100C60000849143908600120091D086002E0FFE707
:100C700000BFFEE7002002498862C8620CBD000088
:100C8000000001401C0C0140300C004050040140A9
:100C90001200000300540140002017490870174952
:100CA00008700820164908700120164908701420A1
:100CB00015490870154981F80102122081F80202D5
:100CC00001201349087000201249087001201249C0
:100CD00008701249087012490870124908701420EF
:100CE00011490870002011490870FF201049087050
:100CF0000020104908707047A8020020A9020020B7
:100D0000AB020020D3020020B2020020300A0020F3
:100D1000B1020020A6020020A7020020B902002094
:100D2000D6020020B4020020B3020020980900205F
:100D300020000020210000202DE9FE4F82468B4636
:100D4000144603200290384810F80A50374810F82B
:100D50000A900299481B04F0BAFA0746002213468B
:100D600002F016FECDE9000104F084FAC6B2304666
:100D700004F0C4FACDE9000102F048F9074604F096
:100D800079FAC6B24FF0000BB9F1000F07D1032D6D
:100D900005DCA019012843DB4FF0FF0B40E0B9F15F
:100DA000010F07D1032D05DCA019022838DB4FF015
:100DB000FF0B35E0B9F1020F07D1032D05DCA019B7
:100DC00003282DDB4FF0FF0B2AE0B9F1030F07D109
:100DD000032D05DBA019032822DB4FF0FF0B1FE0DA
:100DE000B9F1040F07D1032D05DBA019052817DB86
:100DF0004FF0FF0B14E0B9F1050F07D1032D05DB10
:100E0000A01905280CDB4FF0FF0B09E0B9F1060F24
:100E100006D1032D04DBA019052801DB4FF0FF0BE1
:100E20005846BDE8FE8F00003C5F0108E85E0108FF
:100E300010B50346002102F007040348005D984204
:100E400000D1FF21084610BD286201082DE9F04FAE
:100E500087B004460D4616460320059004901848B6
:100E6000005D03901748005D0290029A0499881A69
:100E700004F02DFACDE90001039A0599881A04F0CF
:100E800026FA0746DDE9002302F082FD824604F0DF
:100E9000F1F900F0FF09484604F030FA074602F085
:100EA000B5F8824604F0E6F900F0FF090025A6F146
:100EB0001D00484500DBFF25284607B0BDE8F08F40
:100EC0003C5F0108E85E01081C4A02EB8002525CAC
:100ED000012A19D1194A283202EB8002525C5AB910
:100EE0000023164A02EB800253540123134A1432A2
:100EF00002EB800253541FE0114A92F80822521C60
:100F00000F4B83F8082217E00C4A283202EB8002CC
:100F1000525C012A10D10123084A02EB800253548B
:100F2000064A143202EB80025354054A92F8082212
:100F3000521C034B83F80822704700005D0C002010
:100F4000300A002078B50446264D2D78012D0DD1AC
:100F5000072B0BD003EB4305234E745D03EB4305D6
:100F60003544697803EB43053544AA78002035E021
:100F70001E4D2D5C1E4E755D8DF800501B4D2D5C79
:100F80001C4E755D8DF80150184D2D5C1A4E755D27
:100F90008DF80250154D2D5C184E755D8DF803507F
:100FA0009DF80050012D09D19DF80150144E745543
:100FB0009DF8025071559DF8035072559DF80050F0
:100FC000022D09D19DF801500E4E74559DF8025026
:100FD00071559DF803507255451CE8B20E28C7D3D1
:100FE00078BD0000BD0200208C6001088962010804
:100FF000405E01086A5E0108945E0108BE5E010859
:10100000661400203E15002010B53D4800880028D9
:1010100074D03C48007801282ED104203A49087049
:10102000FA204870364800788870354800880012E9
:10103000C8700020087148718871C87108723348FF
:10104000007838B904200870042215212E4803F0D6
:101050002FFE0DE0042215212B4803F029FE50211C
:101060002B48F6F796F901221521294803F020FEB6
:1010700000202349088041E02148008802F0D0FD8B
:1010800028B1E920234948700020887004E0EA2054
:1010900020494870002088701E4844781B4800781A
:1010A00018B903201B49087002E002201949087092
:1010B0001348008808B302F0C3FB04281DDD15485F
:1010C00044700222152103F0F3FD002011494870FD
:1010D000022215210F4803F0EBFD0948008800F4B7
:1010E000004028B106480088401C0549088004E0FB
:1010F00003480088401E0249088000BF10BD000060
:101100002A000020210000204B0D00201F0000209D
:10111000E20C0020F401002008B56F49087800EBCC
:1011200080016E4A1144497800297DD000EB80018E
:10113000515C6B4A515C8DF8001000EB8001674AEE
:10114000515C684A515C8DF8011000EB8001634AE4
:10115000515C654A515C8DF8021000EB80015F4ADA
:10116000515C624A515C8DF8031000EB80015B4AD0
:1011700011444978FF2902D15D4A11704BE05D4965
:101180000978012920D100EB8001544A11444978A3
:10119000FE290DD100EB800111444978491E00EB76
:1011A00080024E4B1A4451700021524A11702BE0BC
:1011B00000EB8001494A11444978491C00EB800248
:1011C000464B1A4451701FE000EB8001434A114422
:1011D000497801290DD100EB800111444978491C5F
:1011E00000EB80023D4B1A4451700121414A1170BD
:1011F0000AE000EB8001394A11444978491E00EBAE
:101200008002364B1A44517000EB8001334A11447E
:101210004978374A11709DF8001001292CD100EB54
:1012200080012E4A114400E055E08978304A127856
:101230005143FF2291FBF2F19DF801202E4B99546E
:1012400000EB8001254A1144C978294A127851439C
:10125000FF2291FBF2F19DF80220995400EB8001EE
:101260001E4A11440979224A12785143FF2291FB08
:10127000F2F19DF8032099549DF8001002292AD11B
:1012800000EB8001154A11448978194A12785143BC
:10129000FF2291FBF2F19DF80120184B995400EBCD
:1012A00080010E4A1144C978114A12785143FF2235
:1012B00091FBF2F19DF80220995400EB8001074A5E
:1012C000114409790A4A12785143FF2291FBF2F145
:1012D0009DF80320995408BD20000020461B0020E3
:1012E000405E01086A5E0108945E0108BE5E010866
:1012F000DB020020DA020020661400203E150020E8
:1013000010B52A48007801284FD1002027490870DD
:101310002748007858B126480078012807D024488B
:101320000078072803D022480078112802D1012034
:10133000204908701F4800781D49097801EBC10158
:101340001D4A02F81100FEF7A5FE04201B49087093
:10135000F22048701A48007888701A480078C870DF
:1013600013480078087113480078487116480078CF
:1013700088710020C87108721448007838B90420B8
:101380000870042215210D4803F092FC0DE00422A0
:1013900015210A4803F08CFC50210D48F5F7F9FFA0
:1013A000012215210A4803F083FC10BDB40200207D
:1013B000B9020020B3020020C61700204B0D002008
:1013C0001202002013020020B00200201F000020A3
:1013D000E20C002070B504460D46164600F0B0F849
:1013E00040211148F9F72DFA0220FEF7B3FDC4F3AE
:1013F0000740FEF7AFFDC4F30720FEF7ABFDE0B2F8
:10140000FEF7A8FD03E015F8010BFEF7A3FD301E63
:10141000A6F101018EB2F6D140210348F9F714FA82
:1014200000F062F870BD00000004004070B5044692
:101430000D46164640211048F9F703FA0320FEF73F
:1014400089FDC4F30740FEF785FDC4F30720FEF7CE
:1014500081FDE0B2FEF77EFD04E0FF20FEF77AFD9D
:1014600028706D1C301EA6F10106F6D140210248FD
:10147000F9F7EAF970BD00000004004010B500243F
:1014800040210848F9F7DDF90520FEF763FDFF204C
:10149000FEF760FD044640210248F9F7D5F92046E1
:1014A00010BD00000004004070B505462C0300F09C
:1014B00047F840210B48F9F7C4F92020FEF74AFD10
:1014C000C4F30740FEF746FDC4F30720FEF742FDD4
:1014D000E0B2FEF73FFD40210248F9F7B5F900F010
:1014E00003F870BD0004004010B500BFFFF7C6FF51
:1014F00000F001000028F9D110BD2DE9F0410646A9
:101500000F461446F0B2C0F58075AC4200D82546AF
:1015100011E0AAB239463046FFF75CFFAC4200D179
:101520000AE02F442E44641BB4F5807F02D94FF4A7
:10153000807500E02546ECE700BFBDE8F0810000C3
:1015400010B540210548F9F77CF90620FEF702FDA9
:1015500040210248F9F778F910BD0000000400406E
:1015600001464FF0E022516100224FF0E0239A61E2
:1015700005221A6100BF4FF0E022106900F001025D
:101580001AB100F48032002AF5D04FF0E02212693F
:1015900022F001024FF0E0231A61704710B51348A2
:1015A0000068401C114908600846006840F6B831E0
:1015B00088421AD300200D4908600D48D0F8040273
:1015C00078B94FF400510B48F9F73BF94FF48041DB
:1015D0000848F9F736F900F0E5FC00F0E7FC01F007
:1015E0001FFC00200249C1F8040210BD5400002075
:1015F000300A00200004004030B5214C246834B18A
:10160000012C06D0022C08D0032C27D103E01D4862
:1016100026E01D4824E01D4822E0194C083C2468BF
:1016200004F01F04641C012505EB5401184C2468C8
:10163000C4F38114C4F103040C2505EB8402104C9F
:10164000241F2468012C04D1104C5443B4FBF1F046
:1016500003E00C4C5443B4FBF1F001E0094800BF37
:1016600000BF074C1034246804F07F04641C01257B
:1016700005EB5403B0FBF3F4064D2C6030BD0000C5
:10168000080C014000127A00006CDC02001BB7005D
:1016900074040140A809002010B50320094988629C
:1016A0000C20C86240F2BE7007490860002005495E
:1016B0008862C862FFF770FA4FF000600349086063
:1016C00010BD0000000001409404014008ED00E05E
:1016D00010B501217E4800F0BFF900287ED001211D
:1016E0007B4800F06FF97B4890F81202401C794962
:1016F00081F8120278480068401C774908607748F2
:101700000068401C7549086075480068401C7449B1
:10171000086074480068401C72490860724800689C
:10172000401C7149086071480068401C6F4908609E
:101730006F480068401C6E4908606E480068401C95
:101740006C49086063484069401C6249486108462A
:10175000D0F82001401CC1F820010846C068401C98
:10176000C86008460068401C086008460069401CC4
:1017700008610846B0F8EE01401CA1F8EE010846E9
:10178000D0F8F401401CC1F8F4010846D0F8FC017F
:10179000401CC1F8FC010846D0F81802401CC1F8F2
:1017A0001802084690F82102401C81F82102524894
:1017B000008840F6B831884204DA4F480088401C5F
:1017C0004D4908804D48007820B14D480088401CA4
:1017D0004B4908804B48007830B100E076E04A4839
:1017E0000088401C4849088048480088401C4749F8
:1017F000088047480078062804D146480088401CE5
:10180000444908804248007803280AD142480088A9
:1018100040F6B831884204DA3F480088401C3E490F
:1018200008803B480078072809D13C480088B0F57B
:10183000FA6F04DA39480088401C38490880384873
:10184000007820B937480068401C364908602148B4
:10185000D0F80C02401C1F49C1F80C023248007835
:10186000002804DD31480068401C304908603048D9
:10187000008820B12E480088401E2D4908802D4840
:101880000078012804D12C480068401C2A490860CF
:101890002A480088002804DD28480088401E27497F
:1018A000088027480078002804DD25480078401E7D
:1018B000234908702348007818B12348007801288C
:1018C00004D122480088401C2049088010BD000037
:1018D00000200040300A0020480200204C02002076
:1018E0006402002060020020580200205402002000
:1018F000500200205C0200200200002016000020A0
:10190000180000201A0000201C0000206C0200209B
:10191000B609002070020020740200207602002028
:101920003400002008000020A002002068020020EF
:10193000BC09002035000020780200206E02002043
:10194000440200203A000020380000200C00002053
:101950007FB505460C46012148F20400FBF71CFC4C
:10196000174800F03FF80121154800F0AFF8029544
:10197000ADF804400020ADF80C00ADF8060001A958
:101980000F4800F087F801210D4800F01BF80122F4
:1019900011460B4800F071F815208DF8000000206A
:1019A0008DF801008DF8020001208DF803006846D3
:1019B000FBF7B4F80121024800F008F87FBD0000F1
:1019C00000200040CA4392B20261704721B1026810
:1019D00042F00102026004E002684FF6FE731A4012
:1019E0000260704710B504461748844208D10121AF
:1019F0000220FBF7E1FB00210220FBF7DDFB22E0E8
:101A00001248844208D101210420FBF7D5FB0021B4
:101A10000420FBF7D1FB16E00D48844208D10121D8
:101A20000820FBF7C9FB00210820FBF7C5FB0AE0F3
:101A30000848844207D101211020FBF7BDFB00219B
:101A40001020FBF7B9FB10BD001C00400020004037
:101A5000002400400028004030B50246002000234A
:101A60000024156905EA0103D56805EA010413B1EC
:101A70000CB1012000E0002030BD10B51AB1C368E0
:101A80000B43C36004E0C368CC43A4B22340C360EB
:101A900010BD0000002203689AB24FF68F731A40FF
:101AA0004B881A434FF6FF431A400B891A430260D2
:101AB0004B68C3620B888362034B984201D18B7AD7
:101AC0000363012343617047001C004021B1026899
:101AD00042F00402026004E002684FF6FB731A4011
:101AE0000260704770B500249C4800F08FF90646EC
:101AF000042E7CD1994800F0CDF9C5B29848994997
:101B0000098845540020984908700C20974908809E
:101B10000020974981F821020A2D69D19148008857
:101B2000012865DD8F480088401E8D49085C0D281E
:101B3000F3D101208C49087000BF1BE08848005D8C
:101B40004F2815D18649601C085C4B2810D1A01C79
:101B5000085C0D280CD1E01C085C0A2808D18448D8
:101B600090F8230218B90220814981F8200270BD43
:101B7000601CC4B27B4800888442DFDD002406E09C
:101B80007748005D2B2800D105E0601CC4B2754881
:101B900000888442F4DD00BF00207249088070494B
:101BA000081907227349F5F75FFB28B96C492144EE
:101BB000C81D01F0B5FCDAE76949081906226E492B
:101BC000F5F752FB20B966492144881D01F08EFCCF
:101BD0006349081909226949F5F746FB68B90020ED
:101BE0006749087004F109005D49085C01E0B1E053
:101BF00085E000F001006349087059490819062280
:101C00006149F5F731FB002887D155482044807998
:101C10005E49087001205E4908701E205D490880F9
:101C20005A48007868B94FF480715B48F5F7B1FB0A
:101C30004FF480715948F5F7ACFB01205849087002
:101C400077E052480078FF280FD1421C5349524890
:101C5000F5F75AFB012053490870002052490870DB
:101C6000524908704E49087063E0484800780128DE
:101C700046D1464800784C490978884219DD384AEF
:101C80002244D11D414A1278521E02EB420303EB5B
:101C90000213424A521C98181322F5F735FB4348A9
:101CA0000078401C41490870384800783E49087067
:101CB0003FE0364800783C490978884239DC4FF4E7
:101CC000807236493448F5F71FFB0120354908700A
:101CD0003549087035480078401C34490870204A5E
:101CE0002244D11D294A1278521E02EB420303EB13
:101CF00002132A4A521C98181322F5F705FB18E024
:101D0000174A2244D11D214A1278521E02EB420387
:101D100003EB0213214A521C98181322F5F7F4FA28
:101D200022480078401C21490870184800781E4954
:101D300008700C480088401C0A4908800846008842
:101D4000B0F5C87F07D30120194908700020054964
:101D5000088000E000BF00BF09E700000038004035
:101D60004A410020000A002032000020BC09002067
:101D7000300A0020050A0020240A0020150A00204D
:101D800047000020140200201E0A00202B0A002019
:101D90004F0000206E020020540E0020540D002041
:101DA000500000204E0000202C0A00202A0A0020AB
:101DB000040A002010B504461148844208D10121CC
:101DC0000014FBF7F9F900212014FBF7F5F916E0F0
:101DD0000C48844208D101210420FBF7FDF90021C1
:101DE0000420FBF7F9F90AE00748844207D10121F2
:101DF0000820FBF7F1F900210820FBF7EDF910BDF1
:101E0000003800400080004000840040014688689F
:101E100000F00F0070470146486970471AB14368E7
:101E20000B43436002E043688B434360704700000C
:101E30002DE9FF4104460D46206900F05000E97984
:101E4000084320616846FBF7D7F91148844201D165
:101E5000029F00E0039F286807EB50002968B0FB51
:101E6000F1F606F00F00C4F8C0008020E060C6F371
:101E700007102060C6F3073060600020E06028791A
:101E800069790843A9790843E060BDE8FF81000053
:101E9000003800400146086880B270470160704712
:101EA00010B54FF4A060FAF771FE01214CF260000A
:101EB000FBF772F94FF0805211158805F8F798FC7E
:101EC0004FF480718805F8F7BCFC144A4FF4C061E8
:101ED0004FF08040F8F78CFC1148FFF76BFF4FF490
:101EE000E1301049086003200871002048718871B2
:101EF000C8710B48FFF79CFF1E200B49087000209B
:101F0000487088700120C8700846FAF707FE012261
:101F100011460348FFF782FF10BD000007000120B3
:101F200000380040F8090020F409002010B500F046
:101F3000CBFB10BD10B501200549C87100204872C7
:101F400014210448F5F747FA00F0A2FD10BD000087
:101F5000004001408C30002010B50548807C0328EB
:101F600005D100F0C5FD0248C07C0149887410BD50
:101F70008C30002010B50648807C032807D0044828
:101F8000807C0349C8740320887400F0EDFD10BD07
:101F90008C30002002480078401C014908707047CE
:101FA0000400002010B500F0A9FB10BD10B500F032
:101FB000DDFB10BD70B50020834988730846447C62
:101FC00004F0040018B1002048748049087004F03F
:101FD000100028B180207C49487400207B4908709B
:101FE0007A480078002845D104F00100002841D04B
:101FF000002508227649002000F0FCF900207449F1
:1020000088600846C08888810020C881084600781A
:1020100000F0600010B900F057F9054615B900F05E
:1020200007FC0546002068498873012D04D0022D65
:1020300009D0032D15D10DE04020634948740120DB
:102040006249087014E040205F49487402205F49EB
:1020500008700DE048205C49487400205B49087016
:1020600006E060205849487403205849087000BFB2
:1020700000BF00BF55480078012850D104F002008D
:1020800000284CD15048447C04F0100018B104F0F2
:102090000100002843D102244D4880894D49097828
:1020A000884213DA4A4882898168802000F0DEF98C
:1020B0004748C0894649898908444549C881002064
:1020C000888144F00804414908701BE04048816859
:1020D00040480278802000F0C9F93D4880683D49B9
:1020E000097808443A49886008468089394909785E
:1020F000401A374988810846C0893649097808441A
:102100003349C8813248C0893149C988884204D1DD
:1021100044F0080400202D4908702B4844742B48D3
:10212000007802284FD12848447C04F001000028A0
:1021300049D04024264880892649097888420FDA08
:10214000234882898168002000F054F92048C08922
:102150001F49898908441E49C881002088811BE0E5
:102160001B4881681B480278002000F043F918489A
:1021700080681849097808441549886008468089AC
:1021800014490978401A124988810846C0891149C2
:10219000097808440E49C8810D48808988B944F0FF
:1021A000080400F02BFB032805D044F02004032092
:1021B0000649087002E00020044908700020024926
:1021C00088730148447470BD00400140AE0900208E
:1021D0008C3000204863010810B507484078092872
:1021E00006D1012000F0E2FB08B1032010BD00BFC2
:1021F00000BF0020FAE700008C30002008B531480D
:10220000007800F06000202839D12E4840780C2852
:1022100034D2DFE800F033060C1633333333332087
:10222000272D00F08DFB08B1012008BD26E02548D0
:10223000C088012804D100F077FB08B10120F4E741
:102240001CE02048C088012804D100F06FFB08B1D1
:102250000120EAE712E0002000F0A8FB08B102200C
:10226000E3E70BE000F096FB08B10320DDE705E0B3
:1022700000F092FB08B10320D7E700BF20E011482F
:10228000007800F06000D8B90E484078062817D1D1
:102290000C4AD17810796A4600F0FCFA0949886046
:1022A0000846806858B108468089BDF80010884209
:1022B00003DDBDF80000034988810120B5E700BFB8
:1022C0000020B2E78C30002010B5314840780A2851
:1022D0005AD2DFE800F0050F5916591D2659305023
:1022E0002B48C088022804D100F014F908B101205D
:1022F00010BD4AE0002000F061F908B10320F7E7C3
:1023000043E0012000F05AF908B10320F0E73CE077
:102310001F48007820B900F037F908B10320E7E73B
:1023200033E01B480078802804D100F0BDF808B1E4
:102330000120DDE729E01648007880281AD11448EA
:10234000C088012816D11248807C20B1012803D012
:1023500002280FD108E000BF00200E49088008467F
:102360000B4988600120C3E709481030084988609C
:102370000120BDE709E00648007820B900F052F9D5
:1023800008B10320B4E700E000BF00BF0020AFE7C2
:102390008C300020AC09002000F00F0159B1064A32
:1023A000917300F080021AB14022034B5A7402E08C
:1023B0008022014B1A75704700400140014601F030
:1023C0000F0292B10A48827301F0800030B10848D0
:1023D000407C00F0100040B1012070470448007DAF
:1023E00000F0200008B10120F7E70020F5E7000029
:1023F0000040014030B500F00F04064D05EB8403AA
:1024000004E01C7801F8014B541EA2B2002AF8D156
:1024100030BD00002040014000F00F0159B1064AD4
:10242000917300F080021AB11022034B5A7402E03B
:102430002022014B1A75704700400140F0B5044658
:102440000E4617463A463146204600F00FF804F093
:102450000F053DB104F0800020B1034885730120D1
:1024600001494874F0BD00000040014030B500F063
:102470000F04064D05EB840304E011F8014B1C70BA
:10248000541EA2B2002AF8D130BD00002040014005
:1024900010B514210248F4F79EFF00F0C1FA10BDF8
:1024A0008C3000207047000008B51948C07801281A
:1024B00004D0022808D0032816D10DE0684600F0A9
:1024C000E1F91349886011E011498878694600F004
:1024D000C9F90F49886009E00D498878694600F01C
:1024E00013FA0B49886001E0002008BD00BF0848CE
:1024F000806808B90020F8E705488089BDF8001019
:10250000884203DDBDF80000014988810120ECE725
:102510008C30002038B5002019490880194800780F
:1025200000F01F0020B1012819D0022820D117E0A7
:102530001449087C694600F095F90446E07900F0FA
:10254000400010B101200E4908800E48407C28B19F
:102550000B48008840F00200094908800AE009E0C1
:10256000084805792846FFF729FF0549088001E05A
:10257000002038BD00BF0248024988600120F8E70A
:10258000AC0900208C3000200A48807800F07F01E0
:102590000848807C02280BD00748017019B101203F
:1025A000044A907402E00020024A907401207047AF
:1025B0000020FCE78C3000200040014070B505464B
:1025C0001748007800F01F0010B1022824D10DE058
:1025D00013484088012808D115B11149487402E018
:1025E00000200F494874012070BD15E00C48408858
:1025F00088B90B48047904F00F0060B11DB1E0B256
:10260000FFF70AFF05E0E0B2FFF7C6FEE0B2FFF712
:1026100049FF0120E8E700BF00BF0020E4E7000019
:102620008C30002010B51D488478807C012802D0B1
:1026300002282CD10EE054B1204600F05BFA40B1E4
:1026400016480474022015498874012010BD012029
:10265000FCE720E04CB90020104908740120887480
:10266000002000F01DF80120F0E70C48007CA0429B
:102670000AD0204600F014F8204600F03BFA28B1BA
:10268000064804740120E1E70120DFE703E020466B
:1026900000F006F800BF00BF0020D7E78C30002014
:1026A0000849C97921F00201064AD1711146C97958
:1026B00021F00401D1711146C97921F00801D171CD
:1026C000704700000040014010B5012148F2200091
:1026D000FAF762FD0322D1024FF08040F8F77EF84E
:1026E000044AD1024FF08040F8F782F80E200249E8
:1026F000C87210BD030000200040014010B50E203C
:10270000002817DB00F01F0201219140154A430900
:1027100042F8231000BF00BF00BFBFF34F8F00BFC0
:1027200000BF00BF00BF00BF00BFBFF36F8F00BF7F
:1027300000BF00BF00BF00210846FAF7CFFDFAF73F
:10274000A1FA0948006820F01F0007490860FAF75D
:1027500091FA0020FAF7EAFD00214FF40070FAF731
:10276000DBFC10BD80E100E09004014010B50121C8
:1027700048F22000FAF710FD00224FF4C0514FF04C
:102780008040F8F735F84FF088524FF480518804B4
:10279000F8F72EF84FF480518804F8F752F810BD7E
:1027A00000200149086070471C02002070470000AB
:1027B000002008490860084908600849086008497D
:1027C0000860084908600849086008490860084925
:1027D0000860704720020020240200202802002008
:1027E0002C02002034020020300200203C02002095
:1027F00038020020704770477047000010B5002471
:102800000A48007800F07F0021280DD107480079A0
:1028100038B106480079012803D00448007902281D
:1028200002D1FFF7D9FC0446204610BD8C300020B1
:1028300010B500240A48007800F01F0001280DD1CF
:102840000748007938B106480079012803D00448C8
:102850000079022802D1FFF7D1FC0446204610BDC2
:102860008C3000200246012A08DA05488078044BA3
:10287000DB7840EA03200880014870470020FCE72D
:10288000075C0108014612200880014870470000DB
:10289000F55B0108034663B9212902D0222928D11A
:1028A00003E009201080144870474120108013482D
:1028B000FAE7012B0DD1212902D0222919D104E0F8
:1028C000092010800C481930EEE7DC2010800C48FD
:1028D000EAE7022B0DD1212902D0222909D104E0F7
:1028E0000920108004483230DEE7182010800548A7
:1028F000DAE70020D8E70000195C0108C05A010897
:10290000015B0108DD5B01080246032A08D2054885
:1029100050F8220000780880024850F822007047E2
:102920000020FCE7E801002000207047024803492E
:102930008860012070470000400200208C30002099
:102940001148007960B91048C078012808D10E48B4
:10295000C088082804D10D480B49886001207047C1
:102960000948007902280CD10748C078032808D10B
:102970000548C088082804DB054803498860012011
:10298000EDE70020EBE700008C300020E20C002097
:10299000FD1100200120704702488078024908702C
:1029A000012070478C3000204002002010B5044602
:1029B0001748007988B91648C07802280DD1144804
:1029C000C088012809D1134811498860007800F0B7
:1029D000010011490870012010BD0D48007902283E
:1029E00013D10B48C07803280FD10948C0880828A4
:1029F0000BDB24B90948064988600120ECE7074948
:102A0000002001F0FBFD0120E6E70020E4E70000E4
:102A10008C3000200C02002014020020FD0F00204A
:102A200008B501210804FAF777FB01214802FAF7FB
:102A300073FB01214802FAF79DFB00214FF400705F
:102A4000FAF798FB0120FAF77DFC0120FAF76EFCFB
:102A500002200D49086001210520FAF73FFC002003
:102A60000A49C872C87148720E208DF80000012012
:102A70008DF8010000208DF8020001208DF8030080
:102A80006846FAF74BF808BD404C01400040014051
:102A900000200D4908600D4908600D4908600D4986
:102AA00008600D4908600D4908600D4908600D492E
:102AB00008600D49086001200C4948700846C07A3A
:102AC00040F00100C87270471C0200202002002064
:102AD00024020020280200202C02002030020020C6
:102AE00034020020380200203C0200200040014057
:102AF000704700000146012931D11A4A9073002025
:102B00009074082010744020507408205074507441
:102B10001046C07940F00200D0710220907300206E
:102B20009074082010744020507408205074507421
:102B30001046C07940F00400D0710320907300204B
:102B40009074082010744020507408205074507401
:102B50001046C07940F00800D07101207047002075
:102B6000FCE700000040014010B500F0E9F910BD9D
:102B700010B54FF48020F7F7CBF92848006868B902
:102B80002748006800F0040040B101202349086094
:102B90002348006820F00400214908601F480068AD
:102BA00001280DD11E48006800F0010040B102204C
:102BB0001A4908601A48006820F0010018490860A6
:102BC00016480068022812D11548006800F002007B
:102BD00068B10320114908601148006820F0020024
:102BE0000F49086000200860232000F0FBF80B4824
:102BF000006890B90A48006800F0010068B103203D
:102C0000064908600648006820F001000449086091
:102C100000200860232000F0E5F810BD7C020020B1
:102C2000444C014070B50548847985780679324670
:102C300029462046F7F70CFE70BD00000040014019
:102C400010B52148007901283DD12048807C032817
:102C500039D100201E4908701C48807C032831D1DE
:102C60001A48407CD0B11B480078B8B100F02CF96C
:102C70001948407840F0040017494870322001F0AC
:102C800061FC1548407820F0040013494870FFF7B4
:102C900063F9FAF7EDF90120104908600B48807CD0
:102CA00003280FD10E48006803280BD100200C49DF
:102CB000086000F009F9FFF74FF9FAF7D9F9012098
:102CC0000649086062B610BD300A00208C30002032
:102CD000140200200100002000400140BC0200421C
:102CE0007C02002010B511480068114988421CD1AF
:102CF000FAF7BCF9FBF7EAFCF8F7C6FE642001F02E
:102D000021FCFFF74FF9FFF751F9002403E00A20F7
:102D100001F018FC641C142CF9DB06480649886194
:102D200000200249086000F07BF810BD1802002066
:102D3000A5A5A55AEB9C374A0000014010B51948DB
:102D4000007801282CD1002016490870012016496E
:102D50000870002015490870154908801548007949
:102D6000012801D1FFF7E2F813480078B0B102F072
:102D700055F802200F4981F8FA010020C1F8FC0142
:102D800005210C4890F8892100F5C5708154094847
:102D900090F88901401C074981F88901F6F7DCFDAC
:102DA00010BD00003B000020300000203A00002051
:102DB0000C000020300A00201F000020490050EACB
:102DC000C12018BF04204A0D18BF40F0010040F296
:102DD000FF72B2EB515F08BF40F00200012808BF4C
:102DE00005207047002817DB00F01F0201219140E9
:102DF0000A4A430942F8231000BF00BF00BFBFF3D7
:102E00004F8F00BF00BF00BF00BF00BF00BFBFF3B8
:102E10006F8F00BF00BF00BF7047000080E100E07F
:102E200000BF00BF00BFBFF34F8F00BF00BF00BF98
:102E30000948006800F4E06008490843001D06499D
:102E4000086000BF00BF00BFBFF34F8F00BF00BFCF
:102E500000BF00BF00BFFDE70CED00E00000FA0579
:102E600002F04CB940F2013200204FF0E04102F094
:102E7000D7BD0000024A0020110702F0D1BD0000BA
:102E800001FDFFFF2DE9F04105460E4614460127DE
:102E900072B60B48807C02280BD10A48006840B902
:102EA000092231462846FFF7C9FA01200549086082
:102EB000002762B6204600F0B9FC3846BDE8F08134
:102EC0008C3000203802002010B52320FFF78AFF45
:102ED000F9F7D8FE0220194908600120091F08608F
:102EE00000BF16480830006800F001000028F8D044
:102EF000012012492831086000BF10482C300068BA
:102F00000328FAD101200D4918390860F9F7B2FEFB
:102F10000220FAF7D9F90120FAF708FA012148024C
:102F2000FAF7FAF801210520FAF7D8F9FEF764FB61
:102F300040F26711C720FEF70BFD10BD50040140A1
:102F40001CB500210846FAF7C9F900214FF40070BA
:102F5000FAF7E2F80020FAF7E9F90020FAF7B4F9F5
:102F6000F9F790FE002026490860254928390860B5
:102F7000091F0860224940390860F9F77BFEFEF717
:102F80003BFB2621C720FEF7E3FCF9F77BFE182068
:102F90001B4918310860F9F76DFE01210804FAF7A2
:102FA000BBF84FF47060174908600846006800F4E9
:102FB0007060086001214FF40240FAF7EDF84FF419
:102FC0008020009000208DF8040008208DF8050076
:102FD00001208DF806006846F6F7A0FF00200A4998
:102FE00008602320002809DB00F01F020121914026
:102FF0004209920002F1E022C2F8001100BF1CBD9C
:1030000078040140444C01407C0200202DE9F0414D
:10301000C1F30A52A2F2FF362F4A304B0D46044646
:10302000142E2FDA002E12DA02F068F8002213466E
:1030300002F0B2FA4CD2002DBCBF4FF00045002484
:1030400046DB55EA040018BF254D19D140E0DFF8F2
:1030500094C02CFA06F705EA070C5CEA040C08BFDA
:10306000BDE8F08102F04AF80022134602F094FA1B
:103070002ED2002D03DD4FF48010F0400544BD43F7
:10308000002425E0332EC8BFBDE8F081A6F1140C62
:103090004FF0FF3727FA0CF73C4208BFBDE8F0813C
:1030A00002F0B0FA0022134602F076FA10D2002D98
:1030B0000DDD142E08BF6D1C09D0C6F134000121AE
:1030C00001FA00F02044A04238BF6D1C0446BC4306
:1030D00029462046BDE8F0819C7500883CE4377E97
:1030E0000000F03FFFFF0F0010B50024E74909780A
:1030F000491E01EB8102E6490978491E02EB0111E4
:10310000491C08034FF48072E249FEF78FF900BFB3
:103110000DE0E04904F10800085CDF490855DD498D
:1031200004F11C00085CDD490855601CC4B2142C75
:10313000EFDBD6490978491E01EB8102D4490978B1
:10314000491E02EB0111891C08034FF48072D1491A
:10315000FEF76CF900242EE004EB84000830CD4922
:10316000085C04EB8401CE4A1144487004EB8400EF
:103170000930C849085C04EB8401505404EB840016
:103180000A30C449085C04EB84011144887004EBE4
:1031900084000B30BF49085C04EB84011144C87003
:1031A00004EB84000C30BB49085C04EB840111443F
:1031B0000871601CC4B22A2CCEDBB4490978491EC0
:1031C00001EB8102B2490978491E02EB0111091D88
:1031D00008034FF48072AF49FEF728F900242EE06F
:1031E00004EB84000830AB49085C04EB8401AD4A71
:1031F0001144487004EB84000930A649085C04EBD4
:103200008401505404EB84000A30A249085C04EBAA
:1032100084011144887004EB84000B309D49085CE4
:1032200004EB84011144C87004EB84000C3099490C
:10323000085C04EB840111440871601CC4B22A2CA0
:10324000CEDB4FF4807293490020FEF7EFF89048F0
:103250000078904908708D48007848700020FEF78B
:1032600023F94FF480728B490020FEF746F94FF4A2
:10327000807288494FF4A040FEF7D8F88348007860
:10328000401E83490978491E032202FB01000221E6
:1032900001EB00107F49085C834908707B48007887
:1032A000401E7B490978491E02FB010002EB001019
:1032B0007849085C7D49087074480078401E74495C
:1032C0000978491E02FB0100042101EB001071493D
:1032D000085C774908706D480078401E6C49097891
:1032E000491E02FB0100052101EB00106949085C41
:1032F0007049087065480078401E65490978491E84
:1033000002FB0100062101EB00106249085C6A49DA
:1033100008705E480078401E5D490978491E02FB2E
:103320000100082101EB00105A49085C634908704C
:1033300056480078401E56490978491E02FB010094
:10334000092101EB00105349085C5D4908704F48A2
:103350000078401E4E490978491E02FB01000A21EF
:1033600001EB00104B49085C56490870474800784B
:10337000401E47490978491E02FB01000B2101EB61
:1033800000104449085C5049087040480078401ECD
:103390003F490978491E02FB01000C2101EB001096
:1033A0003C49085C4949087038480078401E384953
:1033B0000978491E02FB01000E2101EB001035497E
:1033C000085C08B1012000E00020414908702F4846
:1033D0000078401E2E490978491E032202FB010095
:1033E000072101EB00102B49085C3A4981F80102E2
:1033F00026480078401E26490978491E02FB010034
:103400000D2101EB00102349085C324981F80202CA
:10341000012031490870FF203049087004203049EC
:103420000870F12048701A480078887017480078B2
:10343000C8701D48007808711C48007848711C4805
:10344000007888711B480078C871002008720A2033
:1034500001F078F82348007840B90420204908702A
:10346000042215211E4801F023FC0DE00422152141
:103470001B4801F01DFC50211B48F3F78AFF012275
:103480001521194801F014FC10BD000013020020A2
:10349000120200208C2D0020DE130020F2130020E9
:1034A000741A0020461B0020B9020020A802002048
:1034B000A9020020A6020020B102002098090020E5
:1034C000AB020020D3020020A7020020B20200209D
:1034D00021000020300A0020C2020020200000202D
:1034E0004B0D00201F000020E20C002010B5044608
:1034F0000B2207A12046F3F7B7FE20B900200749A9
:1035000081F8F80103E00120044981F8F80110BDB9
:10351000474D4D4B204E756D70616400300A0020A0
:1035200010B50446042233A12046F3F79DFE50B99E
:10353000062032490870002031490880FF203149B7
:1035400081F8FA0149E004222FA12046F3F78CFE0E
:10355000A0B903202949087000202D4908802D4971
:10356000088001202C4908702C490870FF2025494B
:1035700081F8FA01002081F824022EE0042228A11B
:103580002046F3F771FE88B907201C490870002017
:1035900025490880254908701A4890F8FA01FF2843
:1035A0001BD10120174981F8FA0116E0042220A15D
:1035B0002046F3F759FE18B90220104908700CE0B4
:1035C00004221DA12046F3F74FFE30B900200B491D
:1035D0000870FF200B4981F8FA010120094981F8A0
:1035E000240108462168C0F826116168C0F82A1134
:1035F00010BD00003030303200000000B60900205D
:1036000070020020300A002030303034000000000A
:103610006C02002074020020B40900201F0000206A
:103620003030303800000000760200201402002004
:103630003030343000000000303030310000000005
:103640002DE9F04104460E4617460025A8464FBB1B
:103650003248407806F0EF01E03908432F494870BE
:10366000702C11DC2E48005D05092D48005D00F02E
:103670000F010120884000F0FF082848405D40EA23
:1036800008002649485538E004F0E000E02834D12D
:103690002248407804F00F020121914008431F495D
:1036A00048702AE0012F28D11C48407806F0EF012D
:1036B000E039884319494870702C11DC1848005DC6
:1036C00005091748005D00F00F010120884000F057
:1036D000FF081248405D20EA0800104948550CE0F8
:1036E00004F0E000E02808D10C48407804F00F0214
:1036F000012191408843094948700A48007818B967
:103700000A200649087002E00520044908700522D5
:103710001521024801F0CCFABDE8F081320D0020FD
:10372000985D01081F00002070B504460E4615463E
:1037300055B9104810F814000F4948700D4800EBB7
:1037400044004078887005E0012D03D100200A492B
:10375000487088700948007818B903200649087035
:1037600002E002200449087002221521024801F0FB
:103770009FFA70BD1C5E0108F40100201F000020AC
:103780002DE9F04105460E461446012772B60B4856
:10379000807C02280BD10A48006840B908223146D3
:1037A0002846FEF74BFE012005490860002762B657
:1037B000204600F03BF83846BDE8F0818C30002010
:1037C0002002002001460A8840F62B039A4201DCC1
:1037D0001A460A800A8840F608239A4201DB1A46F4
:1037E0000A800A88A2F62B0264235A4340F2DD13B2
:1037F00092FBF3F290B2642800DD642000B900BFB0
:103800007047014631B1012906D0022906D00329AB
:1038100008D105E0012007E0022005E0042003E0D4
:10382000082001E0012000BF00BF7047034A10706C
:1038300000BF024909780029FBDC704744020020E0
:103840001348008813490988884201D1C82070476D
:103850000F4800880F490988884209DD0C48008814
:103860000C490988401A401CC0F1C80080B2EEE73C
:103870000748008807490988884207DA0548008810
:1038800003490988401A401E80B2E0E7C820DEE7FD
:10389000B0090020B20900202DE9F05F04468A46F5
:1038A00093461A48007818B119480078012802D1C7
:1038B0004FF0190926E0CAEBCA0000EB4000154999
:1038C000084410F80B90422C0DDD484601F016FD1F
:1038D0000746114A114B01F061FD054601F0CAFC93
:1038E00000F0FF090EE0212C0CDA484601F006FD3D
:1038F0000546094A0A4B01F051FD074601F0BAFCA2
:1039000000F0FF094846BDE8F09F000030000020AD
:1039100034000020590000209A9999999999E93F1B
:103920009999F13F0E480078012808D10D48008888
:103930000D490988884210DD0A4800887047094807
:10394000008809490988884207DA06480088401E2D
:103950000449088008460088F0E703480088EDE73E
:1039600035000020120000201400002010B54FF494
:1039700000510548F6F75CFF08B9012010BD002092
:103980000249086000BFF9E7000800407802002003
:103990002DE9F04D21F0004423F0004786B0824627
:1039A0001546A74204DDAA46054620463C46074682
:1039B000E01BA3463E46B0F1707F08DD06B02A4604
:1039C0003B4650462146BDE8F04D01F097BB8F487D
:1039D0004FF00008844240DD8D48A04235DC2A4685
:1039E0003B4650462146FFF73BFABAF1000F14BFA1
:1039F0000122002202EB4403864A13F5001F04D97A
:103A00009442BCBF06B0BDE8F08D002D14BF012369
:103A1000002303EB470313F5001F04D99742BCBFF3
:103A200006B0BDE8F08DC4F3130252EA0A0204BFE7
:103A30005046594687F07F6282F0E0422A4304BF35
:103A40002846314606B0BDE8F08DABF11654A6F11C
:103A500016574FF41678A3463E46B7F10C5F29DAA5
:103A6000B7F5801F1EDA55EA060001BF5046214611
:103A700006B0BDE8F08D0022674B17461C4628466D
:103A8000314601F08BFC05460E463A462346504629
:103A9000594601F083FC82468B460C463746A8F215
:103AA000FE3807E00BF1165406F11657A3463E46C2
:103AB000A8F516782A463B465046594601F094FE32
:103AC0002A463346CDE9000101F066FD2ED20027DB
:103AD0003A4623465046594601F086FECDE900019C
:103AE0003A4623465046594601F008FBDDE90023DB
:103AF00001F054FC82468B46284686F0004102467F
:103B0000334601F04BFC52465B4601F06DFE054624
:103B10000E463A4623461046194601F03FFC2A4617
:103B2000334601F061FE01F0B9F945E0012250464B
:103B3000594601F075FFCDE90401002292463B464B
:103B4000BB462846314601F04FFECDE90201DDE9D2
:103B50000401002704F580143A46234601F044FE90
:103B60002A46334601F01AFCDDE9022305460E46DB
:103B70003846214601F012FC2A46334601F0BEFACF
:103B800005460E46DDE9000181F000410246019B39
:103B900001F004FC33462A4601F026FE05460E4697
:103BA00052465B463846214601F0F8FB2A4633462A
:103BB00001F01AFE01F072F9B8F1000F04BF06B06F
:103BC000BDE8F08D4FF0000C144A08EB115340F2A1
:103BD000FF74A34207DB0220F3F72CFC06B0BDE81C
:103BE000F04DFFF73FB902EB0853624601F0D6FBF8
:103BF00004460D46FFF7E2F8042808BFFFF73AF93C
:103C0000204606B02946BDE8F08D00000000305F78
:103C10000000F07F0000F87F0000D07F0000F03F40
:103C2000014601F4004008B1002070470120FCE784
:103C30002DE9F84304460E46914600270025A84684
:103C4000B9F1000F50D17B480078012827D106EB4D
:103C500084007949085C79490F5C06EB8400764959
:103C6000085C77490D5C7748007878B9062D0DD14E
:103C70000E2F02D101253A2708E00F2F02D101258E
:103C80003B2703E0102F01D101253C276E4800EBB4
:103C9000840087556D4800EB840085552CE006EBC9
:103CA00084006549085C6A490F5C06EB8400624940
:103CB000085C68490D5C29463846F4F7BBF8804635
:103CC000B8F14C0F02D14746012504E0B8F1000FCE
:103CD00001D0474606255C4800EB840087555B48C9
:103CE00000EB8400855507E0574800EB8400875DB2
:103CF000564800EB8400855DFF2F0CD114225649F5
:103D00005348F3F701FB142254495248F3F7FCFAE5
:103D10000020BDE8F88367B95DB914224E494C48CC
:103D2000F3F7F2FA14224D494A48F3F7EDFA00206E
:103D3000EFE74B4890F8FA01022804D100204849E7
:103D400081F8240208E0464890F82402012803D1B3
:103D50000220434981F82402012D01D0022D04D113
:103D60004A460121384601F0BFF8032D05D14A46E5
:103D700029463846FFF7D8FC59E0052D07D13346D0
:103D80004A4629463846009400F022F94FE0062DB5
:103D900005D14A4629463846F6F736FA47E0072D58
:103DA00005D14A4621463046F3F748FE3FE0082D4C
:103DB00005D14A4629463846F9F724F937E0092D56
:103DC00005D14A4629463846F8F74CFE2FE00A2D21
:103DD00023D1B9F1000F1AD106EB84002149085C08
:103DE00021490978884206D006EB84001D49085C09
:103DF0001D49087002E0FF201B4908701B4800881D
:103E000028B10020194908801949487088704A462D
:103E100021463046F3F712FE09E005F0E000E02805
:103E200005D105F0EF014A463846FFF709FC284660
:103E30006FE70000A1020020345D0108845D0108E5
:103E4000705D0108AE0200202E14002042140020F4
:103E5000F2130020DE1300205C5D0108485D0108BC
:103E6000300A0020AC5A0108200000202A0000205F
:103E7000F40100202DE9F04107460D4616464FF0AB
:103E80000108002415480078012805D1144800785D
:103E900000F077001249087072B61248807C022840
:103EA00015D11148006890B9082229463846FEF716
:103EB000C5FA01200C4908604FF00008002404E016
:103EC000295D0A480155601CC4B2082CF8DB62B6B3
:103ED0003046FFF7ABFC4046BDE8F081A802002069
:103EE000E20C00208C3000201C020020480A002038
:103EF00000B595B0334800883349098888425FD0BF
:103F000030480088C0EBC00000EB40002F49085C3F
:103F100004283FD005DC58B101281DD003284DD11D
:103F200010E0072840D00A2820D0132846D127E0E7
:103F3000152101A800F01EFB022201A98120FFF734
:103F400099FF3CE0152101A800F014FB022201A911
:103F50008220FFF715FC32E0152101A800F00AFBD2
:103F6000022201A9822000F07BFA28E0152101A895
:103F700000F000FB022201A9822000F093FA1EE06B
:103F8000152101A800F0F6FA022201A9822000F012
:103F900067FA14E0152101A800F0ECFA022201A949
:103FA0008220FEF76FFF0AE0152101A800F0E2FA77
:103FB000022201A98220FEF765FF00E000BF00BFDA
:103FC00015B000BDB2090020B0090020A0300020CB
:103FD0002DE9F0410546884614461E46069F002CF2
:103FE00032D12148007858B92048057006EB870087
:103FF0001F49085C1F49087001201F4908702BE009
:104000001E480078012801D11B490870002016497C
:1040100008701B490870012007E01A49095C11B1BA
:104020000121194A1170411CC8B21028F5DB01208A
:1040300007E01649095C11B10121134A1170411CB6
:10404000C8B20828F5DB07E0012C05D1104800882C
:1040500010B9002009490870F8F7B6FC00200D4996
:104060000860BDE8F08100009C0900209A0900204A
:10407000345D0108A50200209B0900209F09002053
:104080009D090020A40F0020A209002004020020A6
:10409000A0090020600200200025CE48CE4908601B
:1040A000FDF7AAFA4FF44070F8F770FDFDF77EFFB8
:1040B000F5F704F8F3F704FFFDF7F2FEF8F770FDEB
:1040C000FEF7E6F9FDF732FFF5F746FC80E1F4F77D
:1040D000DBFFF5F7F9FFFCF797FFF3F76BFABF4843
:1040E0000078082803DB0820BC49087006E0BB48BC
:1040F0000078022802DC0220B8490870B84800683D
:10410000B6490978884210D30020B64981F80802E0
:10411000B5480078012801D1F6F7F8FBF4F7D0FD97
:10412000F6F746FC0020AE4908600321022000F0AB
:10413000C9FC0021084600F081FC00F01FFD00F0E2
:10414000D7FBF5F7C9FDFEF7F9FDA64890F8240165
:10415000012803D10020A34981F82401F4F746FF88
:10416000F4F7C8FEFCF752FCF5F704FAF5F728F867
:10417000F3F7BEFEF5F758F9F4F7DAFEF4F720FF8F
:104180009A4800689A490988884204D300209749D0
:104190000860F8F719FC97480078012809D196487B
:1041A000007830B90020934908709449012000F04C
:1041B00025FA93480078012804D10020904908701E
:1041C000F3F7FCFC8F480078012804D100208D49CA
:1041D0000870F3F78FFC8C480078012806D1002086
:1041E00089490870F5F7F0F8FEF77EFF87480078F8
:1041F000012806D1002085490870F5F7B5F8FEF7CB
:1042000073FF83480078012804D10020804908709A
:10421000F6F70EFD7F48007820B1FBF759FE00202D
:104220007C4908707C480078012804D100207A4934
:104230000870F6F7E7FFF4F7D3FC78480078012818
:104240000AD1002075490870F6F746FEF7F728FCFA
:10425000F7F72CFDFBF71EFF71480068052806D311
:1042600000206F490860F6F787FDF6F7EDFDFDF7D2
:1042700047F86C4800686C490988884204D30020DC
:1042800068490860F6F756FE6848007858B16748F4
:104290000078012807D065480078072803D06348D4
:1042A0000078112802D10120614908706048007827
:1042B00010B901205E4908705E4800885C490978A1
:1042C0004843142190FBF1F05A4909780844C5B2DB
:1042D00059480068A8421ED3002057490860424848
:1042E0000078012817D1F7F7D9F954480078012848
:1042F0000DD153480078012809D15248007801288F
:1043000005D10723002211461046FCF71BFE0120B1
:10431000344981F81D024C4800684C4909788842AC
:104320001DD300204849086049480078B8B92E4894
:104330000078012813D147480088F6F79BFCF6F770
:104340004BFFF6F735FEF6F753FFF6F71BFEF6F7D1
:10435000EFFCF6F7FFFCF6F7D5FCF7F795FB3E48C8
:104360000078032816D13D48006840F6B8318842ED
:1043700010D3002039490860FAF7A8F9F7F784FB51
:10438000002403E00A2000F0DDF8641C0A2CF9DBAD
:10439000F5F7E2FA134890F80002012814D1FAF771
:1043A00095F9F7F771FB002403E00A2000F0CAF842
:1043B000641C0A2CF9DB032027490870F5F7CCFAB6
:1043C0000020084981F80002FEF73AFCFEF78AFC5B
:1043D0007DE600000070000808ED00E0AB02002060
:1043E00048020020300A0020300000206002002037
:1043F000A40900204E0000204F000020540E002091
:104400000F020020100200209602002099020020D6
:104410009F020020AD0200209E020020C202002068
:104420005402002058020020C6020020B9020020D9
:10443000B3020020C402002050020020A602002087
:10444000A7020020140200205C020020C802002005
:104450003400002014000020A00200206802002088
:104460002DE9F04105460E461446012772B60B4869
:10447000807C02280BD10A48006840B908223146E6
:104480002846FDF7DBFF012005490860002762B6DA
:104490002046FFF7CBF93846BDE8F0818C3000208C
:1044A000280200202DE9FF4107460D4616464FF031
:1044B00001080024002000900190029003901C4805
:1044C0000078012805D11B48407800F07700194991
:1044D000487072B61848807C022821D117480068BD
:1044E000F0B9002007E0295C124A125C11430DF874
:1044F0000010411CC8B21028F5DB1022694638466E
:10450000FDF79CFF01200D4908604FF000080024D2
:1045100004E01DF804100A480155641C102CF8D35F
:1045200062B63046FFF782F9404604B0BDE8F0813C
:10453000A8020020561400208C3000202C020020FD
:10454000980A002000B5034605E04FF4C36000F070
:1045500005F8581E83B2002BF7DC00BD07E00721E9
:1045600001E04A1ED1B20029FBDC421E90B20028B5
:10457000F5D1704770B504460D461D480088C0EB64
:10458000C00000EB40001B4A81182A462046F2F783
:10459000BBFE1948007848B9207828B92A46611C22
:1045A0002046F2F7B1FE00E000BF0AE020780128C3
:1045B00005D12A46611C2046F2F7A6FE00E000BFA6
:1045C00000BF0B490988C1EBC10101EB4101094A58
:1045D00088181521F2F7DDFE05480088401C0449C3
:1045E000088008460088C82801DB0020088070BDCC
:1045F000B2090020A03000201F00002070B5054641
:104600000C4615B92078072801D0012D7ED160789D
:10461000012817D1A078032814DC4FF480722146BA
:10462000A348F2F771FE0120A24908700720A249B1
:1046300008706078A1490870A078A1490870E078F6
:10464000A04908706078012806D1A078FF2803D11E
:1046500001209D4981F800026078022816D1C2012C
:1046600021469348F2F750FE012092490870042039
:1046700091490870607891490870A0789049087055
:10468000E078904908702079904908706078032894
:1046900013D14FF4807221468548F2F735FE012090
:1046A0008449087084490870607884490870A0784B
:1046B00083490870E07883490870607883280DD1B9
:1046C0000120834908707C49087060787B49087034
:1046D000A0787B490870E0787A49087060780428EF
:1046E00013D1820121467248F2F70EFE0120714972
:1046F0000870032070490870607870490870A078CD
:104700006F490870E0786F49087000E0CFE060788A
:10471000052811D14FF4807221466548F2F7F4FD67
:104720000120644908700220634908706078634979
:104730000870A078674908706078062814D14FF493
:10474000807221465A48F2F7DFFD0120594908706E
:10475000062059490870607858490870A07858496F
:104760000870E07857490870607807280ED14FF438
:10477000807221464E48F2F7C7FD01204D4908706E
:1047800005204D49087060784C4908706078082809
:104790002BD1420121464648F2F7B6FD607A4E49D8
:1047A0000870012043490870082043490870207AA6
:1047B000FFF727F849490870002011E000210BE0BD
:1047C00000EB40020B320A44A25C00EB4003444E73
:1047D00033445A544A1CD1B20329F1DB411CC8B2FC
:1047E0000328EBDB00203F4908606078092814D1DA
:1047F0004FF4807221462E48F2F786FD01202D49A4
:10480000087009202C49087060782C490870A0783D
:104810002B490870E0782B49087060788A2805D108
:1048200001202B4908700A2023490870607830283D
:1048300002D12D482D49086060781A280CD101203A
:104840001C4908701A201C4908702179E07801EB96
:1048500000201D49A1F8260260781B280CD10120F8
:10486000144908701B20144908702179E07801EB85
:1048700000201549A1F8280260781C2805D10120E4
:104880000C4908701C200C49087060788F2805D1ED
:1048900001200F4908700F200749087060784428EC
:1048A00005D101200349087044200349087070BDF8
:1048B000FD1000200F020020110200200D02002038
:1048C0001202002013020020300A00200E020020F5
:1048D000100200201602002015020020C90200204C
:1048E000CA02002008000020A5A5A55A1802002031
:1048F00010B54348007888B942480088B0F5967FE3
:1049000007DB00F049FB01203D49087000203D49CC
:1049100008803D4800883D4908806FE03C480078A9
:10492000012819D137480088B0F5967F66DB3648F4
:1049300000885F2802DB0120364908703248008871
:10494000324908800020324908702E4908802E48DC
:1049500000882E49088051E0FFF708F82E490870BA
:10496000294908782D490A782D490978FEF794FFDE
:104970002C49087028480078012819D10846007889
:10498000C0F5FA70284991FBF0F02849096888427F
:1049900023D80020254908601B480088401C1A497C
:1049A000088008460088642817DD6420088014E029
:1049B000194800781E490978884209D012480088B1
:1049C0001249088001201249087000200D49088012
:1049D0001848FEF7F7FE0C4908800F480078144984
:1049E000087015480078012804D107480088074955
:1049F000088003E0FEF796FF0449088010BD000020
:104A00003A0000200C0000201200002014000020BA
:104A1000380000203700002035000020B0020020C0
:104A2000B90200205800002000A24A0478020020A9
:104A300036000020880200203900002070B50446AE
:104A40000D461A480078012802D002282BD10BE02D
:104A500017480088B0F5966F05DB164800780128E6
:104A600001D1154908701FE011480088B0F5966F14
:104A700011DA002229462046FFF7DAF80F490870BC
:104A8000012229462046FFF7D3F80C490870002080
:104A90000B4981F811020020074908700449088079
:104AA0000249087000E000BF00BF70BD1A0000207E
:104AB0001C00002030000020A10200202F00002058
:104AC000300A002070B504460D46244800780128BD
:104AD00006D002281BD0032803D004283AD12DE0A9
:104AE00000BF1F48008840F68C2188420EDB1D481D
:104AF0000078012802D11C49087002E001201B49FE
:104B000008700020154908701549088023E01448F2
:104B10000088B0F5FA7F10DB002229462046FFF717
:104B200087F813490870012229462046FFF780F8CC
:104B30000F4908700020094908700CE00948007806
:104B4000012803D10B4908700B4908700020034964
:104B5000087000E000BF00BF70BD0000160000201C
:104B600018000020300000203C0000203B00002006
:104B70002F000020970200209902002010B5434822
:104B8000B0F8260242490988884207DB3F48B0F85E
:104B900026023F49088000203E4908803B48B0F883
:104BA00028023B490988884208DC3848B0F82802C6
:104BB0003749088064203749088012E03348B0F84C
:104BC00028023249B1F82612411A3048B0F82602BC
:104BD0002F4A1288101A6422504390FBF1F02D499D
:104BE00008802D4800882B49098888424CD02B48E2
:104BF000008840F6B831884246DB04202849087016
:104C0000F8204870322088700020C8702148007851
:104C100008711F480088000A48711D480078887193
:104C20000020C87108721F48007838B90420087045
:104C3000042215211A4800F03BF817E00422152140
:104C4000174800F035F8114890F8FA01022804D10D
:104C500000200E4981F8240208E00C4890F8240254
:104C6000012803D10220094981F82402094800885B
:104C7000094908800C480078012802D100200A491F
:104C8000087000200949086010BD0000300A0020AB
:104C9000860200200E0000201000002002000020EC
:104CA000420D00201F0000203400002008000020DA
:104CB00070B505460E461446002034490870344845
:104CC000007870BBACB9002032490988C1EBC10142
:104CD00001EB4101304A50542E490988C1EBC10112
:104CE00001EB41011144481C32462946F2F70CFB06
:104CF0000BE028490988C1EBC10101EB4101264ABB
:104D0000881832462946F2F7FFFA22480088401CEC
:104D10002049088008460088C82836DB0020088023
:104D200033E0FFE71D48007803282ED1012C15D170
:104D3000012018490988C1EBC10101EB4101164A64
:104D4000505414490988C1EBC10101EB41011144E0
:104D5000481C32462946F2F7D7FA0BE00D4909887C
:104D6000C1EBC10101EB41010B4A881832462946CB
:104D7000F2F7CAFA07480088401C0649088008462E
:104D80000088C82801DB0020088070BD5100002089
:104D90001F000020B0090020A0300020B60900202C
:104DA00070B5054600244FF480718805F5F74CFD79
:104DB0001420F5F721F84120154988705421144832
:104DC000C1702B21017100201249088000BF0FE043
:104DD00000BF1148FDF71FF800F020000028F8D0B0
:104DE0000B48801C015D0C48FDF758F8601CC4B2EC
:104DF000AC42EDDB00BF0848FDF70DF800F04000C5
:104E00000028F8D04FF480718805F5F71AFD70BDC1
:104E100008410020000A00200038004010B500249E
:104E200000201B4908804FF480718805F5F70CFDC0
:104E30001420F4F7E1FF41201649887054211548E9
:104E4000C1700D2101710A21417100BF0FE000BF47
:104E50001148FCF7E0FF00F020000028F8D00D48D2
:104E6000801C015D0C48FDF719F8601CC4B2042CCD
:104E7000EDDB00BF0848FCF7CEFF00F04000002843
:104E8000F8D04FF480718805F5F7DBFC10BD000009
:104E9000000A002008410020003800402DE9F041C0
:104EA00006460F4600F0BAFB041E0D4618BF01204F
:104EB000284320F00040C0F17F6000F1E040C00FC7
:104EC0000ED0301C18BF0120384320F00040C0F144
:104ED0007F6000F1E040C00F04BF0120F2F7AAFAA2
:104EE00020462946BDE8F0812DE9F04105460F46F0
:104EF0001646F6B9E02D0BDBE72D09DC23480078D8
:104F0000A5F1E00101228A401043204908702CE0FD
:104F100002240BE01D48005DA84200D108E01B48B8
:104F2000005D10B91948055502E0641C502CF1DBF6
:104F30001BE0012E19D1E02D0BDBE72D09DC134816
:104F40000078A5F1E00101228A4090430F490870E2
:104F50000BE0022407E00D48005DA84202D10020CA
:104F60000A490855641C502CF5DB0948007828B91B
:104F7000002215210548FFF79BFE04E001221521C0
:104F80000248FFF795FEBDE8F0810000E20C00202A
:104F90001F0000207047704710B500240FE001206B
:104FA0000B490870012211460020F2F7ABFC0120EA
:104FB000F2F722FD1420F4F71FFF601CC4B2102C7E
:104FC000EDDB0448FEF7FEFB0349088010BD00003E
:104FD0002E000020880200201200002030B5132887
:104FE0004BD009DC0B286AD2DFE800F069192530C4
:104FF0003169693C1A2632001B2834D008DC142899
:105000003CD015280DD019284ED01A2857D140E091
:105010001C283FD0262848D0272850D12FE000BF99
:1050200000BF2D4C247B0C702B4C647B14702A4CDD
:10503000A47B1C704DE000BF274CE47B0C70264C19
:10504000247C1470244C647C1C7042E000BF00BFC0
:10505000214CA47C0C70204CE47C14701E4C247DEC
:105060001C7036E000BF1C4C647A0C701A4CA47A99
:105070001470194CE47A1C702BE000BF00BF164C72
:10508000A4790C70144CE4791470134C247A1C70BD
:105090001FE000BF104CE4780C700F4C24791470A2
:1050A0000D4C64791C7014E000BF0B4C24780C701C
:1050B000094C64781470084CA4781C7009E0064C04
:1050C000E47B0C70044C247C1470034C647C1C70D6
:1050D00000BF00BF30BD00008C60010810B54FF468
:1050E00080718805F5F7B0FB1420F4F785FE4FF4C6
:1050F00080718805F5F7A5FB10BD000010B591EA99
:10510000030F48BF83F0004300F17683841A71EBEC
:10511000030C05D2121943EB0C03001B61EB0C01CD
:10512000DFF824E14FEA1154A4EB135C1EEA430FAD
:1051300018BF9EEA445F73D023EA0E03DCF1200E11
:1051400021EA045143F4801332D322FA0CFE10EB0F
:105150000E0023FA0CFE41EB0E01CCF1200E03FAF7
:105160000EFE10EB0E0051F10001B1F5801FCCF1E5
:10517000200E32D201EB045112FA0EF2BDE81040BB
:1051800058BF7047401C38BF5FEA420218BF7047E3
:10519000002814BF20F0010041F100014FEA410353
:1051A00013F5001F38BF7047A1F1C04100F0EEB900
:1051B000012A43EB0302ACF1200CDCF11F0E32BFDD
:1051C0004FF0000E23FA0CF310EB030041EB0451F7
:1051D000B4EB115FD0D0A1EB045101F58011490867
:1051E0005FEA300001EB04510ED350F1000038BFEC
:1051F00012FA0EFE08D1BDE81040C9E7401C38BFC6
:105200005FEA4202CAD1C3E7BDE810404FEA41035A
:1052100013F5001F38BF7047A1F1C04100F0B6B9C7
:105220009EEA445F08D011EA5E0FBDE8104004BF5B
:1052300001F0004100207047BDE8104070B500F05B
:1052400057F900BF64FBBE3E0000E0FF02494FF08B
:10525000000000F0B3BB00BF0000F87F491058BF4A
:10526000C1F140415B1058BFC3F140438B42EFF3A3
:10527000008070474FEA1153A3F58063D3F11E03FA
:10528000A8BFD3F1200C08DB4FF0004242EAC12254
:1052900052EA505232FA03F0704709420BD4102BF5
:1052A000C4BF0020704703F5787CBCF1FF3F05D0F8
:1052B0004FF0FF3070474FF00000704770B500F0BE
:1052C00017F900BF4992248000207047F0E710F0E2
:1052D000004248BF4042B0FA80F310FA03F10AD00E
:1052E000C3F11D0303F580634FEA415002EB035203
:1052F00002EBD12170474FF000007047B0FA80F305
:1053000010FA03F10AD0C3F11D0303F580634FEADD
:1053100041504FEA035202EBD12170474FF0000099
:105320007047000051EA030C17D41CF5801F58BFCA
:10533000BCF5801F00F10680994218BF704708BF76
:105340009042704707D711F5801F58BF13F5801F93
:1053500019D499427047894270471CF5801F08D5BF
:10536000BCF5801FF7D58B4218BF704708BF82423B
:1053700070474FF4001C1CEB410F38BF1CEB430F70
:1053800001D28B42704770B500F0B2F89224490008
:105390004FF000514FF08053FFF760BFDFF848C176
:1053A00070B51CEA111E1EBF1CEA13159EEA0C0FF5
:1053B00095EA0C0F00F06F8081EA030423EA4C1396
:1053C0004EEAD47E21EA4C1141F4801143F480135B
:1053D000AE44A1FB024CA0FB0365AEF17F7E361903
:1053E00055EB0C05A1FB034C4CF10003A0FB021C88
:1053F00016EB0C06654153F10003094218BF46F055
:10540000010613F4007F0BD14FEA03314FEA053058
:10541000340341EA155140EA16506FF003020AE0E6
:105420004FEAC3214FEAC520F40241EA555140EA50
:1054300056506FF0020202EB2E4201EB025585EA54
:10544000CE710AD05FEA440C18BF24F0004450F13A
:10545000000041F1000120EAD47040F2FE7C624578
:1054600000D270BDA84214BF4FF080444FF04044BA
:10547000002E08BF0024BEF1806FA8BFA1F1C0417B
:10548000BDE8704080F282804FF0000001F1C04121
:1054900001F0004170479EEA0C0F0CEA131518BF8B
:1054A00095EA0C0F06D04FF0000081EA030E0EF0D3
:1054B000004170BD00F01CF88900013E00F007B803
:1054C00000F009B84FEA430C5FEA5C5C08D081EA5F
:1054D000030100F05BB84FEA410C5FEA5C5CF6D177
:1054E0004FF00000014970470000FF070000F87FFF
:1054F0000EF1020E2EF0030E5EF8046B364205D458
:10550000012A43EB030515F5001F12D8012841EBD2
:10551000010C1CF5001F0CD80ED14FEAD17C15F5FB
:10552000001F0CEB4C0C0CF1020C08BF4CEBD37CB5
:1055300004E04FF0080C01E04FEAD37C0CEB4C0583
:1055400026FA05F606F00706B6F1040C06D20EEBB5
:10555000860CBDE870404CF0010C6047DFE80CF0B1
:10556000090B02024FF000414FF00000A1F50021AD
:1055700070BD19461046012851EB010418BFD4F53F
:10558000001484BF002001F0004170BD0808A0F5A0
:1055900000114FEA3101704753EA010C17D41CF592
:1055A000801F58BFBCF5801F00F106808B4218BFDA
:1055B000704708BF8242704707D713F5801F58BF56
:1055C00011F5801F19D48B4270479B4270471CF520
:1055D000801F08D5BCF5801FF7D5994218BF7047CA
:1055E00008BF904270474FF4001C1CEB430F38BFBC
:1055F0001CEB410F01D2994270470FB40CBC03BCA5
:10560000FFF7C1BE91EA030F10B581F000413FF5ED
:105610007DAD83F0004300F0EFB800002DE9F041CC
:1056200001F5801CBCF5001FC0F2C3804FEA115C7D
:1056300021EA0C510CF1FD0C41F480115FEA5C0C85
:105640000CF5C07C01D3400049413DA4890241EAE8
:10565000905187028E0E0A0CA45D04FB04F602FB37
:1056600006F6C6F14046A4FB0662F60D46EA42265F
:1056700006FB06F4A4FB01235242C3F1404338BFAA
:105680005B1EA6FB02420024E6FB0324D20B42EA87
:105690004446A6FB0623A1FB02E2A3FB07E4A418F1
:1056A0004FF0000252F10002E3FB01426442C2F1FA
:1056B000404E38BFAEF1010EA6FB04234FF00002AE
:1056C000E6FB0E32A2FB03464FF00004B61954F17C
:1056D0000004E2FB0264A1FB06E6A4FB07E816EB6C
:1056E00008064FF0000858F10008E4FB0168764214
:1056F000C8F1405838BFA8F10108A2FB06E4A3FB9B
:1057000008E52D194FF0000454F10004E2FB0854A1
:10571000A1FB05E6A7FB04E818EB06084FF000061E
:1057200056F10006E1FB048618F1200556F100064B
:10573000A809A8F11B08B10908F03F08B8F10A0F41
:1057400040EA86601CD901EB0C51BDE8F08100BF36
:10575000FCF5EEE8E2DDD8D3CFCBC7C3C0BDB9B608
:10576000B4B1AEACA9A7A5A3A19F9D9B9A9896950D
:105770009392908F8D8C8B89888786858483828194
:10578000A0FB006800FB01F208EB4208B8EB872899
